:020000024000BC
:100000006FD0A23B00000000001801180028012852
:100010000228032800290129022903290429052986
:10002000062907290829002A012A022A032A042A64
:10003000052AA62AD8DF0600F24004006804002042
:10004000EA040020EA030020B80300205003002047
:10005000B42900208A410400AC4204004245040057
:100060005C4604004A400400F83F0400B40200204B
:1000700054020020384B04001C080020604104009A
:1000800034480400DE790600C47B06002A7C0600A2
:100090002C5506006655060000850500DA79050036
:1000A000FC73060062480400045D060012FA0400B6
:1000B000A0FA0400FEFA0400305304006E5304005A
:1000C000E451040020BC040006B70400CE2A00203E
:1000D00044C8040096CB0400A8A904004AA904005F
:1000E00016AD0400F4A9040028A90400A0A9040086
:1000F000DEA8040076AA0400CEAA04007EAA0400AA
:1001000082AA040010AB0400D6AA040006AB0400C7
:10011000E8AF0400ECAF040072AA04007AAA04005D
:100120000EAB0400EAAF0400BCAB040048B104000D
:1001300044D90400B6D90400F0D9040066BE040016
:100140007CBE0400B6BE0400C09E0400C6A004002D
:100150008EA10400D07004001A6B0400D494040033
:10016000966B04008A90040018B906004EB1060090
:1001700054B6060090CD06005ACC0600B2D0060058
:100180006ED00600AAD00600FED106000AA0060026
:100190008ED10600ECC3060012C4060032C406006D
:1001A0006ED206004ECA0600E6C90600DED2060080
:1001B0008EA2060026A3060046A30600F8A20600AB
:1001C000385D0500CA470500464B05000649050095
:1001D00058530500A0740600947306003EA0060064
:1001E000BA4C04007C560600E45C0600DC5D0600A8
:1001F000EA6B0600726C0600D06D060020C2040097
:100200003A5C0500005405009A450500AA56050011
:100210007A470500DC09002054570600D8D00600B4
:1002200072D00600A6D00600A2D00600C244040088
:100230009EBF0400E0D00600606006002661060054
:100240008E610600BCB60600DCD0060026D1060092
:100250005C7905002AD10600662000202C200020B1
:100260009CB6060032B806002ED1060082D10600E8
:1002700086D10600E4D006001ED1060022D1060079
:100280008AD10600F05C05000000000000000000BC
:10029000000000000000000000000000000000005E
:1002A000000000000000000000000000000000004E
:1002B000000000000000000000000000000000003E
:1002C00097470000938787D2174700001307875589
:1002D0006373F700828023A007009107D5BF97477B
:1002E0000000938727C317E706E0130727379746D1
:1002F00000009386A6CF63F3F600828010431107B7
:0603000090C39107CDBF80
:100308004111B7E700E022C480433707200006C642
:10031800798C23A0E7180F10000011C199E5B7E701
:1003280000E023A08710014579A80D05334505088D
:10033800130740037199B34705086366A702174579
:1003480000000325A5CA9746000083A6A6C96391A5
:10035800A602174700000327E7EB71D3C207DD8D1C
:10036800054502976DBF174500000325E5C7E1BFA6
:100378007A2131EF5A21636CF704B306F74021481C
:1003880017460000130686E36375D8028328050024
:1003980003586600938687001D8FAA966117DAA214
:1003A80023A016012393060014C15EA1130788FF3A
:1003B8007AA27A226EA12105B307F7407EA2B7E799
:1003C80000E023A08710B240224441018280084106
:1003D800BDBFB7E700E08C433707200023A0E7182C
:1003E800F98D0F10000001E523A0B7108280174394
:1003F80000000323A3BF9748000083A8A8BE9A87DC
:10040800814663FE170903A80700636DF508636B4F
:10041800A808138787006364E508F22321670507A6
:100428006319E600174600001306B6CA1822050726
:1004380018A217450000130565D8D2237A21239303
:1004480007003297334707087AA163856702174385
:100458000000032363B9630FF30003D36600631B33
:100468000300DE2223A0060121073E962106D2A220
:100478007AA1B6879843630417039746000083A6BA
:10048800A6B6630ED700762399EAD62352231843DB
:10049800A106B296D6A398C37E21A1077EA1B7E78D
:1004A80000E099B7BE86C287A9BFAA871747000090
:1004B8000327C7B3174600000326C6B2B305B540E5
:1004C8006314E6003E8529A8930687001843E3E9EC
:1004D800D7FEE3F7E7FE2E85E3E4D5FEE3F2E5FE7B
:1004E800828023AC05FE1C4199E30CC182803E87C3
:1004F80083A787FFEDFF232CB7FE8280411126C218
:10050800B7E400E04AC003A90400B707200006C604
:1005180022C43379F90023A0F4180F10000009E56C
:1005280023A0241101452DA09565938505D0C98D7B
:100538002A842105B3C5050833450508D1336DD193
:10054800FD572320050042A17CA123A024112105E9
:10055800B240224492440249410182804111B7E7E6
:1005680000E04AC003A9070026C23707200006C6D4
:1005780022C4AA843379E90023A0E7180F100000E9
:100588009747000083A7C7A60144014695E311C811
:10059800A285174500001305A5A5974004E0E7804C
:1005A80080CEA1652685974004E0E78040241DA001
:1005B80003C7E7FF631B970215CCA2851745000008
:1005C800130505A3974004E0E780E0CBA1652685E5
:1005D800EF20C068B24022852244B7E700E023A09C
:1005E8002711924402494101828011E03E8683A787
:1005F80087FF69BF3E84E5BF37E700E01C43B706C5
:1006080020002320D718F58F0F10000019C191C1C1
:1006180011E637E700E02320F71082802E960F704E
:10062800B650D5BF37E700E01C43B70620002320AB
:10063800D718F58F0F10000019C1014785E137E77A
:1006480000E02320F7108280B386E50003A80600A7
:10065800B306E5007D1623A00601110775F6C5B798
:1006680037E700E01C43B70620002320D718F58F92
:100678000F10000001C53307C50011E637E700E099
:100688002320F71082800505A30FB5FEE31DE5FEC4
:10069800F5B7B7E600E09C42370620002A87F18FBD
:1006A80023A0C6180F1000000145B306A7008386D3
:1006B800060091E637E700E02320F7108280050561
:1006C800EDB70111B7E700E026CA84434AC83707E7
:1006D800200006CE22CC2A892E86F98C23A0E71882
:1006E8000F1000009305F00432C633450608093997
:1006F8002A8401C53246CA850137F2402285624400
:10070800B7E700E023A097104249D24405618280F0
:1007180037E700E01C43B70620002320D718F58FE1
:100728000F10000001C599C1014711EA37E700E041
:100738002320F710054582800507E309E6FE330804
:10074800E500B386E500034808009422E306D8FED6
:1007580037E700E02320F7100145828037E700E003
:100768001C43B70620002320D718F58F0F10000070
:100778001307F6FFBA952A966317C50037E700E016
:100788002320F71082809821FD150505A30FE5FEAB
:10079800E5B737E700E01C43B70620002320D71849
:1007A800F58F0F10000001C53307C50019E637E7BC
:1007B80000E02320F7100145828014210505E39805
:1007C800B6FEE31CE5FE37E700E02320F7100545F9
:1007D8008280797126D2974400009384E48222D4DF
:1007E800804006D64AD04ECE52CC56CA5AC85EC6AB
:1007F80062C44DC837C9C901814B974A0000938A22
:100808002A801309F937174B0000130BAB9D974942
:1008180000009389A99A174A0000130AAAA13E204A
:1008280091EF5C4463990B009CC0032CC4002285A3
:100838004D366284A9A823A6FB00C5BF83A70A007A
:1008480082971C443307F5406376F50003278A0036
:100858001D8F2A97636BE9069747000023A8079620
:100868002E200820EF20803F5C405844A1CB0C4448
:10087800174600000326869CAE97BE8663E4B70041
:1008880063E4C700B386C74014C4A28B3A8441F816
:1008980017470000130787921C4B854663FBF60435
:1008A800FD171CCBB250225492540259F249624AA5
:1008B800D24A424BB24B224C4561828063940B0072
:1008C80098C0A5B723A6EB008DB703274B0219CB19
:1008D80063EDA7003385A74083A709016374F5007A
:1008E80023A8A900A28B40445DB703278A00BA97C2
:1008F800D5B79747000023AB078C6DB70111B7E751
:1009080000E04AC803A907003707200006CE22CC1A
:1009180026CA4EC652C43379E90023A0E7180F103F
:100928000000974400009384E4909C288844B9CF41
:1009380097470000938787C103D7C70A21CB03A431
:10094800870A6305A404974900009389298783A728
:1009580009016380A710173A0000130A6A6A8327FF
:100968000A0082976364A40E83270A00098C829781
:1009780083A7090198443354F40AB307A4003E85B9
:1009880063E4870063E4E7003385E740B7E700E006
:1009980023A027119C44639DA70217440000130459
:1009A800E48118489737000083A787656315A70A6D
:1009B80082979444374736FE130707C83697B3071C
:1009C800A7003E8563E4E70063E4D7003385D7409A
:1009D80017440000130484DA5C5C99CB9736000056
:1009E80083A6C6749C463707CDFF7D17F98F9CC632
:1009F80011E1884485475CD09747000083A7C780EA
:100A0800829715E15C5C99CF5C5089CF976006E0CE
:100A1800E780A081975006E0E78020F29747000022
:100A280023A007D87D335C5C91CB173700000327E0
:100A3800E76F1C47B7063300D58F1CC7F2406244E6
:100A4800D2444249B249224A056182809C443E947C
:100A580021BF228525BF829714489844B387A600F2
:100A68003E8563E4D700E3E5E7F63385E7408DB7D5
:100A78009737000023A0A75811C5854717370000EE
:100A8800230CF75682809737000083A7A75685C3A3
:100A9800411106C682979737000083C7E75589E753
:100AA8009737000023A80754B24041018280973746
:100AB800000083C7675491E79737000023AC0752BB
:100AC80082808280411122C426C206C64AC0974449
:100AD80000009384A4CA83C73402173400001304A7
:100AE8002474B9C7173400001304446D1739000083
:100AF8001309C951032709001C2014300146B3A566
:100B0800E7208E21A5CD11C21CA00820636FD50651
:100B1800973700002384076A9737000083A7474E5A
:100B2800C5EFB24022449244024941018280829733
:100B38001C40F5FF9737000083C7C77085E3DC4882
:100B4800858B89CFD84C9947631EF70097470000DB
:100B580023A007C4EF10B01F5C4482971C44D9D36C
:100B6800829749B7D84C9D47E31AF7FE974700008C
:100B780023A007C2EF10B01D1C48C5B7850793F71F
:100B8800F70F0546E3EDD7F641B73327E5200E23E7
:100B98002310070097370000239107469737000076
:100BA80083A74746B347F5209C4382971C2083269A
:100BB800090017370000035747443377E540B3A6C9
:100BC800D7209222518F9AA299C385071CA018207A
:100BD8001C30E368F7F42DBF9737000083A707663A
:100BE8001CC8C53E83C734028DFF83C7140299CB46
:100BF800DC4C89EB97470000A38207BA975006E0C0
:100C0800E78080009737000083A7076099DBD84CFE
:100C18009147E3E8E7F09747000083C7A791918BD6
:100C2800E39107F09737000083C7073DE39B07EE82
:100C380018308326090063C8E7002244B240924472
:100C48000249410165B933A6D7201222E31B06ECFD
:100C58008507D5B7B7C700401387C7201443139635
:100C6800264910C301000100938787261735000025
:100C7800032585569C436A0514C393C7F7FF9983D8
:100C88005D8D82809737000083A7C73891C382871C
:100C98001305F00F8280174600001306E686974674
:100CA800000093866688DC36383E4C4ABA97FD8B3E
:100CB80033D7F5001CB2DCB6058B0DE7943A130563
:100CC8000002B3F7D702814633D8E5486309080024
:100CD8006394D70018B28280850693F6F60F05074D
:100CE800E314A7FE82809747000083A767AAC1E79D
:100CF80041114AC09737000083A7873006C622C42F
:100D080026C28297174900001309098283278900A0
:100D1800638DA7046363F5041D8D973400009384E5
:100D2800A47EBC2C135455006361F404AD37BC2C6D
:100D3800032789009396570036971D8C2324E900D2
:100D4800E376F4FE22448830B24092440249814559
:100D58004101173305E06700634517370000032793
:100D6800E74DB307F7403E954DBFB2402244924449
:100D78000249410182808280011126CA973700000A
:100D880083A7072806CE22CC4AC84EC652C48297EB
:100D980097340000938444799844AA870145630DE9
:100DA800F70463E3E706998F173900001309C9753B
:100DB80093F9F70113D457008347A901636AF40232
:100DC800173A0000130A0A47F9350347A9018C446A
:100DD80003268A0093175700AE97198CBE8663E4E2
:100DE800B70063E4C700B386C74094C4E37EE4FC5D
:100DF8001315540033653501F2406244D244424928
:100E0800B249224A056182809736000083A60643CC
:100E18003387E640BA9749BF411126C2974400007C
:100E28009384C4959C4422C406C6858B173400005D
:100E380003240478A1C718289747000023A407941F
:100E48008947630DF7020146930550020145EF10EB
:100E5800701D014681450545EF103005DC44858B42
:100E680091CF2244B24092448145177505E013059D
:100E780065BE4101174304E0670003B3EF20D07259
:100E880022852244B240924441016F10107B97376B
:100E9800000083A7A775639F071C011122CC2A8431
:100EA800094506CE26CA4AC84EC697340000938420
:100EB800E426EF20907790409307800717390000C9
:100EC800130909257CD283270900973900009389E3
:100ED800E925B7053300D8572285719B136717009A
:100EE800D8D798431377F7CF98C398431377F7CF9A
:100EF8001367072098C303A709001447CD8E14C7AA
:100F0800B70603009386862534CA5457F59A54D7F2
:100F180098433424137707F893F6F607558F98C348
:100F2800EF20E0069440370500827D15DC4293E708
:100F38001700DCC203260900030784065C56937574
:100F4800F703E605E98FCD8F5CD69305A00383A749
:100F5800090063D9E50AF84FB70500074D8FF8CFA8
:100F6800B7C7898E938767ED1CC6B7575500938717
:100F780057555CC28347A40683494406B3E9F90080
:100F88008947174700002329F7809737000023ADCA
:100F9800077E7C44BCDE9737000083C7A72AD9CFD9
:100FA800FC52FDFF0C384E859737000023AC077CB8
:100FB800EF10006718289D47172500001305653DA9
:100FC8006306F70017050000130545E55534832728
:100FD800090098431317772998C3D857719BD8D716
:100FE8009737000023A6077A9737000023AA0778C7
:100FF8009C40F2406244094798C3D2444249B249EE
:10100800056182809305200263DAE500F84FB70591
:1010180000F9FD156D8FB705000589B7B70500F90B
:101028006945FD156357E500F84F6D8FB705000357
:1010380035B7F84F6D8F1317872915B718289D47AF
:101048008145172500001305C5346306F700170509
:1010580000001305A5DC974004E0E780E094103811
:101068006244F240D2444249CE85B2490145056105
:101078006F10A0638280973700009387274DE8534D
:10108800054754256390E60203C747079147631A4B
:10109800F700011106CE2AC6EF10B0553245F240CE
:1010A8000561F5B3828083278511E5CB411122C400
:1010B80006C658258345E5049437D2272A84137732
:1010C800C70F1395466063F7C50663510506882761
:1010D80093F6F60794B70546936627006314C50090
:1010E8009366170054A4D8430907D8C303250411ED
:1010F8004CB82E86CC430905EFF00FD08327841116
:101108005438D8433697D8C3DA27158FDAA78947D2
:101118003CBC034764039737000083C7C70D636966
:10112800F706B24022440145410182801367170047
:1011380058A46DBF9376F60F635505028827854539
:10114800136627006314B5001366170050A454B83B
:10115800A384070085473CBC832784119C43D5FBA7
:10116800C9B71367170058A454B8A3840700032508
:101178000411CC430905EFF02FC883278411543894
:10118800D8433697D8C3DA27158FDAA78D47E1B742
:101198005C2493E707015CA469B705458280411187
:1011A8009737000083A707F522C406C6858B2A84D3
:1011B800C5E74165130525F5978005E0E78080566A
:1011C80041CD3C253EA583270412ADE32320A4127C
:1011D8002322A41285472311F404232005007C2828
:1011E80054415EA5583418A5054718B5138517024C
:1011F800173700000327475C15811C437D151375BD
:10120800F50F9CC25C43DCC21C479CC65C47DCC62D
:101218001C4B9CCA5C4BDCCA1C4F9CCE5C4FDCCE82
:101228000DC19386060213070702C1BF8327441224
:1012380088C3835724042322A4128507B3C7070849
:1012480059BF17370000130767301E2785071EA7E9
:10125800B2402244410182805C24230904000545F0
:1012680093C747005CA4EDB7142D854763EED70AF2
:101278001C3D2A870145DDEB5C2713F507013C2B54
:1012880099CB834667039737000083C7D7F663EC8B
:10129800F60001E5828059E582808357271E0357AF
:1012A800671EBA9721A08357271E75F90145BDCF40
:1012B8009387C71217350000035585F8B3B5A70201
:1012C80037460F00411113060624814622C426C260
:1012D80006C67D543385A70297C006E0E780204103
:1012E8009734000083C494F1AA949737000083A729
:1012F800272F03A707099C433354E40AFDFB9737BC
:10130800000083A7E7CF829781476364A400B307EF
:10131800A440B240224433B59700134515009244C7
:10132800410182808147A5BF0145828082801737AD
:1013380000000327A7DE3C5BFDFF0100010082805F
:1013480035C901116C0022CC06CE2A84EF2050004A
:1013580029C9FD57630CF50417370000130787E800
:101368005453B2479DC22547637BF700938567FFB7
:10137800034594026244F24005616F10501217371A
:1013880000000327A7EBBA97D5B70C3F63E5B70072
:10139800B385B740F1BF17370000032727EABA978C
:1013A800C5BF6244F24005616F20403EF24062448E
:1013B800056182808280797152CC173A0000130A45
:1013C800EA1826D283244A0906D622D44AD04ECE19
:1013D800D5C8973700009387673AD44F1547638677
:1013E800E604DC532A8989CF975006E0E780E0E3DA
:1013F800974006E0E78060549737000023A2073A39
:10140800FD596C002685EF20A0740DE91725000012
:1014180013050538EFF0CFE59737000083A707D00D
:101428003707100098C70547B8DB0D45B25022545E
:1014380092540259F249624A4561828063743501C7
:101448003244AA898440D5FCFD571305F00FE38F79
:10145800F9FC914763F187029307B4FF2320F90051
:101468002324FA0A99E79737000083A727DD23206A
:10147800F900014565BF9737000083A727DCED1702
:10148800A297E9BF09455DB7797126D206D622D45D
:101498004AD04ECE52CC56CA5AC85EC68347550368
:1014A80003447513AA843E941374F40F93074002FF
:1014B80063F687001304B4FD1374F40F03A98413AF
:1014C80083A9C413A38B841222864A85CE8597C02C
:1014D80006E0E780001D058915E503CBD412014A13
:1014E800814A337B6403930B500252864A85CE852A
:1014F80097C006E0E780E01A05890DC563916A0385
:101508001374FA0F238B8412B25022549254025946
:10151800F249624AD24A424BB24B45618280850AFF
:10152800939A4A60050AE3127AFDE9BF8327850981
:1015380003560504797193D60701BD8EB3C6060814
:10154800358E93575640898B135776485D8F93573E
:101558003640918B5D8F93571640A18B5D8F931703
:101568001600C18B5D8F9317360093F707025D8FC6
:101578009317560093F707045D8F9317760093F738
:10158800F70F22D45D8F2A849357D6001355B600DF
:101598001189898B93558600C98F1355F6002582CA
:1015A800C98F218AD18F13961500418AD18F13963E
:1015B800350013760602D18F13965500137606046C
:1015C800D18F139675001376F60FD18FA207C545F4
:1015D8005D8F3307B70226D24AD04ECE0329841333
:1015E8008329C4135AC806D652CC56CA36973347ED
:1015F800070813565740098A93577748D18F1356CF
:101608003740118AD18F13561740218AD18F13166C
:101618001700418AD18F1316370013760602D18F2F
:101628001316570013760604D18F13167700137616
:10163800F60FD18F1358B7001356D7001378480008
:10164800098A13558700336606011358F700258366
:1016580033660601218B518F13161500418A518F6D
:101668001316350013760602518F1316550013769C
:101678000604518F131675001376F60F518F220743
:10168800D98FB387B7025EC6B697B3C7070813D515
:101698005740098913D77748498F13D5374011899F
:1016A800498F13D517402189498F13951700418910
:1016B800498F1395370013750502498F1395570005
:1016C80013750504498F139577001375F50F598D18
:1016D80013D8B70013D7D70013784800098B13D64F
:1016E80087003367070113D8F700A583336707011D
:1016F800A18BD98F13171600418BD98F131736007A
:1017080013770702D98F13175600137707041E069D
:10171800D98F1376F60FD18FA2073367F5003307F9
:10172800B702130650024A85CE853697B98EB3C4E0
:10173800060833F6C402137BF60F97C006E0E7806D
:1017480040F6058905E9834AD412014A930B5002F1
:10175800B38A9A02814493DA0A0126864A85CE859D
:1017680097C006E0E780E0F305890DC563914A0359
:1017780013FBF40F230B6413B250225492540259F2
:10178800F249624AD24A424BB24B45618280050A0D
:10179800137AFA0F8504E39274FDE9BF8327C5081D
:1017A80003568508797193D60701BD8EB3C606081E
:1017B800358E93575640898B135776485D8F9357CC
:1017C8003640918B5D8F93571640A18B5D8F931791
:1017D8001600C18B5D8F9317360093F707025D8F54
:1017E8009317560093F707045D8F9317760093F7C6
:1017F800F70F22D45D8F2A849357D6001355B6006D
:101808001189898B93558600C98F1355F600258257
:10181800C98F218AD18F13961500418AD18F1396CB
:10182800350013760602D18F1396550013760604F9
:10183800D18F139675001376F60FD18FA207C54581
:101848005D8F3307B70226D24AD04ECE0329040A49
:101858008329440A5AC806D652CC56CA3697334703
:10186800070813565740098A93577748D18F13565C
:101878003740118AD18F13561740218AD18F1316FA
:101888001700418AD18F1316370013760602D18FBD
:101898001316570013760604D18F131677001376A4
:1018A800F60FD18F1358B7001356D7001378480096
:1018B800098A13558700336606011358F7002583F4
:1018C80033660601218B518F13161500418A518FFB
:1018D8001316350013760602518F1316550013762A
:1018E8000604518F131675001376F60F518F2207D1
:1018F800D98FB387B7025EC6B697B3C7070813D5A3
:101908005740098913D77748498F13D5374011892C
:10191800498F13D517402189498F1395170041899D
:10192800498F1395370013750502498F1395570092
:1019380013750504498F139577001375F50F598DA5
:1019480013D8B70013D7D70013784800098B13D6DC
:1019580087003367070113D8F700A58333670701AA
:10196800A18BD98F13171600418BD98F1317360007
:1019780013770702D98F13175600137707041E062B
:10198800D98F1376F60FD18FA2073367F500330787
:10199800B702130650024A85CE853697B98EB3C46E
:1019A800060833F6C402137BF60F97C006E0E780FB
:1019B80040CF058905E9834A1408014A930B500270
:1019C800B38A9A02814493DA0A0126864A85CE852B
:1019D80097C006E0E780E0CC05890DC563914A030E
:1019E80013FBF40F230F6407B25022549254025988
:1019F800F249624AD24A424BB24B45618280050A9B
:101A0800137AFA0F8504E39274FDE9BF8327450929
:101A180003568508797193D60701BD8EB3C60608AB
:101A2800358E93575640898B135776485D8F935759
:101A38003640918B5D8F93571640A18B5D8F93171E
:101A48001600C18B5D8F9317360093F707025D8FE1
:101A58009317560093F707045D8F9317760093F753
:101A6800F70F22D45D8F2A849357D6001355B600FA
:101A78001189898B93558600C98F1355F6002582E5
:101A8800C98F218AD18F13961500418AD18F139659
:101A9800350013760602D18F139655001376060487
:101AA800D18F139675001376F60FD18FA207C5450F
:101AB8005D8F3307B70226D24AD04ECE0329040BD6
:101AC8008329440B5AC806D652CC56CA3697334790
:101AD800070813565740098A93577748D18F1356EA
:101AE8003740118AD18F13561740218AD18F131688
:101AF8001700418AD18F1316370013760602D18F4B
:101B08001316570013760604D18F13167700137631
:101B1800F60FD18F1358B7001356D7001378480023
:101B2800098A13558700336606011358F700258381
:101B380033660601218B518F13161500418A518F88
:101B48001316350013760602518F131655001376B7
:101B58000604518F131675001376F60F518F22075E
:101B6800D98FB387B7025EC6B697B3C7070813D530
:101B78005740098913D77748498F13D537401189BA
:101B8800498F13D517402189498F1395170041892B
:101B9800498F1395370013750502498F1395570020
:101BA80013750504498F139577001375F50F598D33
:101BB80013D8B70013D7D70013784800098B13D66A
:101BC80087003367070113D8F700A5833367070138
:101BD800A18BD98F13171600418BD98F1317360095
:101BE80013770702D98F13175600137707041E06B9
:101BF800D98F1376F60FD18FA2073367F500330715
:101C0800B702130650024A85CE853697B98EB3C4FB
:101C1800060833F6C402137BF60F97C006E0E78088
:101C280040A8058905E9834AF408014A930B500244
:101C3800B38A9A02814493DA0A0126864A85CE85B8
:101C480097C006E0E780E0A505890DC563914A03C2
:101C580013FBF40F230F6407B25022549254025915
:101C6800F249624AD24A424BB24B45618280050A28
:101C7800137AFA0F8504E39274FDE9BF411126C275
:101C880006C622C44AC09734000083A4A49163897D
:101C9800041003A4C40AAA86054525C43C241307D6
:101CA800700A6392E70858301C341729000013099A
:101CB800695803268900B387E7020357C900B38729
:101CC800E7021307003293870719B3D7E70203A780
:101CD80044093E97BA846364F7006364C700B30499
:101CE800C7409727000083A7A73184C28297B3878C
:101CF800A44063F5A40003278900BA9789EB13056C
:101D0800F00FB24022449244024941018280583087
:101D18009306204E3307D702E3F3E7FE930780FAD2
:101D28003CA40145F9BF1307800AE39AE7FC97270B
:101D3800000083A7E72C82972A893545EF20E00E1B
:101D4800AD47173700002329F7A458301C3417264D
:101D580000001306264EB387E7025A261046B387BB
:101D6800E7021307003293870719B3D7E70203A7DF
:101D780044093E97BA866364F7006364C700B306F4
:101D8800C740E31ED9F617D505E01305E5A5EFE032
:101D98003FCE9727000083A767380947F8D785B74C
:101DA800054585B7397156D2973A0000938A0A9D3E
:101DB80083A70A033707080026DA06DE22DC4AD89A
:101DC8004ED652D45AD05ECE62CC66CA6AC86EC6A7
:101DD800F98F9724000083A4E47C638A071C83A9F5
:101DE800C40A83C7990003A4C90092073E94282017
:101DF800B14705053305F5025E203E9533450508D4
:101E0800EFE0CFEFAA8C630F051A130DC50023244A
:101E1800A50134203146370B0300B386C6022313CD
:101E280004000149172A0000130A4A2F972B0000C3
:101E3800938B0B2E972D0000938D4D2F130B8B1525
:101E4800054CEA9654C483C679009307D0078325C6
:101E58000A00B386F602C1679CC5370833008606B8
:101E6800B4D183A60B0090421376F6CF90C290426D
:101E78001376F6CF1366062090C203A50D00104511
:101E88003366060110C503A6090023A86505930556
:101E9800500290C672205444B2962324DD001430B8
:101EA8000146CA96A301DD0003C504089736000061
:101EB80023A8068CEF00101783260A00CC46139639
:101EC8001549D0C60F10000083260A003706020005
:101ED80090C61306000823A8CA0003A60B001042E8
:101EE80013567648631E860B1306E018F0D2CCC64C
:101EF80017360000232E068817360000232206888E
:101F080023A08601A925EF10306A83A64A00858A96
:101F1800D9CAEA85268597E005E0E78000950DE9AE
:101F280003465D0049C276204E20B29663DDB606B0
:101F3800B428AC4803258D00918E8906B695EFE04C
:101F4800AFEB23020D0003465D007620B29676A023
:101F580003260A00310D3452FDFE34200509137999
:101F6800F90FE362D9EE9C246685A381FC001C204E
:101F7800A3820C002383DC002382FC006254F2500D
:101F8800D2544259B259225A925A025BF24B624CCD
:101F9800D24C424DB24D2161172305E0670003ADD5
:101FA8001306E01AA1B7FD562302DD0055B797279F
:101FB800000083A7A716FC5791C78547172700007D
:101FC800230CF702F2506254D2544259B259225AA1
:101FD800925A025BF24B624CD24C424DB24D216197
:101FE8008280797122D426D22E84AA84414697C54C
:101FF80006E0938565AB0A8506D6972004E0E7805E
:10200800E01B414697C506E0938505AA0808972076
:1020180004E0E780A01A3C3010088A85DC875C2041
:1020280026855C875C30DC86973006E0E780004BCD
:102038000347F1011C200145631EF7000347E10136
:102048001C3001456318F7000345D1013C201D8D64
:1020580013351500B2502254925445618280011103
:1020680022CC26CA4AC84EC606CEAA841724000027
:102078000324045A13092500854905C09C303830CB
:10208800858B6304F700405CCDBF19469305440077
:102098004A85EFE0EFE7E31835FFF2402285624416
:1020A800D2444249B24905618280411122C426C204
:1020B8004AC006C61724000003248455930425004B
:1020C800054901E8B240228522449244024941016F
:1020D8008280A6851305A4022937E30525FF405C05
:1020E800CDB7411122C426C24AC006C61724000033
:1020F8000324045293042500054901E8B2402285CF
:1021080022449244024941018280A6851305A40114
:10211800C93DE30525FF405CCDB7011126CA6441DE
:1021280022CC4AC84EC652C406CE2A841D499309F9
:102138006505054A3C4463E4F4000545A1A058340C
:10214800DC2063192705034784026304F7008440F1
:10215800D5B7D83083475405E31BF7FE19469305D6
:10216800640513856400EFE0AFDA8547E311F5FEF7
:10217800D82483479402E31CF7FCFA243E34E3187E
:10218800F7FC0145F2406244D2444249B249224A2E
:1021980005618280E31DF7FAD83083475405E318B8
:1021A800F7FA1946CE8513856400EFE06FD6E31081
:1021B80045FBC1BF411122C406C626C24AC0172426
:1021C8000000032424405DC88347840B1307700A6A
:1021D8006393E7080347140E8347A40B17290000ED
:1021E8001309490583268900B387E7020357C90005
:1021F800B387E7021307003293870719B3D7E702BB
:102208000327440A3E97BA846364F7006364D700DF
:10221800B304D7409727000083A787DE04C18297BD
:10222800B387A44063F5A40003278900BA9785CB38
:102238000347140E9306204E3307D70263F1E702D3
:10224800930780FA230CF40A0145B24022449244D1
:102258000249410182801307800A639EE70017251F
:1022680006E013054543EFE0BF809727000083A7EA
:10227800E7EA0947F8D71305F00FC1BF0545F1B7DD
:10228800011122CC26CA06CE2AC42EC61724000065
:1022980003248437854419E001450DA09C84183037
:1022A800858B6304F7000044FDB719469305A10028
:1022B80013052400EFE0CFC5E31795FEF240624412
:1022C800D244056182800000EFE0EFFB730000005C
:1022D8000000000097220000938202D203830200CC
:1022E80023800200630F0300F32510342EC09705E6
:1022F80000009385A5FD73901534EF00E05A730034
:10230800203086DCEF00405AE65082800000411100
:102318004AC0172900001309A9DF0327090026C2AC
:1023280006C61C5F22C497240000938424DE93D73A
:102338006748C1C7930700061CDF17240000130471
:10234800E443184C930700086317F7009C409C432C
:1023580093F707041CCC1C4093F7070499CB9727E5
:10236800000083A7E7C9829748D81C4093F7F7FB7A
:102378001CC01C4093F7070299CF1C401727000088
:102388000327C7D9B706080093F7F7FD1CC05C54AC
:1023980014C786077CD71C4893F7070499EF85472D
:1023A8005CC8370702009727000083A727D798C77C
:1023B8001307000C18C81854F8D383270900985F2E
:1023C8001357474805C3985F1367070198DF972796
:1023D800000083A7A7D423A2070685471727000074
:1023E8002326F73A9C40D8431357174819C7D843B0
:1023F800759BD8C3D843799BD8C3B2402244924432
:10240800024941018280213773002030972700005C
:102418009387C7363707040088DB698F11CF1727E2
:1024280000000327A7CFFD5634D7972600009386D0
:10243800E6D8D84E0507D8CE137785000DC3984740
:102448009726000083A6C6CC1367170098C7130702
:10245800000898CBD856719B13671700D8D6137706
:10246800150011CFD8439726000083A666CA1367C4
:102478001700D8C3D856719B13671700D8D613779F
:1024880065000DC31377450059C7984313671700B4
:1024980098C39726000083A6A6C7D856719B1367D2
:1024A8001700D8D64167698F0DC39726000083C6E9
:1024B8002611C18A1727000013074709B5C28346AA
:1024C800470793E60602230AD70637070200698FF3
:1024D80011CF984B1377070819C3054798CB97274F
:1024E800000083A7A7C33707020098C7B7070800EB
:1024F8007D8D0DC1172700000347970C058B972783
:1025080000009387A7041DCB03C75707136727004D
:10251800A38AE7068280D84713671700D8C795BFF4
:10252800834647070946BD8A6388C600834647072E
:102538000D46BD8AE39BC6F8914671B703C7570796
:10254800118B69DB03C7570713678700D1B7972635
:10255800000083A6A6BC97270000938727229843EC
:10256800058B19E7D843058B01E7F8526DFBDC4B67
:102578009727000023AE07208280972600009386C5
:1025880026B92A8788421C5D93D75748C1EB81C575
:102598001C59BD839CA115C69C42945BC60693D763
:1025A800660163D6060093E707C0B3C7070883161A
:1025B800060093975760A9CABE968947B3C6F60224
:1025C80016A29727000083A767B5BC4B083393D79B
:1025D80057488DCF29C59726000083A6A61B93F6DA
:1025E80006049307950009459DCABA979C23054799
:1025F800194593F6F7066394E602014593974760F9
:1026080063DF0700394582801EA265BF2A974833D9
:102618001375F5077D153335A00082800545828046
:102628009727000083A707AF99CB944BD04B9842CC
:10263800518F98C294439C479842D98F9CC21726C1
:1026480000001306A6AD054818429726000083A689
:1026580026AC9727000093876712631D05038842FD
:102668001365050888C283C62702B3C5D52093859C
:10267800A50C54471395164948C70F100000184277
:1026880037060200860510C71306000890CB6CD3E6
:1026980054C7828088421375F5F788C283C627021B
:1026A800B3E5D5209385E50EE9B7411126C2AA877F
:1026B80006C622C42E8597240000938424A6B285DA
:1026C800C9EF9C40F8537DFF3707020098C797274A
:1026D800000023A9070AB7E700E03707200037F40E
:1026E80000E023A0E728130404D01C48ED9B1CC875
:1026F8001C4893E787031CC87300501015379727A9
:10270800000083A7E7A098431317772998C3D857E1
:10271800719BD8D79727000023AC0706972700009E
:1027280023A007069C40094798C31C4893E78700E5
:102738001CC87300501094401727000013070704A3
:102748001C47858B91E75C47858B99E3FC52EDFB31
:10275800B24022449244410182800D47639AE704C3
:102768009727000023A007029727000023AE070041
:10277800B7E700E03707200037F400E023A0E72898
:10278800130404D01C48ED9B1CC81C4893E787031E
:102798001CC87300501069359727000083A7479716
:1027A80098431317772998C3D857719BD8D7B5BFC3
:1027B8000547E392E7F837F700E0130707D0144B13
:1027C800ED9A14CB144B93E6860314CB7300501088
:1027D800984050479316164954C70F100000984068
:1027E800B706020014C7930600089725000023AF18
:1027F800D5F89726000083A6A691944293D67648EA
:10280800639FF6009307E0187CD350C737F700E0C2
:10281800832707D193E787002328F7D019BF9307A9
:10282800E01ADDB79727000083A7C78E89CFD44366
:1028380003A8870098423367070198C2D447DC4B46
:102848009842D98F9CC205479727000083A7478CD9
:102858009505631BE50298431367070898C3984FCB
:10286800137707C01367A71398CF13078007B8BB60
:10287800939735009387C70319C293171600172734
:1028880000002321F7F2828098431377F7F798C363
:10289800984F137707C01367271398CF1307F007CC
:1028A800B8BB93974500F9B79727000083A7078718
:1028B8008847D847798D01C988C79727000083A71B
:1028C800A78591C38287828089671727000003271D
:1028D800E784938707F47CD39726000083A60685B0
:1028E80083A7060993D7A74991C783A7060993D752
:1028F800974999E37C53EDF78280411106C622C4BB
:1029080026C24AC063030510AD472A8463EAA70CB0
:102918001304F5FF1374F40F1385F5FF01469305AF
:10292800F00F1375F50FFD3D972400009384048084
:102938009840171900001309A97D136404045C5713
:102948001374F407170500001305250DF59B5CD7D4
:10295800032709001C4393F707F8C18F1CC3B74727
:102968007671938797121CC7B757550093875755A9
:10297800171400001304847A5CC3184097270000DA
:1029880023AE07DE5C43F99B5CC3A547172700000D
:102998002324F7E0EFE0CF8D14409727000023A908
:1029A80007DE9727000023AD07DC032709008547CA
:1029B8009CC21C4337063300014593F7F7CF1CC36D
:1029C8001C4393F7F7CF93E707201CC398401C4795
:1029D800D18F1CC7B707030093878715BCCA05A00A
:1029E800B1476307F5029307600263E5A700130484
:1029F800E5FF0DB7930770024945E30FF4F0B240C5
:102A0800224492440249410182801304500229B7AA
:102A18001304600211B717270000032767D6058B38
:102A280097270000938787B201CF17170000032765
:102A3800276E185F1357574801E79A2705079AA783
:102A480003C68703EC33C8234DBDAA8717150000BA
:102A58000325855B11E182803A216315B7001821AF
:102A6800E30BF7FE4845FDB7411122C406C626C24E
:102A78004AC02E849DCD13F9150081474147630450
:102A88000904131745003E97B1463307D702971438
:102A9800000083A4E457B317F02833C90708BA9491
:102AA8009C40C840829723A0040023A2040033441A
:102AB8008900B24022852244924402494101828021
:102AC800B356F448DDFE8507E39CE7FECDB7011158
:102AD80026CA06CE22CC4AC84EC6AE84B1C593F7E4
:102AE800150001444147A1CF93174500A2973147EC
:102AF800B387E702971900009389895103A9090050
:102B08003E998327090081C70325490082973147E9
:102B18003307E40283A70900BA979C478DC733148B
:102B28008028B3470408BD8CF24062444249B24948
:102B38002685D24405618280B3D68448D5F605043B
:102B4800E31CE4FECDB72320090023220900C1BFFE
:102B58007971B7E700E022D4804352CC06D626D25A
:102B68004AD04ECE56CA5AC85EC662C43A8A370799
:102B78002000798C23A0E7180F10000005E123A09E
:102B880087100945B250225492540259F249624AB8
:102B9800D24A424BB24B224C4561828097170000C3
:102BA80083A70746B6892A89AE8A328B971B00000D
:102BB800938B0B46829703A70B008144B146C1470C
:102BC800338CD40233068701104241E2C1659385F4
:102BD80005F04145EFD0CFF219ED9717000083A714
:102BE800676381C7814511458297B7E700E023A055
:102BF80087102D4541BF171700001307E7401C43F6
:102C0800A1E308C323000500B31790283EA183A7BA
:102C18000B00232605002324650123224501E297A2
:102C280023A0270123A2570123A447016384090095
:102C380023809900B7E700E023A08710014599B7E2
:102C48003E87DC47F5FF48C775BF8504E39AF4F66D
:102C5800B7E700E023A0871021452DB7B7E700E0CC
:102C68009843B706200023A0D718758F0F100000CF
:102C78009716000083C69654637FD5009716000008
:102C880083A6C6383325D5201621D58D0EA123A0BD
:102C9800E7100145828023A0E7100D4582800111CD
:102CA800B7E700E022CC80433707200006CE26CACB
:102CB8004AC8798C23A0E7180F100000BD4763E9C4
:102CC800A70431473307E5029717000083A7473465
:102CD800BA979C4395CF3315A0282E89B34505088C
:102CE80001452EC69D33AA8409C9B24501459710EE
:102CF80004E0E780407423A42401B7E700E023A0A0
:102D080087100145F2406244D244424905618280FD
:102D1800B7E700E023A087100945EDB79716000034
:102D280083C6467E9717000083A707370147639439
:102D3800E600014582808E23138687026394A500EE
:102D48003E85828005071377F70FB287CDB79717AF
:102D5800000083C7377BAA8685071715000003255F
:102D68006534014712216307D60005071905E36B8F
:102D7800F7FE014582802A871715000003250533D1
:102D880011E182801C45B227636BC70003584500D8
:102D9800B306C8006355D70081466394060108410D
:102DA800C5B703D3A700938807016316E30091C151
:102DB80092A13E8582808506C687B3C60608F1BF04
:102DC8009716000083C606749717000083A7C730BC
:102DD80001476394E60001458280AE231386C7034A
:102DE8006394A5003E85828005071377F70FB287A5
:102DF800CDB7411122C406C6971700002382077C6D
:102E0800171400000324442E05C06C390145B3157E
:102E1800B028B3C50508972004E0E780E0AE930723
:102E280010273305F50202942244B240814501453A
:102E38004101172304E0670023B7383D09C734254B
:102E48006312D7027DB73C2DF5DF3825E30CF7FE7A
:102E58003CA5814517E5FFFF13052522172304E04C
:102E6800670083B43C2D89C7E394F6FE38A5D5B72F
:102E7800F1FAEDBF41114AC0172900001309099062
:102E88008327890022C426C206C6971400009384AB
:102E9800E46B858BE0509DCB9727000023A4078E19
:102EA80083C74407C18B85CFEF00107083C74407E1
:102EB80093F70702E5DF83C74407228593F7F70CEA
:102EC800238AF406974005E0E780A0D7EF00D06D8D
:102ED80022852244B24092440249410119BF83C766
:102EE8005407858B91CBEF00306C8D47230EF40689
:102EF800BC5822858297D9BF83C744071547BD8B25
:102F08006394E7048347B4060345340601469305F2
:102F180050025D8D013A014681450545EFF0EFF815
:102F28008327C900858BDDD322859727000023AD31
:102F38000784974005E0E780E0B849F9B2402244A9
:102F4800924402494101828083C744071947BD8BD7
:102F5800E39EE7F68347B406034534060146930526
:102F680050025D8DEFF01F8C014681450545EFF05D
:102F7800CFF38327C900858BB1DB22859727000013
:102F880023A40780974005E0E780608D7DB7411155
:102F980022C426C206C67C2578452A84BD8B1CA976
:102FA8001CA31D476445639BE7340547B8A08347C6
:102FB800F5058D466395D7185E2DCDE37C491147FD
:102FC800B18B638DE70831476398E700034715061F
:102FD8008347F5076304F7088547BCB0194693058E
:102FE800640313854400EFD02FE1BC20990793F7C1
:102FF800F70FBCA0034704061377070401CFB830C6
:1030080013670704B8B07844BA975838B8B3BC20E7
:103018008507BCA0971700002384075ABC2013F724
:10302800F703050718B80347E4051A07D98FBCA0AA
:1030380083475403858B91E7034744038947631704
:10304800F70078441C2393E707041CA37C44183832
:1030580098B3B2402244924441018280A147BCB057
:103068008357C406971500009385454E1716000030
:103078001306C60ADCA08357C40603471406744423
:10308800A1831207BD8BD98FDCB2B420854789068E
:1030980093F6F60FB4A01717000003476752631E94
:1030A800F706183C9387E6008E07231AF4069387E1
:1030B800C708B387E702794510420948238A0507FC
:1030C800C1650CC6938707FBB3C7070893877716B4
:1030D800B3C7A70233C70708B387A70286073CD23E
:1030E800BC3093E70701BCB07C44B69783462406FE
:1030F80093E60604B4B3B4207C44B697D8A3B420AE
:103108007C4421837D8BB697834634069606558F7B
:10311800D8B3BC208D07BCA011B71042F94738526C
:1031280005833357F7023C5268528583FD8BAA9773
:103138007CD28D47238AF5063347070855B71946C9
:10314800639DC7125E2DC1E393056503B8B013856F
:103158004400EFD06FCABC201385A4009907BCA017
:10316800BC3093E72700BCB083475403898B95CFC5
:103178000C58BC299DCB1946D105EFD0EFC7784430
:103188001C2393E707F81CA3BC20990793F7F70FB4
:10319800BCA00347040613770704E30D07E6B43021
:1031A800784493E60604B4B085B58347D40391C741
:1031B80078441C2393E707F81CA319469305E403F6
:1031C800EFD08FC3D1B7A147BCB08357C506DCA0E9
:1031D8008357C506034615066C45A1831206BD8BA9
:1031E800D18FDCB1B02017150000130525369715CF
:1031F80000009385A5F209061376F60FB0A097177D
:10320800000083C7E73B6398E704183C9307E60090
:103218008E07231AF4069387C708B387E70279480D
:103228008946230AD5069441C1658CC6938707FB56
:10323800B3C7070893877716B3C7070333C70708C9
:10324800B38707038607BCD2BC3093E70701BCB03D
:103258007C44B29761BD8C41B851F9470583335717
:10326800F702BC5103A845068583FD8BC297FCD1A4
:10327800230AD50633470708C1BFA147BCB0835707
:10328800C506DCA08357C506034615066C45A18311
:103298001206BD8BD18FDCB1B020171500001305C5
:1032A800E52A09061376F60FB0A09717000083C722
:1032B80027319715000083A565E6E39FE7F8183CDA
:1032C8009307E6008E07231AF4069387C708B38787
:1032D800E702F9460948230A0507416588C5938727
:1032E80007FBB3C7070893877716B3C7D70233C757
:1032F8000708B387D7028607BCD1B9B70547639ECD
:10330800E706B1471CB983475503898BA1CB0C59F4
:10331800BC29A9C71946D10513858400EFD0CFADC4
:1033280078441C2393E707F81CA3684419469305BF
:1033380064030905EFD04FAC11679717000083A706
:10334800E72DF98FE38607CE7C24B98BE39207CE6D
:1033580078441C2393E707021CA3D9B98347D403F5
:1033680089C79C2093E707F89CA0684419469305F1
:10337800E4032105EFD04FA84DBF522D0C559307FC
:10338800660093F7F7031CB913858400E5B70111AC
:1033980026CA971400009384643E9C4422CC06CE2F
:1033A800171400001304841A858B6850D9C32AC6E1
:1033B8009717000023A8073CEF00101F0347440796
:1033C800894732456307F700034744078D47631E63
:1033D800F7029716000083A666D4BC520357450728
:1033E80085831307C71263F2E702BC528583B1C312
:1033F800914703474407E31EF7FE6244F240D24474
:103408000561174305E06700A3AC382D3C3D09CFA3
:1034180034256309D7026388F60238A56244F2406E
:10342800D24405616FD0BFA699CF382509EF3CA5D6
:10343800F5B72AC6EF00501762443245F240D2442D
:10344800056145BAEDF7DC4CEDF7034744078947BA
:103458006307F700034744078D47E31CF7FC9147D0
:1034680003474407E31EF7FE49BF63000532011115
:1034780022CC06CE26CA4AC84EC652C456C25825C1
:1034880085472A846318F72C971700009387072F1E
:10349800D44F1547638AE600D44F0D476386E6008C
:1034A800D84FAD476312F7026C386244F240D244F9
:1034B8004249B249224A924A01450561B315B028EA
:1034C800B3C505086FF08FF9163113070064971418
:1034D80000009384A4073347D7029C20E8D08507CF
:1034E80093F7F70F9CA063CAE700972004E0E780F2
:1034F800A08997170000238B070478249D47631F32
:10350800F70483479406B1C38356040763ECF602B5
:103518000C24930730041CAC1305300493F6F60F03
:103528000146977006E0E78000A522856244F240D4
:10353800D2444249B249224A924A0561174305E0FA
:103548006700434885062318D406930530020545CD
:10355800971004E0E780807B2301A4060549238AAD
:103568002407183C8D47631CF70E971004E0E7808A
:1035780000E30D89630F051463162517930760028E
:103588003CA4930750023CAC9307700278243CBCDF
:1035980085476302F70889659385F5701305102739
:1035A800171A0000130A0AC983497401971004E026
:1035B800E78040780E30835ACA002A8913060064CF
:1035C800B3855503814613850532B335B50097A0F9
:1035D80006E0E780C011AA84B335590337460F00C7
:1035E8001306062481463305590397A006E0E780B1
:1035F800001083270A00AA948297B307950003272F
:103608008A00BE8563E4A70063E4E700B385E7406A
:103618004E85EFF0CFE883475403898BE9CB834786
:10362800C403F1C70C58E1C5BC25F1C38947230A77
:10363800F4021946B10513056403EFC0FFFB034705
:10364800C407894763E9E70A22856244F240D24405
:103658004249B249224A924A05616FD05F8389463E
:103668007C346315D70213F7170019CB898B13071E
:10367800500291EB9307700238A43CAC814739B7EC
:1036880013076002C5BF93076002FDB799CF93F691
:1036980017001307500291E6898B13B71700130719
:1036A800670238A4230D0400D1BF3C2C1307400245
:1036B8006368F700930750023CAC3C2C3CA47DBFE8
:1036C800850793F7F70F3CAC13077002E364F7FE26
:1036D800EDB713077002930750023CAC38A4930768
:1036E80060026DB51307500293077002FDB7854756
:1036F800230AF402A9B70327C40A9716000083A671
:1037080026903C27ADC31C37583397140000938488
:1037180064B29044B387E702DA24B387E702130759
:10372800003293870719B3D7E702032744093E9766
:103738003A896364F7006364C7003309C740829617
:10374800B307A9406374A9009844BA97035764075C
:10375800E3FCE7EEF2406244D2444249B249224ACD
:10376800924A0561828083248409829663E9A400D1
:10377800835764073385A440E378F5ECE1BF9717D6
:10378800000083A7A7ABBE94E5B7828001114EC69F
:1037980097190000938989DB22CC03A4C90926CA9A
:1037A80097140000938404A9DA244AC803596408CA
:1037B8008327040906CE3309E90237470F00930629
:1037C800F7231307072452C456C25AC036993359EF
:1037D800E90263E02705171A0000130A6A82338991
:1037E800274183270A0082976368A9023305A94005
:1037F8006347050283570404A30F040085072310B9
:10380800F40483470414639707102285EFD0DFC7B9
:1038180029A29844BA97C1B79C443E99C1BF83274F
:103828000A008297032784086363E50A198D7E3CA2
:10383800DA248E07B387E702130700329387071944
:10384800B3D7E70263E9A708B74A0F00138BFA2337
:10385800938A0A248357040485072310F4048347B2
:10386800041481E72285EFD03FC22285975005E0F6
:10387800E780C0FD63130524032604090327C40851
:1038880094443297BA876364C7006364D700B30768
:10389800D740783CD2242328F408050778BC03577E
:1038A80064083307C7025A97335757033389E740E9
:1038B80063F5E700998E3389F60083270A0082971B
:1038C8006365A9043305A940E34605F825B79C4478
:1038D800998F3E95A9BFA1452285975005E0E780BD
:1038E80000EFA305A4029717000083A7A792638699
:1038F800071C6244F240D2444249B249224A924AE1
:10390800024B89451545056182879C44CA973385D2
:10391800A7405DBF2285EFD07FC12285975005E083
:10392800E780C0F2631B0518CA2483576408B746AA
:103938000F001386F623B387A7029386062403276E
:103948000409230B040283AA8400B297B3D7D702D1
:10395800636FF716B307F7408326C4082324F408D7
:10396800014BB387E6003E8963E4D70063E457015F
:10397800338957411E3023282409A1CB83560404D8
:103988005A3037460F0056B03387E640B387E70210
:103998003A301306062481468145BA97B3C707080B
:1039A8003385A7023EB097A006E0E78040D411CD4A
:1039B8004A9533392501CA95AA876314BB00636405
:1039C8005501B30755412328F40883270A00829735
:1039D8002A8983270A008297E30D25FF83270A0097
:1039E8000329840882976369A90E3305A9406306F1
:1039F800051003DAC4008357640837490F0013071A
:103A0800F923B387470313090924BA97B3D72703C0
:103A1800170700000347977EBA9763E0A70EB335F0
:103A28002503035B2402528681463305250397A0AC
:103A380006E0E780C0CBB30AAB0033054B0337463B
:103A48000F00130606248146814597A006E0E7800B
:103A580000CA15C1B337250352868146B305B9029A
:103A68003305A902BE9597A006E0E78040C8330B4E
:103A7800AB402311640335454D2E23AE89083834F5
:103A88008547631EF704930700FD7CA41705000013
:103A9800032545679C28A1CFEFC09FFD95471717C1
:103AA8000000232BF7CE370710009707000083A7E5
:103AB800E76698C7860A23A85707F2406244D244AB
:103AC8004249B249224A924A024B05618280B306B2
:103AD8005701B387F64049B59C443E9939B79307D7
:103AE80010FC7CA4170500000325456165B78145D6
:103AF800971004E0E78040EB55B79717000023A51F
:103B080007AE9C2885C7170500000325255E97107A
:103B180004E0E780C0266244DC40F240D2444249D7
:103B2800B249224A924A024B056182878345940230
:103B38006244F240D2444249B249224A924A024B74
:103B480001450561B315B028B3C505086FF00F919D
:103B5800011122CC26CA4EC606CE4AC852C456C245
:103B68005AC038358547832405092A84AE896314E9
:103B7800F70C83570508835AC503170A0000130A70
:103B88006A6B035BCA0063FE57191429639BE61826
:103B980003278511631707180327450A63130718B6
:103BA80074351D47639FE6162A3DB38AFA4093078A
:103BB800204E330555030329440937460F001306E1
:103BC800062481463305F5029707000083C707637B
:103BD80033592503B335AB023E99334909082313FA
:103BE80024093305AB0297A006E0E78040B0B3078D
:103BF800950033B5A7002E9503278A00BE8419E1E6
:103C080063E4E700B384E740B307690337470F006D
:103C18009306F7231307072423A09900B697B3D771
:103C2800E702D69763E4F4009D8C31A003278A004D
:103C3800B307F740BE94170900001309693C8327AE
:103C4800090023A09900829763E2A4103385A44059
:103C5800635D050A83270900170B0000130B8B5DB2
:103C6800829703A709006369E50E198D7E3C035707
:103C7800CB008E07B387E702130700329387071933
:103C8800B3D7E70263EFA70C374A0F00930AFA236A
:103C9800130A0A248357040485072310F40483476E
:103CA800041481E72285EFD02FFE2285975005E086
:103CB800E780C0B961E5832604098327C408032780
:103CC8008B00B697BE8463E4D70063E4E700B3844F
:103CD800E7407C3C8356CB002328940885077CBCAE
:103CE80083576408B387D702D697B3D7470363E6E9
:103CF800F40A9D8C8327090023A09900829763E129
:103D0800A40A3385A440E34705F89707000083C752
:103D1800F74E63E6A7069717000023A7878C01458F
:103D2800B9A88357640837470F009306F723B3876A
:103D3800670313070724B697B3D7E702E3F6F4EE51
:103D480003278A002697B304F740F5B597070000C4
:103D580083A7C74EBE94DDBD83278B00998F3E9500
:103D680031B7A1452285975005E0E78040A6A30515
:103D7800A4029707000083A7E74981EF7D55F24029
:103D88006244D2444249B249224A924A024B0561EE
:103D98008280894515458297D5B71D8FBA9499BFFA
:103DA80083278B00BE94B1BF970600009386063721
:103DB8009C42B84B1377F78FB8CB984313678700AB
:103DC80098C39C4393D7374889C701000100010075
:103DD8000100170700000327A7331C4393F7F7CF09
:103DE80093E707101CC317060000032626341C4659
:103DF8003707CEFF7D17F98F1CC69C423707030093
:103E0800B8CB9707000083A7E73099CBD4439047F6
:103E18009842518F98C2944BDC4B9842D98F9CC2E0
:103E28009717000023AA079682809707000083A7A8
:103E3800E72E9C438D8BF9C74111B7E700E04AC0D4
:103E480003A9070026C23707200006C622C4AA8491
:103E58003379E90023A0E7180F10000017140000B9
:103E68001304C491584C8D47631AF7009707000054
:103E780083A7876A01468145454582971947639319
:103E8800E4048347140289CB8347040263969700AE
:103E980097170000A3840790584CA1476315F700B3
:103EA800930780101EB09707000023870714ED3D85
:103EB800B2402244B7E700E023A027119244024908
:103EC800410182809D47639BF40083471402E9D730
:103ED800034704028D47E311F7FC5DBF544C638927
:103EE800E600584C6306F700584CA147E31DF7FA63
:103EF80083471402CDFB5C4C2300F4028547A300E2
:083F0800F40255B782800000AD
:103F10002A8309CA83830500230073007D160503E5
:103F200085056DFA82809707FC1F83A7A7E1170715
:103F3000FC1F0327A7E001456313F7008280F623E7
:103F400099E2D62336959C43C5BF1707FC1F13077C
:103F5000E7FE1C435A23411193860711E117BA97D4
:103F600085651706FC1F232FD6DC1706FC1F2327A9
:103F7000F6DC06C69D051356370063F4E50013060C
:103F800000203387C6009705FC1F23ABE5DA6116D6
:103F900098C2D2A2239306001CC3998FE1175EA397
:103FA000231307004937B2409707FC1F2397A7F652
:103FB000410182809707FC1F83A7C7D81707FC1F02
:103FC0000327C7D701456313F7008280F62381E6F4
:103FD000D6233375D50A9C43FDB7184183A785FFC7
:103FE0006319B7001CC1FD5723AC05FE238FF5FEF6
:103FF0008280232CF6FEC5BF411122C437E400E0C5
:1040000026C204403707200006C6F98C2320E41896
:104010000F10000009E9232094101545B2402244F6
:104020009244410182800347E5FF9307F00F630646
:10403000F700232094101145D5B797C0FB1FE780E8
:10404000000F014523209410D1BF41114AC037E928
:1040500000E022C403240900B707200006C626C2D8
:104060007D8C2320F9180F10000089E5232089108A
:10407000154515A0AA849707FC1F83C7B7E92E85AD
:1040800063F5F400894763EE9700BD37B7E700E0BA
:1040900023A087100D45B2402244924402494101B9
:1040A000828083A785FF99E703C7E5FF9307F00F99
:1040B0006308F7009137B7E700E023A087104DBFF2
:1040C000238F95FE1705FC1F130505C897C0FB1F1E
:1040D000E780E016A165268597F0FB1FE780C08D7D
:1040E00001452320891045BF9707FC1F23AE07C455
:1040F00082804111B7E700E026C2844337072000E1
:1041000006C622C4F98C23A0E7180F1000009707F9
:10411000FC1F83A7A7E41704FC1F130424BA91C74C
:1041200082971C40AA971CC031A09707FC1F83A749
:10413000A7C2FDF70840B74703009387D73F330571
:10414000F502B7A72600938737ECB2403E9508C02A
:104150002244B7E700E023A09710924441018280F7
:10416000411122C406C69707FC1F83A7A7BE1704E8
:10417000FC1F130424DA89C782975C48AA975CC89D
:104180004848B240224441018280B7E700E09843AA
:10419000B706200023A0D718758F0F1000009706D0
:1041A000FC1F83C636D76370D5029706FC1F83A613
:1041B00066BB3325D5201621B3F5B6400EA123A04A
:1041C000E7100145828023A0E7100D4582807971B8
:1041D000B7E700E026D284433707200006D622D472
:1041E0004AD04ECE52CCF98C23A0E7180F10000015
:1041F000930705FF93F7F70F7D476363F70A31478E
:104200003307E5029707FC1F83A707B6BA979C43BD
:10421000C1CB135445003D893315A028AE89B34561
:10422000050822852EC697E0FB1FE780C0572A8924
:1042300039C9B2452285170AFC1F130A2AD5B1379E
:104240009707FC1F83A747B182978357CA002A8428
:1042500081463387370313060064B3B7370313056A
:104260000732B335E500BE95EF90A21DB307850078
:1042700083268A003E8763E4A70063E4D700338780
:10428000D7402324E900B7E700E023A097100145B9
:10429000B250225492540259F249624A45618280D6
:1042A000B7E700E023A097100945DDB7797122D464
:1042B00037E400E04AD003290400B707200006D6FF
:1042C00026D24ECE52CC56CA5AC85EC63379F900B1
:1042D0002320F4180F1000009707FC1F83C797C313
:1042E0006378F500970BFC1F83AB0BA763970B005C
:1042F000B7E700E023A0271199A0970AFC1F938A33
:10430000EAC803AB8A00B74736FE938707C83E9BCF
:1043100083D7CA002E8AAA84B385C702B289814690
:10432000B3B7C70213850532B335B5001306006471
:10433000BE95EF9002116370AB022320241101455A
:10434000B250225492540259F249624AD24A424B24
:10435000B24B45618280829B83D7CA002A841306B0
:104360000064B38537038146B3B73703138505323D
:10437000B335B500BE95EF90C20CB307850003A717
:104380008A003E8463E4A70063E4E7003384E740E7
:10439000D285268597E0FB1FE780E04001C900C574
:1043A000B7E700E023A02711054559BF93E504F0C6
:1043B0004145B3C5050897C0FB1FE78020CA11E936
:1043C0009707FC1F83A787BA85D7A68511458297D3
:1043D00005B71707FC1F1307A7981C4389EF08C3ED
:1043E00085472326050000C52311450104A11CB102
:1043F0002322050075B73E87DC47F5FF48C7CDB7D8
:104400007971B7E700E026D284433707200006D64B
:1044100022D44AD04ECE52CC56CA5AC85EC662C4C6
:1044200066C2F98C23A0E7180F10000035C12A8955
:104430002E8AB28AB6894144B14C170BFC1F130B6C
:10444000AB92130C0003B30B940383270B00DE978E
:104450009C43B9EF135544409375F4005686137589
:10446000F50FB315B028B3C50508893531C18327C9
:104470000B00DE9723A0270123A2470163840900D4
:1044800023808900B7E700E023A09710014521A011
:1044900023A097100945B250225492540259F24970
:1044A000624AD24A424BB24B224C924C45618280C6
:1044B0000504E31A84F9B7E700E023A0971021452B
:1044C000D9BF011122CC37E400E026CA04404AC813
:1044D0004EC652C406CEB70720002A892E8AB2895A
:1044E000FD8C2320F4180F100000C933D2854A85B3
:1044F00097E0FB1FE780202B01ED2320941021453E
:10450000F2406244D2444249B249224A0561828063
:104510009707FC1F83D747A8B38537032A8913065B
:1045200000648146B3B7370313850532B335B50050
:10453000BE95EF8012712322A9002320941001451B
:10454000C1B7011126CAB7E400E04AC803A90400B4
:1045500022CC4EC6B707200006CE52C4AA892E84AC
:104560003379F90023A0F4180F10000097E0FB1F27
:10457000E7806023170AFC1F130ACA991DE1A28570
:104580004E85213183470A006382370523A0241119
:104590001945F2406244D2444249B249224A056177
:1045A000828023110500A2854E85C53683470A0007
:1045B0006386370123A024110145E1BF17F7FB1FD4
:1045C000130727791E23C18F1EA3EDB797F7FB1F93
:1045D000938727789A23598C82A34DBF01114AC82B
:1045E00037E900E022CC03240900B707200006CEFB
:1045F00026CA4EC67D8C2320F9180F1000009307A1
:10460000F00263E7A704B144B304950297F9FB1FD6
:104610009389897583A70900A6979C4395CB9375C9
:10462000F5001181B315B028B3C50508193F83A75C
:1046300009000145A69723A0070023A20700232015
:104640008910F2406244D2444249B24905618280F5
:10465000B7E700E023A087100945E5B74111B7E7A8
:1046600000E026C2844306C622C437072000F98C26
:1046700023A0E7180F10000097E0FB1FE780A012AF
:1046800019E90145B2402244B7E700E023A09710A2
:10469000924441018280004597F7FB1F83A7C76BB7
:1046A00082979707FC1F9387678E6367A4029847DA
:1046B000B74636FE938606C83305A4403697E372A4
:1046C000E5FC13070064B335E502D22781463305C4
:1046D000E502EF8012577DB798473A94C9BF411160
:1046E00006C697F7FB1F23A7A7660295B240970758
:1046F000FC1F23ADA782014541018280914763E9F8
:10470000B7009707FC1F93872787B3C5F52088C19B
:1047100082804111514681451705FC1F1305C5854F
:1047200006C622C426C297F7FB1F23AB076297F782
:10473000FB1F23A1076297F7FB1F23AF076097F7C3
:10474000FB1F2387076097F7FB1F23A1076097C014
:10475000FB1FE780A0C613068002814517F5FB1FEB
:104760001305457B97C0FB1FE78040C5EFF0EFFDC9
:1047700097F7FB1F9387877CE82BFC3B17F4FB1F05
:104780001304447985453E958D473305F5029947D5
:1047900097F4FB1F9384445D39051375F50F28A02A
:1047A0003305F502130505243345050897C0FB1FA3
:1047B000E780C08A88C035C93020994781453306D3
:1047C000F6021306062497C0FB1FE78020BF9C401B
:1047D000382097F4FB1F93846458938707249CC068
:1047E000B347F72017F7FB1F232EF756F5381D2187
:1047F0001C30944017E6FB1F1306260333C7D7204F
:1048000010C3138717001377F70F17E6FB1F130664
:1048100066FB3347D72010C313873700890718B0CA
:1048200093F7F70FB3C7D72090C3B2402244924406
:104830004101828097F6FB1F9386C66D2A87BC22B2
:104840008832637DF5001306150097F7FB1F83A7D9
:10485000E75090B2B347F52098C382801305F00F5C
:1048600082801C41E5CB370700F07D8FB706002022
:1048700089476312D70E5A21411122C406C62A84E1
:1048800069C719469305F00F690597C0FB1FE780BC
:1048900000C605478D47630AE50A1C4491C758586E
:1048A000994745C7185C55C31306C003814517F5E2
:1048B000FB1F1305A56897C0FB1FE78020B01306F8
:1048C000C003A28517F5FB1F1305456797C0FB1FA3
:1048D000E78040A897F7FB1F93874766DA2701E731
:1048E00013070010DAA7F82719E30547F8A79A2B52
:1048F00019E36D479AABF83719E31547F8B7B82BAA
:1049000019E30547B8ABB83B19E3F837B8BBD83B58
:1049100011C7937637000983F4ABF8BBD82B19E3A2
:104920005547D8AB182C01E71307C00398AF9C5725
:1049300091C7829797F7FB1F2392A75EFD5717F742
:10494000FB1F2307F75CF1338147B24022443E85C9
:104950004101828089473E85828079714ECE97F9E8
:10496000FB1F9389A96283A7090006D622D426D209
:104970004AD052CC829713090064B335250303D67D
:10498000C900814617FAFB1F130ACA5832C63305FD
:104990002503EF80122B83248A012A840145638634
:1049A000840232463305944063EF840003A58900F6
:1049B0008146B335A9023305A902EF809228B307D7
:1049C000954033858700232C8A00B250225492549C
:1049D0000259F249624A45618280011122CC0A855E
:1049E0002E84414697950200938585DF06CEEFF031
:1049F0002FD218083324E420035704FFF240624406
:104A000097F7FB1F83D7675937450F00BA971305F0
:104A100005243355F5020561828097F7FB1F83D784
:104A2000C75751471D45637CF7027947194563789D
:104A3000F7021307200315456373F7021307B00449
:104A40001145637EF700130740060D456379F700B3
:104A50001307600909456374F70013B5B70F828027
:104A6000411122C426C22E84AA8406C6058CEFF00A
:104A70004FE8B327A402B240224433859700137550
:104A8000F50F924441018280411122C426C22E8436
:104A9000AA8406C6058CEFF0CFE5B327A402B24086
:104AA00022443385970033450508924441018280B2
:104AB000411122C426C22E84AA8406C6058CEFF0BA
:104AC0004FE33335A402B24022442695924441017B
:104AD000828097F7FB1F23ABA728828041114AC031
:104AE00017F9FB1F130989458327890206C622C4CB
:104AF00026C28DCF829797F4FB1F9384A4419E24F6
:104B00002A848DC733F7A70A33470708B3D7A70A04
:104B1000B3C70708B307F74051476359F700832726
:104B2000C90291C38297EF10622B82A4B240224443
:104B30009244024941018280011122CC97F7FB1F68
:104B400023A6072217F4FB1F1304443F5C5406CE30
:104B5000AA8581C72AC68297B245C1C19C41054535
:104B6000ADCB9C45BDC7DE25ADC7FE25BDC39C2989
:104B700081CB7C287838BA97634DF504DC41B1CB02
:104B80001306400217F5FB1F1305454097B0FB1FA6
:104B9000E780407C97F7FB1F9387473F984397F642
:104BA000FB1F23ABE61A183C19EFCA27930780575F
:104BB00037460F003305F50213060624814681456A
:104BC000EF80320808BC17050000130545D9013EE7
:104BD0000145F24062440561828097F7FB1F23A9DB
:104BE000073497F7FB1F9387673A17C7FB1F130715
:104BF00027DC98C337873200FD56130727A194C7D7
:104C0000D8C797F7FB1F238B0738B7C7004023A4EB
:104C1000D72649B7011122CC17F4FB1F1304043225
:104C2000084406CE26CA4AC801E90545F240624456
:104C3000D2444249056182805C58E5DB185C75D737
:104C40007000854582971844B247E300F7FE4A2476
:104C50009305E00417F9FB1F1309C92B97B0FB1F3D
:104C6000E780C03F2320A90269D152249305F00FA9
:104C7000814497B0FB1FE78060747C2403260902FF
:104C800063C1F402328597B0FB1FE780404A0145BB
:104C900097F7FB1F23A0072A97F7FB1F23AE0728D0
:104CA00071B74E241844B3879502898185043385F2
:104CB000E7001C5C08C28297C9B7011122CC17F427
:104CC000FB1F1304A4271C4426CA4EC656C206CE98
:104CD0004AC852C45AC0AA84AE89B28A6388071AE5
:104CE000585839CB1307F01F6366A71017FAFB1F3C
:104CF000130A4A2203290A02631209044A24956509
:104D0000938515E097B0FB1FE78040352320AA026A
:104D10002A861DC14E245C580844898182971C4410
:104D200003290A022322FA028947639EF402C1473B
:104D30009305090C6381F9042945BDA003274A02A4
:104D4000E384E7FE4A249565938525E097B0FB1F31
:104D5000E780C0302A896DD14E242A865C580844E9
:104D600089818297D1B78D47639AF404C14793052F
:104D7000490DE393F9FCB8219307A0056312F706E8
:104D80009E21639F97044E869105568597B0FB1F21
:104D9000E780405C83270A02638727014A8597B032
:104DA000FB1FE780C0380145F2406244D2444249CB
:104DB000B249224A924A024B056182809147639729
:104DC000F4009305890EE39999F675B793070010DF
:104DD000E394F4F6A147E3E137F79305090F61BFC8
:104DE00083270A02E38A27F54A8597B0FB1FE780ED
:104DF000003499B71D67637FE506130705E0994600
:104E00003347D702562417FBFB1F130BAB10330796
:104E1000D702330AF70083274B0263964701032921
:104E20000B02631109024A249305E00497B0FB1FAB
:104E3000E780C0222A8909D14E245C582A868981BC
:104E40005285829791451307A00593F5C50FB307C7
:104E5000B900B4236399E602962363949602910500
:104E60004E86CA95568597B0FB1FE780A04E8327D4
:104E70000B021DB7A166F916E3E0A6EC3307E54087
:104E800051B7AC33D9B783270B02A9BF97F5FB1FE6
:104E900083A5450AE38205EA91479306A00593F7A7
:104EA000C70F3387F5003023E318D6E81223631BBE
:104EB000960091074E86BE95568597B0FB1FE780FA
:104EC0006049D5B53C33E1BF97F7FB1F93870707D0
:104ED000984721C7985F31C385466310D5044111B7
:104EE00022C417F4FB1F1304E402105006C615C2B7
:104EF000CE27485089810297085097B0FB1FE78062
:104F0000002397F7FB1F23A7070297F7FB1F23A593
:104F10000702B240224441018280828001114AC8C6
:104F200017F9FB1F130989014EC68329890022CC7A
:104F300026CA52C406CE56C2AA842E84328A638DF3
:104F4000091A8327890399EB2945F2406244D24428
:104F50004249B249224A924A056182808327490325
:104F6000E5D79307F01F63E0A70C97F9FB1F938920
:104F700069FA83A7090295CF0325890083A749020F
:104F80006395A7048947639FF404C147E31EF4FABD
:104F900003A509021305050C9307A0053CA106A172
:104FA0002286D285110597B0FB1FE780A03A014504
:104FB00069BF0355C9009305E00497B0FB1FE78064
:104FC000E00923A0A9024DF941B78355C900832701
:104FD000490303A60902898182978327890023A2B6
:104FE000F9024DB78D47639AF400C147E31EF4F40C
:104FF00003A509021305450D45B791476399F400D0
:10500000E31494F403A509021305850E71B7930701
:105010000010E39BF4F2A147E3E887F203A509023D
:105020001305050F95BF9D676373F506930705E0AC
:105030001947B3C7E7020357C90097FAFB1F938AC2
:105040006AEDB387E702BE9983A70A02A1CB83A7C3
:105050004A026391370703A50A0291479305A00509
:105060001308F00F13F7C70FB306E500B022631360
:10507000B60683D80600B032639C9804B307F640A6
:1050800063C6870411072286D2853A9529BF216716
:105090007917E36BA7EAB307F54071BF0355C90061
:1050A0009305E00497B0FB1FE78040FB23A0AA0212
:1050B00059FD59BD8355C9008327490303A60A0238
:1050C00089814E85829723A23A0371B72390060106
:1050D000B28749BF3386870011061308F00B63744B
:1050E000C8002D459DB5ACA213063400719A110677
:1050F000B29786A2BCB279B797F9FB1F938989E171
:1051000083A709029DCB03A5090291471308A005B7
:105110009305F00F13F7C70FB306E500B022631035
:10512000060583D80600B03263979800B307F640AF
:10513000E3DA87F48EA2B287F1BF8347E900035513
:10514000C9009305E0043305F5023345050897B01F
:10515000FB1FE780A0F023A0A90255F5F5B3035685
:10516000C9008345E900B385C5023386870011066F
:10517000E3E9C5F62381060185BF014582809C21B4
:105180001CA1BE211CB1BE21A1833CA1DC213CB1EC
:105190001145828097F7FB1F23AE07BC97F7FB1FD3
:1051A00023A807BC82800DCD411122C426C206C6A9
:1051B000AA842E84014585C1228541469785020037
:1051C0009385056597B0FB1FE780C0189C200545B7
:1051D0005CA49C305CB4B240224492444101828081
:1051E00001458280011122CC26CA06CE8947AA84B5
:1051F0003284639EF5006383B6024147814763951D
:10520000E6048A854D3741468A8522850DA84147A7
:105210006392E504638FF600639EB6022E86A28534
:105220006244F2402685D244056117B3FB1F670034
:10523000E3238A853285853F41468A85268597B056
:10524000FB1FE780A022AA87F2406244D2443E8539
:10525000056182808147CDBF97F7FB1F23AAA7B0C6
:10526000828097F7FB1F23A7A7B08280011122CC71
:10527000622106CE26CA4AC84EC63DC8832985008B
:105280002A88AE8403C90900814713174960635512
:105290000702B147054563F68704035528005114FA
:1052A000334404084E8633878900A2868545EFB0D3
:1052B0007001B337A0008507135569487D14137931
:1052C000F903334404089CA088B023812401C2A0C0
:1052D000014719C01387190098C409476383E70081
:1052E0000145F2406244D2444249B249056182809C
:1052F0000545C5BFC167F917630AF502D94763F7CA
:10530000B702011122CC2EC606CE2A84EF90600689
:10531000B2456368B50022856244F24005616FA022
:10532000407BF240624405450561828005458280EC
:10533000C167F9176314F5006F90A003411106C609
:10534000EFA0C06711E15D45B24041018280914705
:10535000639DF5001C211CA23C211831A207D98FA6
:105360003EA23C3101455CA2828011458280411100
:10537000814522C426C206C6AA849D232A8409E93F
:1053800097F7FB1F83A7C79E81C7F945268582979C
:10539000B2402285224492444101828039714ED626
:1053A00052D45AD05ECE06DE22DC26DA4AD856D255
:1053B0002A8A2E8BB289B68B0DE79D3F9145EF90DF
:1053C00060092A844D49854A19EDF2506254D2543D
:1053D000B259225A925A025BF24B4A8542592161D4
:1053E00082803A84814A230034018544630A0B0099
:1053F000DE8513051400029B93041500B3C4040852
:105400009399496063D30902C1455285EFA0406971
:10541000654915E533069400A6852285EFB0A030D6
:105420002A8911EDB104B3C4040891472C005285B8
:105430007C8422C66485EF90707E2A8959D5E386E4
:105440000AF8228597B0FB1FE78060CEBDBF01112F
:1054500022CC26CA4AC84EC606CE2A893284B689CC
:10546000353FAA840DE197F7FB1F83A7A79081CF53
:1054700005476317E40003C4090005041374F40F1F
:10548000A2854A858297F24062444249B249268504
:10549000D24405618280AE8601470546970500002B
:1054A000938525CE6DB79E211CA19E21A1831CB1A1
:1054B000094582809E211CA19E21A1831CB1BE2191
:1054C0003CA1BE21A1833CB1114582809E211CA13B
:1054D0009E21A1831CB1BE213CA1BE21A1833CB170
:1054E000DC315CA1FC215CB18A2519053345050836
:1054F00082809E211CA19E21A1831CB1094582802E
:105500009E211CA19E21A1831CB1BE213CA1BE21D4
:10551000A1833CB111458280CA21060533450508A7
:1055200082809E211CA19E21A1831CB1AA21090574
:105530003345050882809E211CA19E21A1831CB1B8
:10554000BE213CA1BE21A1833CB1CA211105334536
:10555000050882809C211CA1054582809E21411165
:1055600022C406C61CA19E212E841105A183A30E70
:10557000F5FEBE219505230FF5FE83D7D5FFA18348
:10558000A30FF5FE03C6F5FF97B0FB1FE78080DC95
:105590004820B24022441105410182808947639925
:1055A000F5001C3118210145A207D98F1EA2828067
:1055B000114582809A21011106CE22CC2EC6D947F0
:1055C00063F4E7022A84EF80D05AB2469E22636DCC
:1055D000F50022856244F240014709469705000024
:1055E0009385A5EC05615DBBF24062440945056108
:1055F0008280AA87A9C11421FD150547B3C50508F6
:105600006398E60013D725008D89114589CD8280E6
:10561000094711456392E602494533D7A502B3F520
:10562000A502114591E9114501CB850734A21AA2C3
:105630005CC20145828011458280AE8601471146D9
:1056400097050000938545E791BB13F73500AA87BE
:1056500001EB8981114591C50EA25CC20145828092
:1056600011458280D8218947631BF702011122CCA2
:105670002A84C84506CEAE8601C92EC69D4597B080
:10568000FB1FE78040B8B2462A8722856244F24079
:105690001946970500009385A5E3056101B3094507
:1056A000828099E1114582801C2105473EA2E37B5F
:1056B000F7FEFD1593F5F50F33D7F502B387E70233
:1056C000E392F5FE050548C21AA201458280DC215D
:1056D0000947AE866385E70041476399E7000147C4
:1056E0002146970500009385A5E74DB909458280BD
:1056F0000EA291E1014548C201458280AE86014774
:10570000294697050000938505DF49B90EA291E16E
:10571000014548C201458280AE8601473146970562
:105720000000938525DE9DB90EA291E1014548C296
:1057300001458280DA21854763FFE702011122CC0F
:105740002A84884106CE2EC615C1854597B0FB1F19
:10575000E78060AB2A8722856244B246F240394630
:1057600097050000938585DB05610DB9F240624421
:1057700009450561828009458280AA878DC5182167
:105780008D46114563F2E602FD15B3C50508B3C6A3
:10579000E5023308D70263990501850716A23AA2EC
:1057A0005CC20145828011458280DC210947AE86BA
:1057B0006385E70041476399E70001474146970544
:1057C00000009385E5D9D9BE094582803335B00004
:1057D0000A058280011122CC26CA06CE982585476B
:1057E000AA842E844946631FF70099363E20491546
:1057F0001306200963C8A700F2406244D244094559
:1058000005618280183485476314F7001366060427
:10581000484001C98D4532C697B0FB1FE780A09E66
:105820003246A2866244F2402A872685D2449705F2
:105830000000938545CF056195B68D4763F7B702A4
:105840001C311821F115A207D98F1EA23C31382135
:10585000B3C50508A207D98F014799C113074500B1
:105860003EA24EA218C601458280114582800111D8
:1058700022CC2A84884506CEAE8601C92EC695451F
:1058800097B0FB1FE7802098B2462A8722856244A2
:10589000F240594697050000938525CA0561FDBC75
:1058A0003335B0000A058280AE8601476146970510
:1058B0000000938565CADDB48547114563F1D702C1
:1058C0001C320C220945A207CD8F81456384A600B6
:1058D00093052600F9161EA336A34CC3014582800A
:1058E000014781467946814555BC9E211CA19E21D8
:1058F000A1831CB109458280BC2105471CA18A21D6
:105900006397E7000A050505334505088280C94706
:105910003305F502CDBF8A210A053345050882808B
:10592000BE211CA18A21BE213305F50205053345A0
:10593000050882808A2182808A2182808A21828051
:10594000BE211CA18A21BE213305F5020505334580
:10595000050882809E211CA19E21A1831CB1BE212D
:105960003CA1BE21A1833CB1CA21110533450508E4
:1059700082809E211CA19E21A1831CB1AA21090520
:10598000334505088280894711456398F6001C322B
:1059900014220145A207D58F1EA382809A21D947E0
:1059A000AE8663F9E70001470D4697050000938531
:1059B00005F471BC094582801145639DA6001C3227
:1059C00014220145A207D58F1EA33C323422A20720
:1059D000D58F3EA38280BC210547FD1793F7F70FB3
:1059E0006361F7049E2195CF011122CC2A84C8411E
:1059F00006CE2EC615C1894597B0FB1FE780A08053
:105A00002A8722856244B246F24015469705000077
:105A10009385C5EE056125BCF240624409450561E8
:105A2000828009458280954763F0D706411122C4E0
:105A300026C24AC006C61C323A841822A207B28483
:105A4000D98F1EA03C32382293854400A207D98FFB
:105A50003EA089475CA0094613055400368997B0DB
:105A6000FB1FE780208F194781476304E900938774
:105A70006400691923142401B2405CC42244924496
:105A80000249014541018280114582809E2195CFC6
:105A9000011122CC2A84C84106CE2EC615C18545E7
:105AA00097A0FB1FE78020762A8722856244B246B2
:105AB000F2401D4697050000938525E6056141BA31
:105AC000F240624409450561828009458280994718
:105AD000B2856388F600D147114541466384F600DC
:105AE00082800946411106C650A39C3194211305BA
:105AF0005700A207D58F1EA3BC31B4219105A20780
:105B0000D58F3EA397B0FB1FE780C084B24001450C
:105B1000410182809E219DCF011122CC2A84C8415F
:105B200006CE2EC61DC1894597A0FB1FE780A06D3C
:105B30002A8722856244B246F24025469705000036
:105B4000938545DE05616FF09F90F2406244094500
:105B50000561828009458280894711456398F60076
:105B60001C3214220145A207D58F1EA38280011189
:105B700022CC2A84C84106CEAE8601C92EC68545F0
:105B800097A0FB1FE7802068B2462A8722856244DF
:105B9000F2402D4697050000938505DA05616FF008
:105BA0001F8B19BD011122CC2A84C84106CEAE86B6
:105BB00001C92EC6854597A0FB1FE780C064B24689
:105BC0002A8722856244F240354697050000938576
:105BD000E5D605616FF0BF8793F71600114581EB9D
:105BE00089476386F600858256A310C301458280EB
:105BF000011122CC2A84C84106CE2EC61DC185457E
:105C000097A0FB1FE78020602A8722856244B24666
:105C1000F2403D4697050000938585D205616FF0FF
:105C20001F83F24062440945056182809E219DCF19
:105C3000011122CC2A84C84106CE2EC61DC1894539
:105C400097A0FB1FE780205C2A8722856244B2462A
:105C5000F2404546970500009385C5CE05616FF07B
:105C60000FFFF24062440945056182800945828048
:105C7000854763F4D70208A70CB71C320C220945EC
:105C8000A207CD8F81456384A60093052600F916EF
:105C90001EA336A34CC30145828011458280014773
:105CA00081464D4681456FF08FFA8D47114563F56A
:105CB000D7021C320C22A207CD8F1EA33C322C220D
:105CC000A207CD8F81456384A60093054600F11697
:105CD0003EA356A30CC701458280011122CC2A8421
:105CE000884506CEAE8601C92EC6954597A0FB1FF6
:105CF000E7806051B2462A8722856244F2405D46C1
:105D000097050000938545C505616FF04FF4854701
:105D100011456395F6001C2201451CA382800147B2
:105D20008146654681456FF08FF2011122CC2A84AD
:105D3000C84106CEAE8601C92EC68D4597A0FB1F71
:105D4000E780604CB2462A8722856244F2406D4665
:105D500097050000938525C205616FF02FE40111BE
:105D600022CC2A84C84106CEAE8601C92EC68D45F6
:105D700097A0FB1FE7802049B2462A87228562440C
:105D8000F2407546970500009385E5BE05616FF00A
:105D9000EFE0011106CE2EC6EF90703E19C5B24558
:105DA000F2402A2105616FD0B07AF2404945056181
:105DB000828097E7FB1FA38507FE97E7FB1F2381E0
:105DC00007FE97E7FB1F23AB07FC97E7FB1F23A505
:105DD00007FC97E7FB1F23AF07FA97E7FB1F23A9F1
:105DE00007FA97E7FB1F23AB07F897E7FB1F23A5ED
:105DF00007F897E7FB1F9387A71B3706840390D309
:105E00003707B40037C6070098C3130606B83747EC
:105E1000A000D8C3D0D33707100041669306070A05
:105E2000B70550009308060194C723A4170393866F
:105E30000501930816F8D4C723A61703B706D007A1
:105E4000B7087F001308070513850601410723A83B
:105E50001703B0C393081600938606051386150032
:105E6000D8CBF8C323A8070188CF23AE070023AA05
:105E7000170323AC070223AE070223A40704F0C7CD
:105E8000B4CB23AA0704ACCF23AE0705B8D337079A
:105E9000A000F8D71307000AB8DB1307C01CF8DB13
:105EA00037071400B8DF0547F8DFE8D323A4070657
:105EB000930710F817E7FB1F232CF71682800111B8
:105EC00052C42A8A214522CC26CA4AC84EC606CECA
:105ED0002E84B2893689BA8497A0FB1FE780C03729
:105EE00005C9930700FD1CA19947A30045013CA1EA
:105EF0002303250164B123123501AA85228562445A
:105F0000F240D2444249B249224A05616FE0EF9320
:105F1000F2406244D2444249B249224A0561828039
:105F200097E7FB1F23ACA7E6828097E7FB1F23A51B
:105F3000A7E6828097E7FB1F23AEA7E4828097E75E
:105F4000FB1F23A7A7E48280011122CC26CA4AC8DE
:105F500006CE4EC62A89AE840144B309890063691E
:105F60009400F2406244D2444249B24905618280C1
:105F7000EFE02F98B3470508A1832380F90093072A
:105F8000140093F7F70F850963F89700CA9709047F
:105F900088A31374F40FD1B73E84D1B7411122C442
:105FA00017E4FB1F130404096A20C16706C6FD1726
:105FB000630EF50017E6FB1F0346C62997E5FB1F96
:105FC000938505DCEF90A07CFD577EA0B240224473
:105FD0004101828009C925151375F50F1335850E0A
:105FE0001345150082800145828023900500C9C2B7
:105FF000797122D426D252CC56CA5AC806D64AD073
:106000004ECE5EC62A8B2E8AB28A3684814463FFC6
:106010005405B307940083C907001389140033495A
:10602000090863850904B387290163C1FA04B3072A
:10603000240183CB07005E85713F0DC99387F9FF6B
:106040002310FA0063906B03050933052401B25055
:10605000225492540259F249624AD24A424BB24BFC
:1060600045618280CE94B3C4040855B70145C5B7D5
:1060700001458280011122CC26CA4AC84EC606CEEE
:1060800097E4FB1F938404FB2E89D0C88CC8C8C436
:106090002A8441469305F00F4A8597A0FB1FE780AD
:1060A00000458549631935038848C145713D41461E
:1060B0009305F00F228597A0FB1FE7804043054919
:1060C000631525036244C844F240D2444249B249B0
:1060D000C145056195BD414681454A8597A0FB1F95
:1060E000E780E040E31535FDC1B741468145228593
:1060F00097A0FB1FE780A03FE30625FDF240624426
:10610000D2444249B24905618280411122C426C26B
:106110002E84AA8413060002814517E5FB1F130590
:1061200065F106C64AC097A0FB1FE780202917E942
:10613000FB1F130929F097E7FB1F238F8710A3018B
:106140009900EFD03043854719C181474945230065
:10615000F900B240224492440249410182809DC923
:106160001DC985476318F500DC3193E707FCDCB1F6
:106170000545828089476316F500DC3193F7F70304
:10618000FDB78D47E316F5FEDC3193F7F70393E790
:106190000704F1BF014582808DC10DC1DC311307B9
:1061A000000C054593F7070C638AE700130700040A
:1061B00009456395E7000D458280014582804111C4
:1061C00022C4005D06C626C21DC8AA84085009C59F
:1061D00097A0FB1FE780A0F5485009C597A0FB1FBB
:1061E000E780E0F4085409C597A0FB1FE78020F47E
:1061F000228597A0FB1FE78080F323AC0402B24006
:10620000224492444101828019ED97E7FB1F83C726
:1062100087E217E5FB1F130565E391CB17E5FB1F2D
:10622000130585B6828017E5FB1F130525E28280E2
:1062300017E5FB1F034525E0828017E5FB1F0325BB
:1062400025E0828017E5FB1F0325C5DF828097E7E5
:10625000FB1F83A767DF8843828017E7FB1F1307B5
:1062600067DD544B9C4285079CC228339307F00F8F
:106270006307F500916517C3FB1F6700E373828016
:10628000011122CC06CE2E8432C6EF90C07F9147FA
:10629000B245631EF50097E7FB1F83A767AF99CF51
:1062A0009C4389CF22856244F2400561828797E74B
:1062B000FB1F83A767AE99C3DC43E5B7F240624496
:1062C000054505618280797122D42A844A214ECE07
:1062D00006D626D24AD097D0FB1FE780208497E9C4
:1062E000FB1F9389E9AB29E983C409009307F00FE9
:1062F000639DF40097E5FB1F83C595AA2685513C55
:1063000009E597E7FB1F238D07A84A20EF90A077A8
:106310009147631CF50097E7FB1F9387A7D1562091
:10632000FA236394E6007D57FAA3B25022549254A4
:106330000259F24945618280582504212A893AC6CA
:10634000BD3D4A85EF90F0324A20EF90006F83C741
:106350000900324799C3E38F97F89307F00F522053
:10636000E385F4FA74202820A685913E79BF7971DF
:106370005AC82A8B2E854ECE52CC56CA06D622D467
:1063800026D24AD05EC62E8AB28AB68997C0FB1F33
:10639000E780C07875C5045D2A89FDC09C5013054F
:1063A000400391E361459C5489C79307450133C578
:1063B0000708638609009307C50133C50708DC5049
:1063C00089C79307750133C5070897A0FB1FE780AE
:1063D000A0E82A8455C56146814597A0FB1FE78048
:1063E000E0FD97EBFB1F83CBABBF63940B00834BAC
:1063F0000900930700FD1CA0A947A30064013CA06D
:10640000230354018C50231244011305840191C9C4
:1064100008C47146130A440397A0FB1FE78080F36A
:1064200052858C5491C948C45146130A450197A01E
:10643000FB1FE78020F25285638C090008C8714673
:10644000CE85130AC50197A0FB1FE780A0F05285F7
:10645000CC5099C548C85D4697A0FB1FE78080EFE8
:10646000A2855E85EFD07FBE2254B2509254F2498D
:10647000624AD24A424BB24B4A850259456181B3C6
:10648000B250225492540259F249624AD24A424BC3
:10649000B24B4561828001114EC6AA892E8526CA5B
:1064A00006CE22CC4AC8AE8497C0FB1FE7800067A7
:1064B00021C917E9FB1F0349A9B263140900034965
:1064C0000500194597A0FB1FE78000D92A840DC954
:1064D0008145194697A0FB1FE78040EE930700FD1A
:1064E0001CA0B947A30034013CA046A0A285624489
:1064F000F240D244B2494A85424905616FD0FFB4A7
:10650000F2406244D2444249B249056182807971C5
:1065100062C42A8C2E8526D24ECE52CC56CA5AC878
:106520005EC606D622D44AD0AE84B28B368BBA8AE7
:106530003E8AC28997C0FB1FE780405E35C52A8925
:10654000414597A0FB1FE78020D12A8431CD4146E9
:10655000814597A0FB1FE78060E617E5FB1F034519
:1065600025A819E103450900930700FD1CA0BD47BC
:10657000A30084013CA023047401A3046401230547
:106580005401A305440146A023263401A2852254C8
:10659000B25092540259F249624AD24A424BB24B2B
:1065A000224C45616FD07FAAB250225492540259B6
:1065B000F249624AD24A424BB24B224C4561828038
:1065C000011126CAAA8439454AC84EC652C406CE0D
:1065D00022CC2E8AB289368997A0FB1FE780C0C7DC
:1065E00015CD9307000D1EA1B1472A842312450142
:1065F0003CA1CE851905194697A0FB1FE78080D5E1
:1066000023062401A2856244F2404249B249224A4B
:1066100013F5F40FD24405616FD03FA3F2406244FA
:10662000D2444249B249224A05618280411126C2C0
:1066300006C622C44AC097E4FB1F9384A49FB830C7
:106640009307F00F6308F7042A89394597A0FB1FC9
:10665000E78080C02A841DCD930700FD1CA1A30004
:1066600025012301050097E5FB1F9385259E0D0558
:10667000194697A0FB1FE780E0CD9E24A285A83095
:106680003EA49C305CA42244B240924402494101A1
:106690006FD0BF9BB24022449244024941018280A4
:1066A000011156C2AA8A314526CA4AC84EC652C4EA
:1066B00006CE22CC5AC0AE84328AB6893A8997A0D7
:1066C000FB1FE78060B92DCD2A84268597C0FB1F6C
:1066D000E780C04409C55825A1476311F70417EBAB
:1066E000FB1F034B5B95930700FD1CA09D47A30078
:1066F00054013CA046A02313440123143401231564
:106700002401A2856244F240D2444249B249224A5D
:10671000924A5A85024B05616FD03F9317EBFB1FDE
:10672000034B9BB3E3910AFC97D7FB1F83A7477BDF
:106730009C47D5DBCA864E86D2852685829765B76B
:10674000F2406244D2444249B249224A924A024B40
:1067500005618280411126C2AA84214522C406C651
:106760002E8497A0FB1FE78020AF15C5930700FD7F
:106770001CA1C5473CA13C30AA853CB15E205EA16E
:106780007C207CA17C307CB12244B240268592449E
:1067900041016FD09F8BB2402244924441018280DC
:1067A00041114AC02A89714526C206C622C4AE8458
:1067B00097A0FB1FE78040AA3DC5930700FD1CA1E1
:1067C000F5473CA1BC302A849385C4003CB1DE204F
:1067D00031051946231CF5FEFE20231DF5FE9E24DF
:1067E000231EF5FEBC24230FF5FEBC34A30FF5FEDB
:1067F00097A0FB1FE78000B6BC28A2854A853CA86D
:10680000DE285EA8FC287CA8FC387CB89C2C1CAC3C
:106810009C3C1CBCBC2C3CAC2244B240924402497F
:1068200041016FD09F82B24022449244024941010B
:10683000828001114AC82A89614526CA4EC606CE01
:1068400022CCAE89B28497A0FB1FE780E0A025C1CF
:10685000930700FD1CA1BC302A84938584001CB1E1
:1068600095473CA1FC3011051946A30FF5FE97A0F2
:10687000FB1FE78020AEDE2023063401A2853EA464
:10688000BE2C4A857EA4DE2C1EA8FE2C3EA883C703
:1068900004025CA883C714025CB8BE30F240D24444
:1068A0007EA862444249B24905616FD00FFAF240B6
:1068B0006244D2444249B24905618280411122C4F6
:1068C00006C617D4FB1F1304E4763C209DCBAA8593
:1068D000194617D5FB1F1305254B97A0FB1FE78013
:1068E00060A7282097D5FB1F9385054AEFF03F87C7
:1068F0002244B24017D5FB1F1305054941016FD053
:106900002048B2402244014541018280411126C203
:1069100006C622C44AC097D4FB1F9384A471B83022
:106920009307F00F6302F7042A89294597A0FB1FFC
:10693000E78080922A840DC9930700FD1CA1A1471E
:10694000A30025013CA1BC2097D5FB1F9385C5431F
:106950001105A30FF5FE194697A0FB1FE780809F46
:10696000A830A285EFD06FEEB8208D47631FF700E7
:1069700097D7FB1F83A7074289CB9C4799C722441F
:10698000B2409244024941018287B240224492447B
:10699000024941018280797122D406D626D24AD09A
:1069A0004ECE52CC56CA09444DCD2A890A212E8A90
:1069B000514497C0FB1FE7806016AA845DC197EA27
:1069C000FB1F938A2A8983C74A0005474944FD175C
:1069D00093F7F70F6377F7085825A1476314F7007B
:1069E00063110A089C5C4544ADEF91659385457140
:1069F0001305C0029790FB1FE780406688DCAA89D8
:106A00004D4425C11306C002814597A0FB1FE780B6
:106A1000E09A835709009386490036852391F9004F
:106A200071469305490036C697A0FB1FE780809208
:106A300089472380F900DC24B2460356090083C548
:106A40000A00E11713B51700EF90507B2A84630604
:106A50000A00D2852685EF90207101C42685EFF0CB
:106A60000FF6B2502285225492540259F249624ADA
:106A7000D24A4561828097D7FB1F83C7E77DFD1708
:106A800093F7F70F05476377F70801114AC806CE59
:106A900022CC26CA4EC652C4328989472DC22A8AC0
:106AA000AE89368497C0FB1FE7804007AA84D14790
:106AB00039C5485509C59790FB1FE7804067F145E8
:106AC0004A8597A0FB1FE7808095C8D4AA85CD474B
:106AD0001DC5D824A147631DF70209C8382D122906
:106AE000930625015285EF90806E2A84D820936703
:106AF00047006384090093676700DCA0A287F24027
:106B00006244D2444249B249224A3E8505618280AC
:106B10000144E9BFC9473E8582809307000463EAC8
:106B2000A70097D7FB1F9387A7483325F5200A2195
:106B3000828041657D158280011122CC2A842E85B8
:106B400026CA06CEAE8497C0FB1FE78020FD0DCD80
:106B5000B7470F009387F723094563E28702814512
:106B60000A85414697A0FB1FE7804085A685608087
:106B70000A8541804081A3010100EF90F048F24076
:106B80006244D244056182804945D5BF97D7FB1F37
:106B90002383A76C82806F90D060797152CC2A8A4F
:106BA000328526D24AD04ECE56CA5AC85EC662C474
:106BB00006D622D42E8CB28A368BBA8B3E89C289F5
:106BC000C68497C0FB1FE78060F505C92A84631A55
:106BD0000A1893774B000343450085CF13632301C5
:106BE00063940B1663100914639F090885E81C5C05
:106BF0001373B3FF23026400C5EBB25022549254C6
:106C00000259F249624AD24A424BB24B224C456188
:106C100082801373D3FF13630301D9B71363430057
:106C2000230264009C484146A6851CD413058401B8
:106C30009790FB1FE780007263130C12638C0B0AA2
:106C4000485409C59790FB1FE780604EF1455E856B
:106C50009790FB1FE780A07C48D4005C59DC1C5057
:106C600091EB91659385357171459790FB1FE78096
:106C7000E03E08D008500DC17146DE859790FB1F9D
:106C8000E780406D11A81363430023026400D9F824
:106C9000005C630C0C0235D0639A0902A5E029A0C0
:106CA000005C21DC639409022254B2509254F249F0
:106CB000B24B224CCA865A860259424BD68552851F
:106CC000D24A624A45616FF08FEA05D85C5091EB79
:106CD0009165938525715D459790FB1FE78000388E
:106CE00048D0485045DD5D46CE859790FB1FE78034
:106CF00060666DB7005C11D0E39A09FC1C5491EBFF
:106D000091659385157151459790FB1FE78000357C
:106D100008D4085451D95146A6859790FB1FE780A7
:106D2000606359B71363430023026400E39C04EEDD
:106D3000E3080CF6485405EDF1454A859790FB1F92
:106D4000E780E06D48D431A8136343002302640058
:106D5000E39A04ECE3060CEEE31E09FCFDBDE31B25
:106D600009FC005CE30B04E8E39B0BEE35B797905E
:106D7000FB1FE780C03BC9B7011126CA52C406CE2B
:106D800022CC4AC84EC62A8AAE8497C0FB1FE78031
:106D9000E0D835C12A8939459790FB1FE780C04B61
:106DA0002A8431C997D9FB1F83C9892363940900B9
:106DB000834909009307000D1EA0AD473CA0930531
:106DC00069001305340019469790FB1FE78080582F
:106DD00093F714005CA493D4144844B423154401DD
:106DE000A2856244F240D2444249224A4E85B249C9
:106DF00005616FD08FA5F2406244D2444249B24946
:106E0000224A0561828001114EC652C456C206CE86
:106E100022CC26CA4AC8AA8A2E8AB28997C0FB1FEA
:106E2000E780C0CF35CDAA841305C0029790FB1F21
:106E3000E78080422A842DC517D9FB1F0349491AD0
:106E40006314090003C904009307000D1EA0E9475D
:106E50003CA0938564001305340019469790FB1FEE
:106E6000E780404FD285231554011305C4004146E5
:106E70009790FB1FE780004ECE851305C401414665
:106E80009790FB1FE780004DA2856244F240D244F8
:106E9000B249224A924A4A85424905616FD0EF9A27
:106EA000F2406244D2444249B249224A924A0561C0
:106EB000828017D5FB1F032525EC11CD411106C695
:106EC0009790FB1FE780A026B24097D7FB1F23A512
:106ED00007EA410182808280411122C406C626C28F
:106EE0004AC02E8497C0FB1FE78040C329CD00D540
:106EF00017D9FB1F0349C90EAA846314090003496B
:106F0000050041459790FB1FE78000352A8405CD99
:106F10009307000D1EA1A5473CA1DC3093856400BA
:106F20001105A30FF5FE19469790FB1FE7808042DD
:106F30009C54A285B2405CC4224492444A850249D2
:106F400041016FD08F90B2402244924402494101E6
:106F500082805D71A2C4A6C286C6AA842E8497C010
:106F6000FB1FE780A0BB0DC954251147AA874945DF
:106F7000639FE6009C5F91C3E02B97B60000938669
:106F8000E6920A86894526854080EF90E014B64057
:106F900026449644616182805145D5BF97D7FB1F37
:106FA00083C7872BFD1793F7F70F0547637AF7041D
:106FB000411126C206C622C44AC0B284894715CAF6
:106FC0002E8997C0FB1FE78060B52A84D14715C181
:106FD000630609005C2193E727005CA14146A68572
:106FE000130584019790FB1FE780C0369C481CD492
:106FF0008147B2402244924402493E854101828049
:10700000C9473E858280011122CC26CA06CE2A8439
:10701000AE8497C0FB1FE78060B019C96C00228561
:107020004486EF900011F2406244D24405618280B0
:107030005145D5BF6F80301AC1671387E7FF63934F
:10704000E50297D7FB1F83A727D591EB494582809F
:107050004945B240224492440249410182809C4306
:10706000F5D78287411122C426C24AC006C6FD1741
:107070002A892E84B284639AF50297D7FB1F83A7CF
:10708000A7D189C79C4399C3829711C5A6854A8514
:10709000EFE03FD05DFD97D7FB1F238327D197D724
:1070A000FB1FA38F97CE01456DB72E8597C0FB1FA1
:1070B000E780C0A651DD1C210D45E39C27F9228500
:1070C0002244B2400249A685924441016FC0504813
:1070D0009307000463E1A7064111C16722C426C2D9
:1070E00006C6FD172A84AE8409456380F502C547AC
:1070F0006312F4022E85EFC0504D97D7FB1F938784
:1071000027EB3324F420014506A0B24022449244E8
:10711000410182809307A0036316F4002E85EFC01F
:10712000F043E1BF9307B003E319F4FC13F5F50F47
:10713000EFC01043D9B709458280011106CE2AC697
:10714000EFE03FC7EF20404EEF10C07CEF50122918
:10715000324597D7FB1F9387E7ED130700F0BAA3DB
:10716000238207007D5797D7FB1F9387A70EB8A3ED
:1071700088A3F240954505616F70E028757126C3BC
:1071800006C722C54AC1CEDED2DCD6DADAD8DED6D0
:10719000E2D4E6D2EAD0EECEAE849397556063D1C6
:1071A000075817DAFB1F130AEA0A03450A00130BF4
:1071B000200A930BF00F9790FB1FE780E00FC16749
:1071C000FD172A84130C1009954C394D97DDFB1FD0
:1071D000938D4DE63ECC15E01395F468BA402A44F1
:1071E0009A440A49F659665AD65A465BB65B265CFB
:1071F000965C065DF64D496182801C20639A6701AA
:1072000003C93D00E2452A202286EFF06F87E1A006
:1072100003492A00639A87091C30639097032285EB
:10722000EFF06F8A2285EFC03FDD03450A0097909B
:10723000FB1FE78060082A8479BF639BA7194A2057
:107240008567A507631AF5040C4497D9FB1F93893A
:1072500069DE882115E51946850517D5FB1F13053D
:10726000E5DE9790FB1FE780E00E03C70900854726
:10727000631CF70289472380F900EFC030305DB707
:1072800003C7090085476311F70297D7FB1F2383C4
:1072900007DAEFF0AFB979B709679307C70063EF73
:1072A000A7040507636BA702E30E79F7A2854A8559
:1072B000EFC0BFD99DBF370700181307F770B3574A
:1072C000F748E5CB97D7FB1F83A7C7ACA1DF9C434B
:1072D000B1DB2285829739F5C1BFF977F917AA97F3
:1072E0002947B3C707086366F70C1767020013073F
:1072F0002753B3C7E7209C43BA978287F9779387D0
:10730000A7FCAA97F146B3C70708E3F6F6FA3907D0
:10731000E31CE5F897D7FB1F83A707A8E38407F0D2
:10732000DC43E38107F00965A2853905A5A8832917
:107330008400E38B09F603C7090097D7FB1F9387E7
:1073400067CF19EB03C7290083C619002207558FA1
:107350009AA703C7390098B394230947E396E6F444
:1073600003C7090001CB97D7FB1F238507CC03C5B3
:10737000090005B78C338A270D4798A3EF70400B9F
:10738000FDB71C448823EFF06FD869BD97D7FB1F6A
:1073900083A7C7A0E38807E89C43E38507E809655E
:1073A000A2852D05829705BF1C449C23E39E07EE12
:1073B00095BD896793871704E318F5EE97D7FB1FF0
:1073C00083A7C79DE38007E69C43A285E1FF99BDA3
:1073D0003D476394E7064A2089671387D700630611
:1073E000E50013879701631AE50097D7FB1F83A772
:1073F000A79AE38907E2DC43C9BFCD07E316F5EAA4
:10740000C16717D7FB1F035747C3FD17631FF7005B
:1074100097D7FB1F83A74798E38607E0DC43E38306
:1074200007E00965A2854D05B5BF97D7FB1F83A768
:107430002796E38907DE9C43DDB71307E003E39556
:10744000E7E63C2005476398E7127C2097DAFB1FAC
:10745000938A8A926390071083A70A006387070EB6
:1074600083C907002149683093078400BE853ECE5A
:10747000EFE09FD268B013064002814568109790F4
:10748000FB1FE780A0F33C30194693058400A30757
:10749000F1027C304818A309F1029790FB1FE780A6
:1074A00060EB5E207010CA852318F1027E244E85A1
:1074B0002313F1041E282314F1043E282315F1049C
:1074C0005C282306F104FD57A306F1042317F104F9
:1074D000EFF02FB63C309DE3DD478358040103589D
:1074E000E40074304E203EC23E28130784003EC0A4
:1074F000CA8705464E85EF80407028B083A70A00F2
:1075000081C71145EFF0FF9A97D9FB1F93894989ED
:1075100003C50900E30805D097D5FB1F83C555882F
:10752000EFE03F87E30005D0343093071003638911
:10753000F600522083C509004A873685EFE03F9860
:1075400097D7FB1F238E0784F1B997D9FB1F83C9F7
:1075500099AE09BF97D7FB1F83A7C78397D9FB1F96
:1075600083C979AD99C3DC4399E31149EDBD8145E8
:1075700001458297DDBFF91793F7F70F13077002E4
:10758000E364F7D2176702001307472CB3C7E7205D
:107590009C43BA9782877C2097CAFB1F938ACA7D37
:1075A000A9EB83A70A00A9C383C907002149683052
:1075B00093772500A5C305891307440168B0228687
:1075C000CA854E853ACEEFF0CFA63C3072479DF784
:1075D000DD478358C4010358A40174304E203EC2D5
:1075E0007E2C3EC0CA8731B797D9FB1F83C9B9A487
:1075F00075BF97C7FB1F83A7E77997D9FB1F83C97F
:1076000099A399C3DC4399E3114955B781450145D5
:107610008297DDBF13078400BA853ACEEFE0DFB76B
:10762000724769BF97C7FB1F83A74777E38C07BEE5
:10763000DC43E38907BE22858297EDB697C7FB1F1F
:1076400083A7C775E38007BE9C47E5B722868D45B3
:107650004A2065BE9305A10213051031EF50E25F89
:107660006C1013052031EF50425F72208357C10226
:107670004A2063E7C70016240357A10263F7E60018
:1076800093050002EFC0607371BE6373E6007AA0D9
:1076900063F3D7001EA45A24362412246E20014816
:1076A0008147EFC04071BDBE2286B14555B797C72F
:1076B000FB1F83A7A76EE38707B6DC479DBF228524
:1076C000EF00607B85B697C7FB1F83A7276DE38B11
:1076D00007B49C4BB9BF2285EF00F003A1B601456A
:1076E000EF00301381B697C7FB1F83A7A76AE38D0E
:1076F00007BADC43E38A07BA8145054582976DB630
:1077000097C7FB1F83A70769E38007BADC43E38DB4
:1077100007B8A2850945DDB72286930560020DBF33
:1077200093F7150089CF97C7FB1F83A7276789C7E2
:10773000DC4399C30145829713C5140045B493F700
:10774000250091CF97C7FB1F83A7C76491C7DC4370
:1077500081C781450545829713C5240041B413F5BF
:107760004500E30D05A697C7FB1F83A7276117D424
:10777000FB1F1304248C89CF85475CA097C7FB1F90
:1077800083A7476191C7DC4381C78145054582973F
:1077900048446C10EF80D0736810EFF02F9297D7A9
:1077A000FB1F83D7078381CF130600643386C7028C
:1077B000914517D5FB1F0345E5A9EFC03FAF13C5A2
:1077C000440029BC011122CC2A84554506CE26CA84
:1077D000EFF0AFB4AA8413054002EFF00FB42AC64D
:1077E00013055002EFF06FB3AA8622856244324639
:1077F000F240B3359000D24405616FC0E063397147
:1078000022DC06DE0D472E84631AE500BA25962594
:10781000F2212830CE21EFE0BFE899A8096793064E
:10782000D700AA87631BD504BC21B9C317C4FB1FAB
:10783000130484540C408DCDDC87BC31194691056E
:107840004808A309F1009790FB1FE780A0B09307B9
:1078500000F03ED61C40231801002313010202D47D
:10786000882370008145EFE0DFFC0545EFF06FE411
:107870000545F2506254216182809306E700E309D6
:10788000D5FE930637016319D500A82175D10147AC
:1078900081460146814541B76507E30BE5FC314769
:1078A0006319E50017C5FB1F0345F578EFE09FEA74
:1078B000C1B7130760026319E50017C5FB1F034535
:1078C0009577EFE0FFED6DB741677D170145E392D6
:1078D000E7FAD831C947E31DF7F8F625D2250A247F
:1078E000AE25EFC0005D854711C55D45EFF0EFA205
:1078F000B337A0004C202A2030007C84EF70906ABF
:107900003C84BDF79305A10013051031EF50E2341C
:107910006C0013052031EF5042343C851A24637308
:10792000F7001EA43C863A2463F3E7003EA41E241D
:107930003A246373F7003EA42A20EF40A1137A246F
:10794000562432240E242A2001488147EFC0804467
:1079500005B741114AC006C622C426C217D9FB1F6B
:107960001309498F034779009307F00F6302F70665
:10797000AA8439CD682551059790FB1FE780C08DFB
:107980002A8439C59307000D1EA1D9473CA1DE20EA
:107990005EA1FC207CA1FC307CB19C241CA5DC34C5
:1079A0005CB5F02470A515C28C48510508C89790A5
:1079B000FB1FE780209AA285224403457900B2404C
:1079C0009244024941016FC04FE823280500E5B702
:1079D000B24022449244024941018280C1679386A9
:1079E000E7FF2A87639DD50097C7FB1F83A7C7388A
:1079F0008DC39C230D45639FE7006FC0E038FD17E2
:107A000049456399F50097C7FB1F83A7E736F5F74C
:107A1000828049458280397122DC06DE26DA4AD826
:107A20004ED652D456D25AD0182185472A84630B99
:107A3000F7001025930695009305E1010545EFE059
:107A4000CFDA0DED8147014514201147638FE6021F
:107A500017C7FB1F0327873518338D466307D702E7
:107A60008DC705C711ED0145F2506254D2544259F9
:107A7000B259225A925A025B216182801C21E9B7D5
:107A800085466311D7048D8BF9DF083093052400F8
:107A90002EC6EFE06FF008B017C9FB1F130949317C
:107AA00083270900AA8981449DC3B24517CAFB1FD9
:107AB000130A4A30130BF00F83470A0063EBF400FC
:107AC000814481A08946E310D7FA858B75BF0545AF
:107AD00061BF83270900939A4400D6979823630CCB
:107AE00067059833631937051946138527002EC695
:107AF0009790FB1FE7808097B24515CD832409003E
:107B0000D69418209147C1E8E30FF7F483240900C5
:107B1000B9D883460A0081471306F00FE385F6F4CF
:107B200003C8040013850401630BC800850793F79D
:107B3000F70FAA84E5B7850493F4F40FB5BF98A0B6
:107B40001C301385240019469CB09790FB1FE780DA
:107B50006080082491659385F57105059780FB1F6A
:107B6000E780C04F05C1182091476314F702C8C4CD
:107B70001024930594000505A30FC5FE9780FB1FF5
:107B8000E780407D1C24A1F708207D1513351500E2
:107B9000E1BD88C4F1BF6311F706C8441C2405C1C8
:107BA0001021630DF604182091476317F706C844A7
:107BB00019C59780FB1FE780805723A6040008247F
:107BC00091659385E57105059780FB1FE780004966
:107BD00005C118209147631AF704C8C410249305FF
:107BE00094000505A30FC5FE9780FB1FE7808076F4
:107BF00008243335A0008DBD88444DB7930594000B
:107C000005059790FB1FE78060868547E31DF5F823
:107C10005545EFE09FF09DBF884455D19780FB1FED
:107C2000E780E05023A4040059BF88C445BF3971E0
:107C300022DC4AD84ED652D406DE26DA56D25AD0A4
:107C40005ECE2A84130925000831CA8517CAFB1F96
:107C5000130ACA15EFE04FD408B083270A000D4776
:107C6000AA899C336391E70217CAFB1F130A4A14BF
:107C700083270A00814497CAFB1F938AAA13639340
:107C8000071005452DA0EDD3144C70389305E10085
:107C90000545EFE08FB5AA841DC903270A00854674
:107CA0001C2118336310D7028D8BDDFF0145F25084
:107CB0006254D2544259B259225A925A025BF24B40
:107CC000216182808946858BE310D7FAF9BF1C2099
:107CD00011476385E7002D47E39AE7FC97CAFB1F2E
:107CE000938A0A0D83A70A00014A97CBFB1F938B47
:107CF0006B0CCDDF03C70B00B3470A0863E4E70052
:107D0000A5F46DB703A50A00131B4A001C205A9561
:107D100018216310F7021C31639D37011946CA858B
:107D200009059780FB1FE780607401C583A40A00E2
:107D3000DA94050AC1B783A9840059A80C4C1385AD
:107D400019009780FB1FE780607285476317F5086D
:107D50005545EFE09FDC4DC191BF1C201147638565
:107D6000E7002D47639DE700C8C470380505A30FE1
:107D7000C5FE0C4C9780FB1FE780C05DB5A888C48A
:107D8000EDB7850403C70A00B3C7040863F8E70624
:107D900003250A00139B44001C205A951821E31266
:107DA000F7FE1C31E39F37FD1946CA850905978008
:107DB000FB1FE780A06B71D583240A001C201147AC
:107DC000DA946385E7002D47E397E7F683A9C400BB
:107DD0007C3803C60900E303F6F64E859780FB1F47
:107DE000E780E034683891659385E57105059780F3
:107DF000FB1FE780A02635F1E39504E803C70A00DE
:107E000083240A0081479306F00FE3FCE7E68C2009
:107E1000138604016387D5008507B284B3C70708BA
:107E2000EDB7E38004E61C20CA85138524009CA0DE
:107E30001C3019469CB09780FB1FE780A051683822
:107E400091659385F57105059780FB1FE7800021FB
:107E5000E30905E218209147631DF700C8C4703894
:107E60000505A30FC5FE0C4C9780FB1FE780804ED5
:107E700009BD88C4EDB701114AC806CE22CC26CA76
:107E800017C9FB1F1309093D034779009307F00F3A
:107E9000630DF706AA8435C961459780FB1FE7800B
:107EA000A03B2A843DC19307000D1EA1D5473CA1EC
:107EB000BC30938584002EC63CB1DE205EA1FC2040
:107EC0007CA1E830EFE04FADB24568B0194613052C
:107ED00084009780FB1FE780E047FC24A2850345D0
:107EE00079007CA49E281EA8BC283CA8BC383CB8BD
:107EF000DC285CA8DC385CB8FC287CA86244F24032
:107F0000D244424905616FC04F94F2406244D2446A
:107F1000424905618280411126C206C622C497C427
:107F2000FB1F93842433F8309307F00F6309F702A3
:107F30002A8415C519459780FB1FE780E031AA8583
:107F400019CD9307000D1EA1DD473CA15E20224400
:107F5000B2405EA1E830924441016FC00F8FB24041
:107F60002244924441018280011126CA97C4FB1F1A
:107F7000938404E49C4006CE22CC4AC84EC652C428
:107F80009DC32A89AE89131A4500014488406314B1
:107F90004403638C09049780FB1FE780401997C74F
:107FA000FB1F23A707E0F2406244D2444249B24992
:107FB000224A05618280B3078500884709C99780F6
:107FC000FB1FE780C0169C40A29723A407009C409B
:107FD000A297C84709C99780FB1FE78040159C40BE
:107FE000A29723A60700410455B755DD2286814597
:107FF0009780FB1FE780803C944081477D5613F7B4
:10800000F70FE37227FB13974700369710A38507F6
:10801000FDB7797152CC17CAFB1F130A2AD98327DF
:108020000A0006D622D426D24AD04ECE56CA5AC804
:108030005EC6E9C72A8997CAFB1F938AAAD78144DB
:1080400019ED97C6FB1F83A6A6D691CA03C60A00E0
:1080500081479305F00F13F7F70F6369C702139574
:10806000340021059780FB1FE780001F2A8415E953
:1080700021459780FB1FE780201E2A8435C1C567F4
:108080009387073D1CC123220400A9A01397470032
:10809000369718236305B700850493F4F40F85071A
:1080A0005DBF930700FD1CA18547A30025013CA1EE
:1080B00024B1F1D81309850023222501814917CB6A
:1080C000FB1F130BEBCE930BF00F83C70A0063F378
:1080D000F900A1E083270A00A2858823EFB0FFF60C
:1080E00003C50A008145493503250A009780FB1F17
:1080F000E780E00397C7FB1F23AA07CAB2502254A8
:1081000092540259F249624AD24A424BB24B4561FB
:10811000828083250B0093974900BE959C21638341
:1081200077032300F9009C3113052900FD14A300F7
:10813000F9001946890593F4F40F9780FB1FE78037
:1081400060212109850993F9F90F41B797C7FB1FF2
:1081500083A7C7C5A9C7411122C406C62A8415E151
:108160000945EFE09F9B2A8601C9854517C5FB1F7E
:108170000345450EEFC08F930545EFF0AFE42A8429
:1081800011C9854517C5FB1F0345C50CEFC06FBB63
:1081900022854135B2402244054541018280014596
:1081A000828089679386B7006315D5009C45882334
:1081B00071BF9386C7006317D5009C458546882309
:1081C00019C9FDB793861704E302D5FE93872704E8
:1081D0008146E304F5FE36858280011106CE22CC6D
:1081E00026CA4AC84EC652C456C261C13C312A8909
:1081F0008DC3444199CC5945EFE03F92814997CADC
:10820000FB1F938AAABA131A45608347390063EBB0
:10821000F900F2406244D2444249B249224A924AA9
:10822000056182808387840263C8470783A70A00A9
:10823000A5C72685EFF02FFE25C18824510597801C
:10824000FB1FE78060012A8421C99307000D1EA14E
:10825000B5473CA19C201946938524003CB18387F7
:10826000840215057CA19C30A30FF5FE9780FB1FAF
:10827000E780400E902450A415C61305440108C899
:10828000938594009780FB1FE780C00C83A70A00AA
:10829000A2858823EFB07FDB85099384940293F94C
:1082A000F90FA5B723280400D5B797C7FB1F83A7ED
:1082B000E7AFA5D3B93B6244F240D2444249B24948
:1082C000224A924A014505616FF0CFCF797106D6F7
:1082D00022D426D24AD04ECE52CC56CA5AC85EC6F6
:1082E00055CD3C312A898DC744419DC05945EFE0A9
:1082F000DF828904814997CAFB1F938A2AAB130B3B
:1083000000FDC14B131A45608347390063EDF90046
:10831000B250225492540259F249624AD24A424B14
:10832000B24B456182808387D40063C4470783A72B
:108330000A00A5C351459780FB1FE780E0F12A841E
:1083400029C923006501A30005002301750183C726
:10835000E4FF1946A6853CB18387D40015055CB5BA
:1083600083C7F4FFA30FF5FE9780FB1FE78080FE15
:10837000FC20938574001305C4003CB41946978013
:10838000FB1FE78020FD83A70A00A2858823EFB0AA
:10839000DFCB850993F9F90FC104BDB797C7FB1F60
:1083A00083A7C7A0B5D7B5312254B2509254025911
:1083B000F249624AD24A424BB24B014545616FF0E5
:1083C0006FC0797106D622D426D24AD04ECE52CC76
:1083D00056CA5AC85EC662C466C2630C05223C31E6
:1083E0002A8985CB404115C45945EFE00FF30904B4
:1083F000814917CAFB1F130A6A9B914B354C175BC7
:108400000200130BAB4E931A45608347390063EFAC
:10841000F900B250225492540259F249624AD24AA7
:10842000424BB24B224C924C456182808307A400A0
:1084300063CA571583270A0063860714834CE4FF39
:1084400093F70C01CDC793870CFF93F7F70F636980
:10845000FC00B3C767219C43DA978287230F04FE91
:108460001305E4FFEFF0AFFC630E05108347E4FF54
:1084700063EFFB1005476398E70A51459780FB1FA0
:10848000E78080DDAA84630F050E930700FD1CA121
:10849000C147A30005003CA18347E4FF1946A2851C
:1084A0003CB18307A40015055CB58347F4FFA30F17
:1084B000F5FE9780FB1FE780E0E97C2419469305D1
:1084C000F400BCB41385C4009780FB1FE78080E8EC
:1084D00065A08547230FF4FEA30A040051B789471E
:1084E000230FF4FEB5BF8D47E5BF9147D5BF93F786
:1084F0008C0099C3AD47EDB713F71C0093F74C0000
:1085000011C799C39547F9B7A147D9BF13F72C00F5
:1085100011C799C3A5477DBF9947D9B799C3A94743
:10852000C1B79D4775BF483851059780FB1FE7804D
:10853000A0D2AA8421C99307000D1EA1B5473CA172
:108540008347E4FF1946A2853CB18307A4001505C3
:108550007CA18347F4FFA30FF5FE9780FB1FE78004
:1085600060DF5038D0A419C61385440188C883251C
:10857000640199BF23A8040083270A00A6858823E5
:10858000EFB0BFAC850993F9F90F7104BDBD483850
:10859000130505029780FB1FE78000CCAA847DD1DC
:1085A0009307000D1EA1C9473CA18347E4FF93FC3C
:1085B0000C061946B3E797013CB18347F4FFA28547
:1085C0001505A30FF5FE9780FB1FE780A0D87C2040
:1085D00019469305F400BCB47C3013853401DCA447
:1085E0001C24DCB41C34FCA48307A400FCB45E246B
:1085F0009EA87C24BCA89780FB1FE780A0D550389C
:1086000090BC09C613850402C8CC95B723AE0400FC
:10861000A5B797B7FB1F83A76779E38C07DEEFF059
:108620005F9F2254B25092540259F249624AD24A90
:10863000424BB24B224C924C014545616FF08F98F2
:1086400017B7FB1F0327877605CB1823AA870D458D
:108650006315F7024111854517C5FB1F034585BF0B
:1086600006C6EFB01FEE13050003EFF09F9AB2406D
:10867000014541016FF00F954945828079714AD0DB
:1086800017B9FB1F130989728327090006D622D464
:1086900026D2CDEB17C4FB1F1304C4BB5820C94717
:1086A000298B51CB9165AA849385D571114597800B
:1086B000FB1FE780A09A2320A900CD472DCD78305D
:1086C0009307F00F6314F7009C207CB01146A68539
:1086D0009780FB1FE78000C8930531011305F04127
:1086E000EF20F22697C7FB1F9387C794A023034769
:1086F00031013334800011C3090413051002EFE087
:10870000CFC11376F50F0589E14715C5154532C66A
:10871000EFE0AFC0BC20E8841945230AF100EFE088
:10872000CFBF3246AC30E8867C0838085408228532
:10873000EFB04070AA87B2502254925402593E853D
:1087400045618280C547C5BF1971A2DCA6DA86DE05
:10875000CAD897C4FB1F9384E4AFDC204944A18BA3
:10876000B9CF97B7FB1F83A767644144A9EB2A8958
:10877000EFE05F8C9C2455446373F50497B4FB1FB2
:108780009384845F9C4045449DEB91659385C571BE
:1087900029459780FB1FE780608C88C04D4405C148
:1087A0002946CA859780FB1FE780C0BA130560027F
:1087B000EFE0AFB61374F50F058909E96144F6508F
:1087C00022856654D65446590961828013060003F7
:1087D000814588009780FB1FE78040BE4145EFE060
:1087E000CFB32316A1043D45EFE02FB32319A10415
:1087F0003545EFE08FB2231CA1043945EFE0EFB11E
:10880000231FA1042145EFE04FB12312A1061D450E
:10881000EFE0AFB09C402315A106136424009C3305
:10882000F1C72D45EFE06FAF2310A1043145EFE014
:10883000CFAE2313A1041305C002EFE00FAE231740
:10884000A1041305B002EFE04FAD231AA1041305F4
:108850009002EFE08FAC231DA1041305A002EFE00E
:10886000CFAB2310A10613058002EFE00FAB23135B
:10887000A10613057002EFE04FAA9C402316A10643
:10888000A83393854700EFD09F8D2AD69305F10337
:108890001305F041EF20B20B97B7FB1F9387877941
:1088A000AC230347F1033256B335B00011C3890539
:1088B0009440FC002287A8223EC8930721053EC6AB
:1088C000BC083EC49307E1053EC2DC103EC09308DD
:1088D000A106130861049C009106EFB020562A847B
:1088E000E30F05EC0D45EFE0CFDCD1BD2545EFE012
:1088F000CFA22310A10429451DBF97C7FB1F83C723
:10890000A795A18B17B5FB1F1305C54991E3014539
:108910006FD0AFE197B7FB1F238E0748FD5717C7EE
:10892000FB1FA30CF79297B7FB1F23A3074897B72A
:10893000FB1F23AD074697B7FB1F9387A771170748
:1089400000001307478698C31707000013072789FD
:10895000D8C3170700001307A79798C71707000089
:10896000130767A6D8C717F7FFFF1307C7FE98CBF3
:1089700097B7FB1F9387074317F7FFFF13074706B8
:1089800098C317F7FFFF1307C7E7D8C382804111C9
:1089900022C426C206C617B4FB1F1304A441AA842E
:1089A00008208545EFF04FDC97C7FB1F83C7C78AB8
:1089B000A98BBDC717B5FB1F1305C56904A0EFD070
:1089C0002FD697B4FB1F9384A43E9C4099C74D4576
:1089D000B2402244924441018280082019E10145BD
:1089E000C5BF91659385B57112059770FB1FE78030
:1089F000E06688C069DD1020814512069780FB1F64
:108A0000E780C09B142090408147FD5513F7F70F76
:108A1000E377D7FC1397470032970CA38507FDB780
:108A2000014597B7FB1F23870738EFD06FCF45BFAE
:108A300017B5FB1F0325853411CD411106C697706C
:108A4000FB1FE780C06EB24097B7FB1F23A8073219
:108A500041018280828001111305700306CEEFE090
:108A6000CF8B2AC613058003EFE02F8B2AC4130592
:108A70009003EFE08F8A2246B245F240AA86054570
:108A800005616FB0603A5D711305D00386C6A2C45C
:108A9000A6C2CAC0EFE06F882A841305C003EFE0C6
:108AA000CF87AA841305E003EFE02F872A891305F7
:108AB000F003EFE08F868A871377F50F9376F90F2F
:108AC00013F6F40F9375F40F0545EFB02038B64058
:108AD00026449644064961618280011122CC06CE6B
:108AE00026CA0D472E846317E504B831E947CA2129
:108AF00097B4FB1F938404546315F700FE2063872B
:108B0000A70497A0FB1FE7806001722011C172A526
:108B10003A2416244E202830EFD09FB85A20FE2049
:108B20006314F700FD57FEA00545F2406244D244AD
:108B30000561828009674D07AA87631CE500BC2197
:108B400031476385E7004547E390E7FEEFD00FC567
:108B5000E1BF31476319E50017B5FB1F0345D56F2A
:108B6000EFD05FBFD1B7130760026319E50017B5F7
:108B7000FB1F0345756EEFD0BFC27DB741677D1700
:108B80000145E394E7FAD831C947E310F7FACC215D
:108B90002A20300023140100EF60D03B71B7197117
:108BA000A2DC17B4FB1F1304641D1C4086DEA6DA8A
:108BB000CAD8CED6D2D4D6D2DAD00545638A070C2D
:108BC0009305F1051305F041EF2062589305F10577
:108BD0001305F041EF20A25797B7FB1F93878745F6
:108BE000BC230347F105B337F00011C389071840D0
:108BF000BEC6283393054700EFD06FD61840AAC4ED
:108C00000D452C23AEC2EFD05FF1AAC01145EFD0C5
:108C1000DFF0832A04002ADE654503C7AA0003CBE0
:108C2000BA003ADCEFD07FEF2A846945EFD0FFEE3F
:108C3000AA847145EFD07FEE2A896D45EFD0FFED14
:108C4000AA897545EFD07FED2A8A7945EFD0FFECF0
:108C50002648B6476257F256064696451375F50FF5
:108C6000137AFA0F93F9F90F1379F90F93F4F40FBC
:108C70002ACC1314446002D002CE52CA4EC84AC64F
:108C800026C422C25AC093884A000545EFB0A014FA
:108C9000F6506654D6544659B659265A965A065B2B
:108CA00009618280411122C44AC006C626C217B992
:108CB000FB1F1309B911834709001307E00F2E8426
:108CC0006382E7041307F00F6385E702114597708D
:108CD000FB1FE7806058AA8509CD930700FD1CA102
:108CE00089473CA1854700B13CB103450900EFB07D
:108CF000CFB5F9572300F900B2402244924402490B
:108D000041018280AA8411459770FB1FE780C054FF
:108D1000AA857DD1930700FD1CA1894700B13CA124
:108D200024B12244B2409244024917B5FB1F0345C7
:108D3000E50941016FB06FB179714AD017B9FB1FD6
:108D40001309C9038327090022D406D626D24ECEA2
:108D500052CC4544C5EB97B4FB1F9384A44FDC2051
:108D60004944958BC5C32E8A916597B7FB1F238F06
:108D7000A704AA899385757131459770FB1FE78019
:108D8000E02D2320A9004D4435CD23003501A3005B
:108D900005002946D28509059770FB1FE780805B97
:108DA0000327090091463C2363E7F606CD4691CFA1
:108DB0000546F546638BC7000946C9466387C70069
:108DC0000D46C1466383C700D54634A393057100A1
:108DD0001305F041EF20A2379C83C5E317B7FB1FB3
:108DE000034767258D47631AF708EFD00FC52C009E
:108DF000EF70100E2800EFD07FAC4545EFD0FFD1CB
:108E000025E50144B2502285225492540259F24978
:108E1000624A45618280ED1793F7F70F9546054446
:108E2000E3E2F6FE975602009386C6AFB3C7D7209B
:108E30009C43B697828789473CA319A0230107006A
:108E40006545EFD09FCD9307F007E301F5F80327C1
:108E500009003C2393E707043CA38DBF8547E9BF86
:108E60009947D9BF9147C9BF130600643306C502AD
:108E700088209145EFB08FC369B715332A8451D14B
:108E8000EFF01FBB41B7011126CA97B4FB1F9384B3
:108E9000E4EE9C4022CC06CE4AC84944A1C79C239C
:108EA0000D446391A70417B9FB1F1309A93A0345A1
:108EB00009008945EFB0EFE803450900914597B7F0
:108EC000FB1F239307F0EFB0CFE79C40014781469B
:108ED00080B31306F100854785450145DC87EFA087
:108EE00070742A84F24022856244D244424905616A
:108EF0008280011106CE22CC26CA4AC84EC68547BA
:108F0000631EF50617B4FB1F130404EC1E20B1CB3F
:108F100017B7FB1F0347471229E71307B003636E18
:108F2000F70297B4FB1F9384E43288208945EFB0A1
:108F30004FE112209307006488203306F60289452A
:108F4000EFB0CFB697B7FB1F239007E8F24062441B
:108F5000D2444249B24905618280938747FC1EA0F2
:108F6000F5B797B7FB1F83A767E1EDD36244F240E3
:108F7000D2444249B2498823056131B797B9FB1FF2
:108F80009389C9DF83A70900F1D317B9FB1F130920
:108F9000692C83474900918BD5DB89476311F5061E
:108FA0002D45AE849770FB1FE780002B2A8459DD86
:108FB000930700FD1CA1E547A30005003CA1BC30C0
:108FC00015051946230FF5FEDC2093855400A30FE9
:108FD000F5FE9770FB1FE780E037034559009307C4
:108FE000F00F6315F50083A709008823A28562446A
:108FF000F240D2444249B24905616FB00F85034542
:1090000009008945EFB0EFD36244F240D2444249AF
:10901000B24997B7FB1F239907DA05616FF05FA18B
:1090200097B7FB1F83C74723958B89CF97B7FB1F44
:1090300083A7C7D891CB854717B7FB1FA307F7D8DE
:109040006FF07FA1494582804145828097B7FB1F21
:10905000A38D07D6854501456FA0905D97B7FB1F8F
:1090600083C7871F958B81CB854717B7FB1F230EBF
:10907000F7D46FF05FA14945828097B7FB1F238625
:1090800007D4814505456FA0B05C97B7FB1F83C728
:10909000A71C958B638B0712011122CC06CE26CA22
:1090A0004AC84EC69307C01C328463FAC7000945FC
:1090B000F2406244D2444249B2490561828097B786
:1090C000FB1F83A7A7CB6384071097B7FB1F93876A
:1090D000F7CFB68994231307E00F639AE60E88A3AF
:1090E0001305860033450508ADC991659385657103
:1090F0009770FB1FE78080F6AA8455D917B9FB1F2C
:10910000130949CC0325090009C59770FB1FE780A7
:1091100000021385840088C022868145232099009F
:109120009770FB1FE7808029832709002286CE8560
:1091300088439770FB1FE780E02183270900A28600
:10914000F240C2A36244D2444249B2499843054620
:109150008D45054505616FA0704C916593855571EE
:109160009770FB1FE78080EFAA8431D117B9FB1FEE
:10917000130909C50325090009C59770FB1FE7807E
:1091800000FB1385840088C0228681452320990036
:109190009770FB1FE7808022832709002286CE85F7
:1091A00088439770FB1FE780E01A83270900A28697
:1091B000F240C2A36244D2444249B24998430546B0
:1091C0008D45054505616FA0B045494582804945FB
:1091D000C5B59307C01C63FCA700094582800945FB
:1091E000F2406244D2444249B24905618280011191
:1091F00022CC06CE26CA4AC84EC62A8425C1AE89CC
:109200009165210593856571334505089770FB1FAE
:10921000E780C0E4AA8461D517B9FB1F130989BA96
:109220000325090009C59770FB1FE78040F01385EF
:10923000840088C022868145232099009770FB1FF7
:10924000E780C017832709002286CE858843977060
:10925000FB1FE780201083270900C2A397B7FB1FDD
:1092600083A7C7B185CF97B7FB1F83C7E7FE958B51
:1092700085CB97B7FB1F83A7E7B491CF9843D6233D
:109280006244F240D2444249B24905468D45054503
:1092900005616FA0B03801478146DDB7014589B748
:1092A00049453DBF9307C01C63FCA7000945828068
:1092B0000945F2406244D2444249B2490561828084
:1092C000011122CC06CE26CA4AC84EC62A8425C120
:1092D000AE899165210593855571334505089770D1
:1092E000FB1FE780A0D7AA8461D517B9FB1F13091C
:1092F00029AD0325090009C59770FB1FE78020E30E
:109300001385840088C022868145232099009770A8
:10931000FB1FE780A00A832709002286CE858843A9
:109320009770FB1FE780000383270900C2A397B74C
:10933000FB1F83A7A7A485CF97B7FB1F83C7C7F1E0
:10934000958B85CB97B7FB1F83A787A791CF9843B2
:10935000D6236244F240D2444249B24905468D4583
:10936000054505616FA0D02B01478146DDB701455A
:1093700089B749453DBF9307C01C63F4A700094561
:109380008280797122D406D626D24AD04ECE2A8443
:109390002DC1AE8991652105938575713345050809
:1093A0009770FB1FE78080CBAA840945A9C817B92D
:1093B000FB1F1309A9A00325090009C59770FB1F0E
:1093C000E780E0D61385840088C02286814523206B
:1093D00099009770FB1FE78060FE832709002286B3
:1093E000CE8588439770FB1FE780C0F6832709006E
:1093F000C2A397B7FB1F83A7679889EB0145B250BB
:10940000225492540259F2494561828097B7FB1F5A
:1094100083C787E4958B4945FDD36C001305D03095
:10942000EF30B203B24793F7070FE9DB97B7FB1FA3
:1094300083A7C7989443D2238D450545EFA0101FFD
:109440007DBF97B7FB1F83A7E79789CFD2238C43B4
:10945000411106C69770FB1FE780C0EFB24001457F
:10946000410182800945828097B7FB1F83A78795BA
:1094700085C717B7FB1F0327A794894719CF522326
:109480000C43411106C69770FB1FE780A0ECB24069
:1094900081473E854101828089473E85828097B71A
:1094A000FB1F83A7279285C717B7FB1F03270791C9
:1094B000894719CF52230C43411106C69770FB1FF1
:1094C000E78040E9B24081473E854101828089477B
:1094D0003E858280797126D206D622D44AD04ECEDD
:1094E00097B4FB1F938404B58D4783C9240063FAA6
:1094F000A7000945B250225492540259F2494561DD
:10950000828098202A844145E316F7FE9307F4FFF2
:1095100093F7F70F854663E8F60A2E89B1ED994572
:109520002800EFC07FA2A0A0914517B5FB1F0345FF
:1095300065D2EFB00F812800EFD04FB855E9930501
:1095400071001305F041EF1092409C83D1EB8D47E1
:109550006318F4084545EFD04FDC59C13776180041
:10956000130606A03306C502914517B5FB1F034538
:1095700065CEEFA01FF5ADA0194681452800977074
:10958000FB1FE780A0E319462C004A859770FB1F5C
:10959000E780C0ED39FD19469305F00F280097705C
:1095A000FB1FE780A0E119462C004A859770FB1F3E
:1095B000E780C0EB1DFD1946CA8528009770FB1F88
:1095C000E78040D98DB7630FE400914517B5FB1FC5
:1095D000034545C897B7FB1F238F07A4EFA07FF66D
:1095E000014509BFC8442C00EF70800EA0A00DDD1E
:1095F0002381340101B797B7FB1F83C7E7C5918B60
:109600008DC3411117A5FB1F1305057B06C6EFC0CF
:109610001F93B240FD5717B7FB1F2310F7A241015C
:10962000828001456FC0BF91FD5717A7FB1F230F15
:10963000F778F95717A7FB1FA30AF77897A7FB1F1F
:10964000A385077897A7FB1F2381077897A7FB1FA0
:10965000239C077697A7FB1F23A6077697A7FB1FD8
:1096600023A0077697A7FB1F23AA077497B7FB1FB2
:109670009387879F170700001307E72098C31707F2
:10968000000013074787D8C317F7FFFF1307675179
:1096900098C717F7FFFF1307473CD8C717F7FFFF17
:1096A0001307A73E98CB97F7FFFF9387474317A76A
:1096B000FB1F2323F7708280411126C297A4FB1F52
:1096C0009384C46B9C4006C622C495CB2A840D4566
:1096D0009770FB1FE78040B8AA8519C9930700FD62
:1096E0001CA18D4700B13CA19C408823EFA0FF95B1
:1096F00019C42244B240924441016FF06FB3B240AA
:10970000224492444101828079714AD017A9FB1FFB
:109710001309C9668327090006D622D426D24ECE65
:109720006383070E98338547AA8497B9FB1F9389F3
:1097300069906301F70483C749008DE70D45977071
:10974000FB1FE78060B1AA8501CD930700FD1CA136
:10975000914704B13CA1832709008823EFA0FF8E25
:10976000EFF00FAD0545B250225492540259F24920
:109770004561828097A7FB1F83A7C76489CB944369
:10978000D2239305E1000545EFC03F8611ED014569
:10979000EFD0AFB82A8621C6894517B5FB1F034510
:1097A00065ABEFA0BFB025A81C21858BEDD3054587
:1097B000EFD0AFB69307B0032A8463F1A7045D66C8
:1097C00013060670894517B5FB1F0345A5A81304AA
:1097D00044FCEFA01FCF97A7FB1F2397875E83272B
:1097E0000900094798B383C7490091C797B7FB1F82
:1097F0002384078485BF2685C135ADB793070064F0
:109800003306F50249BF0145B9BF411122C42A847C
:109810000D4506C69770FB1FE78000A40DC1930796
:1098200000FD1CA1CD4700B13CA12244B240AA8555
:1098300017A5FB1F0345855941016FA01F81B24049
:10984000224441018280411122C42A840D4506C66A
:109850009770FB1FE78040A00DC1930700FD1CA17E
:10986000ED4700B13CA12244B240AA8517A5FB1FD9
:109870000345C55541016FA04FFDB240224441014F
:1098800082805A210111896606CE22CC26CA13860F
:109890006600AA876316C7009C4701458C2371A800
:1098A000138606046365E60413865603636FE600B9
:1098B00013869600630BC7081386A600630DC712B4
:1098C000A1066309D7060145A5A8F9769386A6FCEB
:1098D0003697A94633470708E3E7E6FE97460200B6
:1098E0009386C6053347D7201843369702871386D9
:1098F00016056307C71893862605E316D7FC1C4593
:10990000802397A7FB1F83C7474C2285639D0716BB
:109910000D459770FB1FE7802094AA850DC1930722
:1099200000FD1CA1F14700B13CA117A5FB1F034599
:10993000E54991A29C4705458C23EFF0AFB605455C
:10994000F2406244D2440561828017A7FB1F0327BF
:10995000E742014575D79C47882359E985471CB3E1
:109960000545EFA02042E1BF1C4597A4FB1F93844F
:10997000F4451307E00F80239C20638BE702130755
:10998000F00F6384E70211459770FB1FE780C08CDE
:10999000AA8501CD930700FD1CA1894700B13CA118
:1099A000A30105008820EFA04FEAF9579CA041BF12
:1099B00097A4FB1F9384843C9C400145D1D305E8C8
:1099C00005447D454085EFD04F956886130500021C
:1099D000EFD0AF949C40C8851307B10080B37400EA
:1099E0001306A10085450545EFA0C04389BF228528
:1099F000EFF09FCCA9B79C476244F240D244882341
:109A000005616FF07FD01C4509458C233DB71C458F
:109A100088232DE56C001305D030EF300224B247C7
:109A2000414793F7070FE38CE7F09305B100130567
:109A30006031EF30822288858545EFA0603F01B715
:109A40001C45802397A7FB1F83C7373822859DE7D6
:109A50000D459770FB1FE7802080AA85E30105EE86
:109A6000930700FD1CA1D14700B13CA197A7FB1FA4
:109A700083A7C7308823EFA04FDDD1B57933C1B5B7
:109A80001C45882319C1C1335DBD85450545EFA03F
:109A9000203C75B5411122C417A4FB1F0344C47BAD
:109AA00006C6158809CC17A5FB1F1305E55BEFC09B
:109AB0006FC84D44B2402285224441018280014555
:109AC000EFC04FC7C5BF9821937625009377D70F76
:109AD00099C29367270093F6F707131745606354FD
:109AE000070093E607081378850093F7760F630461
:109AF000080093E786009376050299CE93E7070264
:109B00009CA1635707001C2293E7C7001CA2828018
:109B10001375A5026DF9828093F7F7FD9CA1E344CC
:109B200007FE9377A502E5F37DF11C22CD9BF9BFDB
:109B30002D45631C0710011126CA4AC84EC606CE21
:109B400022CC9821BE8989472E89B684631EF704EA
:109B5000DC413284983394232207558F8D66938796
:109B600046A01316576063C9C7029386F69F63DD4C
:109B7000C602F5779387F75F3E978D47C845334711
:109B8000070863E7E702974602009386E6DD33475E
:109B9000D7201C43B6978287938766AA630EF60880
:109BA000938686B8630FD60823900400054525A048
:109BB0009770FB1FE780A083334605083356360BAA
:109BC00092A08325C9001DA01E2109479AA01CA0B0
:109BD000A1831CB00145F2406244D2444249B249DB
:109BE0000561828099479EA01946AA8522859760C3
:109BF000FB1FE7802076F9BF85479EA01C211CA093
:109C0000D1BF05C9A1479EA01E211CA01E21A18372
:109C10001CB03E213CA03E21A1833CB05E215CA053
:109C20005E21A1835CB07E217CA07E21A1837CB0DB
:109C300055B72390040079BF85479EA0DC459C233F
:109C40007DBFE1479EA06146ADBF8280797122D47D
:109C50004AD006D626D24ECE52CC56CA3A89982140
:109C600089472E84631DF7025C40B684B28503C821
:109C7000170094238D6722083368D800938627A0A5
:109C800013185860630BD8102A8A63CC0601938698
:109C900007A0630BD802938717A06300F80A8547D3
:109CA00011A8138737A0630FE80A138767AA8D47A7
:109CB000E317E8FEB250225492540259F249624A24
:109CC000D24A3E8545618280484432C69760FB1F78
:109CD000E780E0719D4733450508E36D25FD97AAB0
:109CE000FB1F938AEA0F83C70A00B3099900B245A4
:109CF00063D43701B5477DBF48442686B3C90908F8
:109D00004A959760FB1FE780E06403C60A00484459
:109D100081450506330636414E959760FB1FE78067
:109D2000E06997A7FB1F83A7E70B99E3814759B722
:109D30009C438145E5DF528525A0AD47E31C09F62C
:109D4000E39AE4FA1C321822A207D98F58441EA3C2
:109D500097A7FB1F83A70709F1DB9C438545F9D72C
:109D60008297E9B717A7FB1F034737078D4739D3FA
:109D7000AD47E31109F49947E39EF4F648441946C8
:109D80009760FB1FE780005D97A7FB1F83A78705F0
:109D9000D1DF9C43C1DF8D4579BF17A7FB1F034768
:109DA00047F3218B8D4719D7AD47E31509F0854758
:109DB000E392F4F4182293070008E3EDE4EE5C4428
:109DC00098A3ADB7411122C4094497A7FB1FA383F1
:109DD00087F097A7FB1FA38E87EE97A7FB1F238A09
:109DE00087EE97A7FB1F23AF07FE97A7FB1F2380D4
:109DF00007FE97A7FB1F238507FE97A7FB1F23904E
:109E000007FE97A7FB1FA38A07FCA14719468145B8
:109E100017A5FB1F130505FC06C617A7FB1FA30903
:109E2000F7EA9760FB1FE780605997A7FB1F238124
:109E300087EAB707A00017A7FB1F1307E7E8938778
:109E400007051CC3B707E8035CC397A7FB1F238B59
:109E500087E685476146814517A5FB1F1305053534
:109E600017A7FB1FA30FF7E497A7FB1F238B87E41C
:109E700097A7FB1FA38687E497A7FB1F238A07F4F6
:109E80009760FB1FE780805397A7FB1F238A87E219
:109E900097A7FB1FA38D07F297A7FB1F938787DC6C
:109EA000B2402244170700001307C7C898C317071A
:109EB00000001307E7D9D8C323A40700410182801B
:109EC000797122D426D206D64AD04ECE52CCA147A2
:109ED0002E84B28463EBA700174702001307C7A9BB
:109EE0003345E5201C41BA97828793071008630425
:109EF000F51C63ECA70093072004630EF516930787
:109F000000086303F518094591A093072008E31C96
:109F1000F5FE8547639BF50208229377250095E7B8
:109F200097A7FB1F83C767EB1387F7FF97A5FB1F57
:109F30009385C514120792072E97A1075047BE9527
:109F400085AA9307800F63FBB7006145B250225486
:109F500092540259F249624A4561828017AAFB1F56
:109F6000130A4AD783470A0017A9FB1F13090911CF
:109F70009207CA97C84709C99760FB1FE780201B53
:109F800097A7FB1F238E07E4130614001376F60F22
:109F9000916593850571328583490A0032C69760C1
:109FA000FB1FE780A00B83470A009209CA9992071A
:109FB00023A6A900CA97C84749D932468145976068
:109FC000FB1FE780A03F83470A002286A6859207F1
:109FD0003E990325C9009760FB1FE780A03797A72C
:109FE000FB1F238F87DE014595B78947E39FF5F473
:109FF0001E2217A7FB1F2314F7DEF5B78547E3964C
:10A00000F5F41C2217A7FB1FA309F7DCE9BF99474A
:10A01000E39DF5F21946A68517A5FB1F130585DB01
:10A020009760FB1FE78000337DBFA147E39FF5F0FA
:10A030002146A68517A5FB1F130505C9D5B785477A
:10A04000E395F5F01C2217A7FB1FA30CF7C661BF11
:10A05000E147E39CF5EE6146A68517A5FB1F1305B6
:10A06000E5147DBF8547E392F5EE1C2217A7FB1F81
:10A07000A30FF7D48DBF8547E399F5EC1C2217A7F2
:10A08000FB1F2308F7C485B78547E390F5EC97A736
:10A09000FB1F83C727C41387F7FF97A5FB1F938573
:10A0A000E5FD12072E97920750478820A107BE951D
:10A0B000EFF07FA10DBF8547E399F5E897A7FB1F58
:10A0C00083C7C7D1C9BFAA8721472E85636DF70013
:10A0D000174702001307878CB3C7E7209C43411141
:10A0E00006C6BA97828713072004638BE70889475F
:10A0F0003E85828017A7FB1F0347C7BD120797A79E
:10A10000FB1F9387A7F7BA97CC47894785C117A646
:10A11000FB1F0346E6CC9760FB1FE780A02331A01E
:10A1200097A7FB1F83D7A7CB9EA18147B2403E854F
:10A130004101828097A7FB1F83C737CA1CA1F5B7CF
:10A14000194697A5FB1F9385E5C8F1B7214697A54A
:10A15000FB1F938565B7EF90BFDBC1BF97A7FB1FC0
:10A1600083C737B6E1BF614697A5FB1F93850504FA
:10A170005DB797A7FB1F83C797C5C9B789477DB749
:10A1800097A7FB1F83C7E7B49CA1814795B76300DE
:10A19000053A97A7FB1F938787C39823631907384E
:10A1A000054798A397A7FB1F938747ED894698A774
:10A1B00017A7FB1F231907EC17A7FB1F130787B36C
:10A1C00094A397A6FB1F9386A6B6D8C7D4C37D5782
:10A1D000630CE53413771500854529C717A6FB1FC7
:10A1E000231B06EA094797A6FB1F9386A6B317A66B
:10A1F000FB1F130636AE98ABD4CBD0CF854617A63F
:10A20000FB1F2309E6AC2380E70217A7FB1F1307F8
:10A21000E7B0D8D394AF2384D70217A7FB1F23142A
:10A2200007E88D451377250025C3139745003E9712
:10A2300097A6FB1F938606AF094654C317A8FB1FBA
:10A24000130838A9854610A314A723260701231550
:10A250000700138715003347070817A8FB1F230FB4
:10A26000E8B612073E9710A314A717A6FB1F130604
:10A27000A6AA97A6FB1F938686B6890550C3231509
:10A28000070054C7B3C505081377450025C31397C6
:10A2900045003E9797A6FB1F9386C6A8094654C360
:10A2A00017A8FB1F1308E8A2854610A314A72326AE
:10A2B000070123150700138715003347070817A860
:10A2C000FB1F230CE8B012073E9710A314A717A694
:10A2D000FB1F130626A497A6FB1F938616B08905BD
:10A2E00050C32315070054C7B3C50508137785006D
:10A2F00021CF139745003E9717A6FB1F130686A292
:10A3000050C30546894610A717A6FB1F1306569C87
:10A3100014A32315070050C71387150033470708F8
:10A3200012073E9714A397A6FB1F9386669E54C3FD
:10A33000A14614A797A6FB1F9386C6A989052315D6
:10A34000070054C7B3C505081377050121CF13973C
:10A3500045003E9797A6FB1F9386C69C094654C3AB
:10A3600017A8FB1F1308C896854610A314A723152A
:10A370000700232607011387150033470708120734
:10A380003E9710A314A717A6FB1F1306269897A69F
:10A39000FB1F93866693890550C32315070054C796
:10A3A000B3C505081377050221CF139745003E97E3
:10A3B00097A6FB1F93860697094654C317A8FB1F51
:10A3C00013084890854610A314A7231507002326D9
:10A3D0000701138715003347070812073E9710A39C
:10A3E00014A717A6FB1F1306E69197A6FB1F9386DB
:10A3F000568D890550C32315070054C7B3C50508FA
:10A400001377050421CF139745003E9797A6FB1FAE
:10A4100093864691094654C317A8FB1F1308688A00
:10A42000854610A314A723150700232607011387C9
:10A4300015003347070812073E9710A314A717A665
:10A44000FB1F1306668C97A6FB1F938666988905EB
:10A4500050C32315070054C7B3C505081377050873
:10A4600021CF139745003E9717A6FB1F1306868B37
:10A4700050C35146894610A717A6FB1F13065684E2
:10A4800014A32315070050C7138715003347070887
:10A4900012073E9714A397A6FB1F9386668654C3A4
:10A4A000854614A797A6FB1F938646D089052315DA
:10A4B000070054C7B3C505081375051039C91397AC
:10A4C00045003E9797A6FB1F9386C68554C3094651
:10A4D00085461795FB1F1305A57E10A314A723150A
:10A4E000070048C713871500334707081207BA97B4
:10A4F00017A7FB1F1307C780D8C317A7FB1F130796
:10A50000178D890590A394A723950700D8C7B3C5D5
:10A5100005089796FB1F9386E674414617A5FB1F17
:10A520001305C5B56F3000421305300345B9014529
:10A5300082800111FD1522CC06CE328426CA3E86C9
:10A540004AC813F8F50FAD4763E8070B3A89173788
:10A5500002001307E7463348E82083270800B68443
:10A56000BA9782878545EFB05FBA01E5EFF08FD2E9
:10A570000145F2406244D2444249056182808945E6
:10A58000EFB0BFB87DF52285EFE06FC0D5B791453C
:10A5900032C6EFB09FB7324669FDCA852685EFB057
:10A5A0007FADEFF02FCFEFF00F85EF60A079C9B747
:10A5B000A14532C6EFB07FB5324645FDCA85268536
:10A5C000EFB05FAB2285EFE08FBCEFE00FB3EF6041
:10A5D000407579BFB14532C6EFB03FB3324651F94D
:10A5E000CA852685EFB01FA92285EFE04FBAEFE0BC
:10A5F000CFB0EF60007375B70945A5BF79714ECE36
:10A60000AE896C0022D426D24AD006D62A89B284DA
:10A61000EF00306E2A840DE1CE854A85EFB00F8EB3
:10A620002A8419E93245268797B6FFFF9386860C60
:10A630002D468145EF100006B250228522549254D7
:10A640000259F24945618280397126DAAE844C00A4
:10A6500022DC4AD84ED652D406DEAA893289368AFE
:10A66000EF0030692A8421E9A685630D09009E2048
:10A670002C007C84BE207C85930720307C86930749
:10A6800080025C874E85EFB08F842A840DE55946A1
:10A69000A6851305A100230421019760FB1FE78015
:10A6A00060CB1245528797B6FFFF9386C6FF2546BB
:10A6B0002C00EF00307EF25022856254D254425971
:10A6C000B259225A21618280797126D2AE846C00FF
:10A6D00022D44AD04ECE06D6AA893289EF007061C4
:10A6E0002A840DE1A6854E85EFB00F832A8419E9EF
:10A6F00032454A8797B6FFFF938686013546A68581
:10A70000EF005079B2502285225492540259F249F6
:10A71000456182807547AA876365B7021147014585
:10A720006378B702ED1593F5F50F61476361B702E2
:10A73000973602009386C62BB3C5D520984136972D
:10A74000028793F5F50713072005638AE5000145A5
:10A750008280C84782808843828088478280C8433D
:10A7600082809307F00F630FF506011126CAAA84B1
:10A770001305000222CC4AC84EC652C456C206CEA9
:10A780002E8AB28AB6893A899760FB1FE780C0ACEF
:10A790002A844D450DC8930700FB1CA0A30054015B
:10A7A000231144012302340113058400614663052B
:10A7B0000902CA859760FB1FE780C0B9A28526857C
:10A7C000EF90BF880145F2406244D2444249B24909
:10A7D000224A924A0561828081459760FB1FE7808B
:10A7E000E0BDE9BF09458280011122CC06CE2A8452
:10A7F0004C86D0869780FB1FE780403205C15425E8
:10A80000214797A7FB1F9387E7A4639DE600E823F2
:10A8100078009306E0070146A285A137F240624422
:10A8200005618280C83378009306E0070146A2855F
:10A83000EDB7930700643306F6026F907FBC15C135
:10A84000411122C406C62A8408219307D00F63E66B
:10A85000A700EF90BFD8FD571CA0B2402244410191
:10A8600082808280797122D406D626D24AD04ECEFA
:10A870009E2509448DEBAE846C00AA893289EF00D5
:10A8800050472A840DE1A6854E85EFA0BFF42A84A7
:10A8900019E932454A8797B6FFFF938666F34D461E
:10A8A0008145EF00305FB250228522549254025904
:10A8B000F249456182801A219307000B6310F70269
:10A8C0005C214947639AE700183985476398E70098
:10A8D0002A2185456F30902A6D47CDBF82800111B6
:10A8E0006C846C0022CC26CA4AC806CE2A89B6845B
:10A8F0007085EF0010402A840DE12C004A85EFA0FE
:10A90000DFD32A8419E93245268797B6FFFF93865D
:10A9100086CE15462C00EF00F057F24022856244A7
:10A92000D2444249056182807971930720306C845A
:10A9300070857C862C0093078002014606D65C87D2
:10A94000EFF09FD0B25045618280C1777971850761
:10A950003EC4894726D27C86AE84930780024C0091
:10A9600022D44AD006D62A895C87EF0090382A8400
:10A970000DE12C004A85EFA05FE32A8419E9124516
:10A98000268797B6FFFF938686DF45462C00EF00AB
:10A990007050B250228522549254025945618280EF
:10A9A000B28605466FF05FCA797126D2AE846C001C
:10A9B00022D44AD04ECE06D6AA893289EF0070330F
:10A9C0002A840DE1A6854E85EFA0DFBE2A8419E911
:10A9D00032454A8797B6FFFF938686BC0D46A6850B
:10A9E000EF00504BB2502285225492540259F24942
:10A9F000456182807971930720206C8470857C8604
:10AA00002C0093078002014606D65C87EFF0DFC377
:10AA1000B25045618280011122CC26CA4AC806CEB6
:10AA20002A84AE84328936C69780FB1FE780000FE8
:10AA300015C95025A146324797A7FB1F93878781E9
:10AA4000631DD600E823CA862686A2856244F240AA
:10AA5000D244424905616FF0DFD0C833CA862686EA
:10AA6000A285EDB7F2406244D244424905450561F2
:10AA700082806FF0BFB86FF07FB86FF0FFC46FF0E7
:10AA8000BFC479714ECEAE896C0022D426D24AD092
:10AA900006D62A89B284EF00D0252A840DE1CE851E
:10AAA0004A85EFA03FC92A8419E93245268797B61F
:10AAB000FFFF9386A6C73D468145EF00B03DB250EB
:10AAC0002285225492540259F24945618280B2860D
:10AAD00001466FF07FB7011122CC2E846C0026CA8C
:10AAE00006CEAA84EF00F020DD476309F500930746
:10AAF00010101EA4A2852685EFA0DFCDF24062448F
:10AB0000D24405618280239405006FF0BFD5E5BF74
:10AB10001797FB1F03478731854763F8E702011149
:10AB200022CC2E846C0026CA06CEAA84EF00701CAC
:10AB300001E9930700101EA4A2852685EFA09FC9F6
:10AB4000F2406244D24405618280594582809797E1
:10AB5000FB1F23ADA72882809797FB1F23A6A7285A
:10AB60008280011122CC26CA06CE2A84AE84978028
:10AB7000FB1FE780A0FAA6852285EFA0AFF705E9C5
:10AB8000228564869780FB1FE78040F90DC154251C
:10AB900021479797FB1F9387E76B639FE600E823A6
:10ABA00078009306F0070146A285EFF09FBBF240C4
:10ABB0006244D24405618280C833DDB7797122D402
:10ABC0004AD0AE8706D6BA8526D24ECE7547328495
:10ABD00036896364F7042147636CF700154763887F
:10ABE000E7021947638DE708C167FD1785441DA07B
:10ABF00037061400DD1713060620B317F0287D8EE4
:10AC000049EE19677D8F25EB93F71710F1DFC167C8
:10AC1000FD1789446316F40221A813F7F70793067A
:10AC20002005E313D7FC41677D17631EE6048D44BE
:10AC30002EC6EFA0EFEFB24533049540334404082D
:10AC40003385840033450508EF30D000AA87B3C9A7
:10AC5000040821C963040900231089002254B2505A
:10AC600092540259B3053041F2493E85456117536C
:10AC7000FB1F67004359C167FD17954461BFC1675A
:10AC8000FD179D4441BF1307200D8D44E39AE7FA59
:10AC90001304C6003344040865B7C167FD178D442B
:10ACA00095BFB250225492540259F24945618280B4
:10ACB000011122CC26CA06CED0212E841307000211
:10ACC00081469945AA84DD3D2AC621C51E20502013
:10ACD000930554007C803E207C8189477C829307C9
:10ACE00080025C839750FB1FE780C0665C208A85EA
:10ACF00026857C84EFA01F972A8411C53245975082
:10AD0000FB1FE780C042F24022856244D2440561C5
:10AD100082804D44CDBF397122DC26DA4AD806DE66
:10AD200089472A84AE8436896306F600C1470945FF
:10AD30006315F60432C6A9C04C082285EF00607B7B
:10AD4000324605EDC1778507A6851305D1013ECCB6
:10AD5000230EC1009750FB1FE780C05F2C0822859F
:10AD6000813F01ED52454A8797B6FFFF9386268EB5
:10AD70001D462C08EF0010120145F2506254D254C7
:10AD8000425921618280397126DA4AD84ED63289F9
:10AD9000AE893686BA84814613071002D94522DC73
:10ADA00006DE2A8432C6EFF07FE12ACE1DCD324680
:10ADB000A685231A3101F084231B21019750FB1F24
:10ADC000E780405922854C08EFA07FAA2A8411C54C
:10ADD00072459750FB1FE7808035F2502285625400
:10ADE000D2544259B259216182804D44FDB70111BC
:10ADF00022CC06CE26CADD472A84639FF508543943
:10AE0000B1441C49B38696023287B69790431443E7
:10AE10006306D6020A20230601006C00EFA0DFA81B
:10AE20000824B165938505B8EF906FBAE5473CA05B
:10AE300097B7FFFF938707A75CC091A85623D2233B
:10AE4000E31AD6FC88470C479750FB1FE780006247
:10AE5000AA870A2089E7230601006C00C1B75C3885
:10AE60005828850793F7F70F5CB863F4E702B387B8
:10AE700097021848BA979847D623B2238E232137D2
:10AE800051F90824B165938505B8EF904FB4D944C2
:10AE900031A87C285C86D1B70A21AE846C002306D9
:10AEA0000100EFA07FA08547E39CF4F6F2406244E6
:10AEB0002685D24405618280011122CC06CE26CAA5
:10AEC000DD472A840A216398F508EFA06FC6522C4B
:10AED0003E284E286D162A96334606083307F6405C
:10AEE00052ACAA86334707080A206372B706138854
:10AEF000C6FFB388E54063D40803AE97918FB3C60D
:10AF000007081C4C0E283E97EFF0FFE709ED0824D8
:10AF1000B165938505B8EF908FABD944B1A0ED161C
:10AF2000B3C60608F9BF0A20230601006C00EFA093
:10AF3000BF970824B165938505B8EF904FA9E54701
:10AF40003CA097B7FFFF9387E7955CC0F9B78547AB
:10AF50005C866C00E9BFAE846C0023060100EFA0A4
:10AF6000BF948547E397F4FCF24062442685D244BF
:10AF700005618280397126DAAE842C0022DC4AD841
:10AF80004ED606DE2A89B289AD232A8431E54A8568
:10AF9000EFA00FBAD6206D1563C4A600B34605080E
:10AFA0009844B2208E204A85EFF0FFDD2A840DE51B
:10AFB0003146A6850808230601009750FB1FE7804D
:10AFC0006039BE2022454E8797B6FFFF93862687BD
:10AFD0005D466C00FC867D2DF25022856254D25471
:10AFE0004259B2592161828071B769B7797122D40F
:10AFF00006D626D24AD04ECE52CC56CA5AC809449A
:10B00000C1CD3289094449CAAE84BA8A2A8A368BAC
:10B01000EFA00FB21387440081477115162363DE3A
:10B02000A608850793F7F70F3107E319F9FE8A851C
:10B030005285C1212A842DE131453305A90291654C
:10B04000938515704D449750FB1FE7802001AA8916
:10B0500021C531463306C902A6859750FB1FE780FC
:10B06000602F9844D620B2208E205285EFF0BFD1B9
:10B070002A8415ED02458547568797A6FFFF9386DC
:10B08000067C5D464C005C824EC423062101A3066B
:10B09000010023076101FD2BB250228522549254F6
:10B0A0000259F249624AD24A424B456182804E853A
:10B0B0009750FB1FE780A007C5B76D44F1BF7971BA
:10B0C0004ECEAE89C16526D20147AA84894617961D
:10B0D000FB1F1306A6C2FD15054522D406D64AD08D
:10B0E000EF101001054429C92A891307300281464F
:10B0F0001146F5452685EFF07FAC2AC655440DCDA7
:10B100000357A900CE860146788411477885054704
:10B1100018A1B2472C002685A38007003247FD57AF
:10B120003CA332473CB3EF10E0712A8411C532458D
:10B130009750FB1FE780A0FFB25022852254925403
:10B140000259F24945618280411106C6EFF08FDC59
:10B1500019C5B24041011753FB1F670043FDB240C0
:10B1600041018280011106CE2AC6EFA0AF8232458E
:10B1700091459797FB1F23AB07C69797FB1F23A506
:10B1800007C69797FB1FA387A70CEF30C027F24095
:10B1900005616F20700F79714AD006D622D426D26D
:10B1A00001499397556063D807041795FB1F034522
:10B1B000750A2E899750FB1FE78000102A845DC511
:10B1C00018219307000A6310F70A85474C08DC85AD
:10B1D000EFA0CF89AA841DC59C8599C7084409C5DD
:10B1E0009750FB1FE780A0F42A208545EF30001917
:10B1F000CD47639AF406B250225492544A850259BC
:10B20000456182808347610191CF71476363F7068F
:10B210004D476378F7069386C7FE130730143357FC
:10B22000D74825C31797FB1F032707BC01C7034750
:10B2300051012DCB9C8599C7084409C59750FB1F28
:10B24000E780E0EE5247B7070001938707F07D8F54
:10B25000B7071200938707106307F70003476101E0
:10B26000ED476302F70A2285EF801FD91319F968A9
:10B2700059B7138717FE1377F70F93060002E3F30E
:10B28000E6FA858B9DCB9797FB1F83A727B6A5C7AB
:10B290002A201306B1004C0882979C85AA84ADEB46
:10B2A000D5D099B75C8699472308F1002A206C0015
:10B2B00023170100EFA02F9EB5BF9797FB1F83A711
:10B2C000A7B285CB2A201306B1004C088297AA8426
:10B2D00035D183475101E39107F02308910083475B
:10B2E00061012A206C005C8623170100EFA0AF9A51
:10B2F000E5B59944F9BF9C8599C7084409C597509D
:10B30000FB1FE780C0E22A208545EF302007A1BF60
:10B31000084459D59750FB1FE78060E151B75D7134
:10B32000A2C4A6C286C6CAC04EDE52DC56DA5AD8BD
:10B330005ED6A5472A84B2846392F50E8347450200
:10B340001A22322285072302F5029307F7FFB3077B
:10B35000F602D440B3C70708B697542503CB0700BD
:10B3600003C917008547638BF60493178900B3E779
:10B37000670141677D17638AE70A1A2863F7E70ABE
:10B3800050248507B3C7070885467EA40A20930585
:10B39000E400631BD6007C84930720307C869307EF
:10B3A000800278855C872C00EFA06FB20824B1651D
:10B3B000938505B8EF80BFE159458DA83307C702D3
:10B3C000239004008149014A930B3501B34A0708D1
:10B3D000E3FD59F9B620DC402C2813865900ED1600
:10B3E0003E965E85B3C60608EF90DFDF1DC1630B96
:10B3F0003A01C840B220B305350152959750FB1F62
:10B40000E78040F5BE203E9A9E20334A0A08850711
:10B410009EA0BE20BE99B3C909085DBF5822A947A6
:10B420006311F7028347450289CF0145B6402644A0
:10B4300096440649F259625AD25A425BB25B616144
:10B4400082803428130934014A8689451795FB1FE9
:10B450001305058EEF901FD939ED34284A868945AA
:10B460001795FB1F1305858CEF90DFD729E534284E
:10B470004A8689451795FB1F1305058BEF909FD6CC
:10B480001DE934284A8689451795FB1F13058589D0
:10B49000EF905FD50DE1DC2009476380E702ED17EF
:10B4A00093F7F70F29476368F70013079048B357DE
:10B4B000F700858B99E3054595BF834744028507CF
:10B4C0002302F402BE2075B5411122C406C62E84A3
:10B4D0009770FB1FE780405A09C93C251387170066
:10B4E0006315E40093F707F83CA5B24022444101FC
:10B4F0008280411122C406C62E849770FB1FE7800C
:10B50000A0571DC111C008C01C251307E00F5D45E1
:10B510006388E7001307F00F59456393E70001457F
:10B52000B2402244410182800945DDBF411122C45D
:10B530002A84210526C206C64AC0EFF04FB0242057
:10B54000A51493F4D40F81E858248547631DF704AC
:10B550001C483149A1E3FD57230104001CB4230218
:10B5600004021305C4002244B240924402496146D9
:10B57000814541011753FB1F670043E4B387240350
:10B580003E95084509C59750FB1FE78040BA8504E2
:10B5900093F4F40F5C280848E3E2F4FE9750FB1F95
:10B5A000E780E0B84DBF084C75F975B7411122C46A
:10B5B000416406C626C29307E4FF6301F502AA842C
:10B5C0009DE19770FB1FE780204B09E91305F4FF0D
:10B5D0009770FB1FE780404A11C106A1B240224488
:10B5E00092444101828085476392F5049770FB1F66
:10B5F000E78080482A847DD1FD571EA11C241307B3
:10B60000F00F6382E7021307E00F6389E70034203D
:10B61000083401475146A685EFF0AF942285EFF03C
:10B62000FFF0FD571CA4230504004DBF8947E39795
:10B63000F5FA8545EF40C04655F126859770FB1F0A
:10B64000E78080432A845DF951BF21C5011122CCD6
:10B6500006CE18259307F00F2A846308F7023421D9
:10B660000E21083501475D46EFF0AF8F3820E147E6
:10B670006318F7000A206C0023060100EFA0CFA298
:10B68000F9571CA42285EFF07FEAF240624405617D
:10B69000828082809307F00F6306F706011122CCA7
:10B6A00026CA2A844AC84EC652C4B689328A3A8902
:10B6B00093068500AE847946AA8517050000130518
:10B6C00005F906CEEFF0EF96A3042401230144010F
:10B6D0002322340185C01305C4006244F24042496C
:10B6E000B249224AA685D244614605611753FB1F21
:10B6F000670043C6F2406244D2444249B249224AFA
:10B700000561828082809787FB1F2385A76E8280D8
:10B71000411122C406C695472A846391F5068347E2
:10B720004502854685072302F5021E225842302233
:10B73000FD17B3C70708631ED602B3C7E7209823D7
:10B740009C330145A207D98F7A2463F0E7020A20CF
:10B7500085075EA49305C400EF903FEE0824B16511
:10B76000938505B8EF80BFA65945B24022444101F8
:10B770008280C946B387D702BA97D1B75822A94762
:10B780000545E314F7FE0345440213351500F1BFE8
:10B79000411122C406C69D472A846396F504834757
:10B7A000450285072302F5021E225842FD17B3C742
:10B7B000E72098239C33A207D98F7A25014563F0AF
:10B7C000E7020A2085075EA49305C400EFF04FCE80
:10B7D0000824B165938505B8EF807F9F5945B24035
:10B7E0002244410182805822A9470545E319F7FE0A
:10B7F0000345440213351500DDB7411122C426C2AA
:10B8000006C6B5472A84B2846394F504834745028B
:10B8100085072302F5020A21EF909FB19E201307AE
:10B82000F5FF014563C1E7027A240A209305C400AD
:10B83000BA977EA4EF905FEE0824B165938505B8B2
:10B84000EF80FF985945B2402244924441018280E2
:10B8500058229D470545E318F7FE0345440213357A
:10B860001500D5B7411122C406C6C5472A84639086
:10B87000F5061E223A22FD17B387E7020347450269
:10B8800005072302E5025842B3C707083E973C3339
:10B890003823A207D98F41677D176397E7000145D9
:10B8A000B240224441018280138717005AA57A25AD
:10B8B000E3F7E7FE9305C5000A21EF901FEF082488
:10B8C000B165938505B8EF809F905945D1BF582247
:10B8D000A9470545E316F7FC034544021335150057
:10B8E000C1B7011126CA4AC84EC656C206CE22CCDE
:10B8F00052C4BC211547AA8A2E89B289B684639E98
:10B90000E7023686CE854A85EFF09FE02A84631EE3
:10B9100005108547034599006393F910D820A9477E
:10B920006319F70C054A834629000345990001472E
:10B930006946D685EFE0FFE2F9A83547638CE70852
:10B940006361F7041D47638BE7062547638EE706AF
:10B95000A547638FF90A0544034599002687CE86DB
:10B960000146D685EFE0FFDF054A19E5CE8526853D
:10B97000EFE05FDA133A15005DD4D9476306F402AD
:10B9800059A84547638EE7045D47E393E7FCD82554
:10B9900085473686CE854A85631AF704EFF02FC5B2
:10B9A0008547054AE306F5FAF2406244D24442492B
:10B9B000B249924A5285224A056182803686CE85F6
:10B9C0004A85EFF0FFDC99B73686CE854A85EFF0E1
:10B9D0001F952DBF3686CE854A85EFF01FE23DB715
:10B9E0003686CE854A85EFF0FFE70DB7EFF0CFCC76
:10B9F00045BF268785460146D685EFE09FD6E313EF
:10BA000005F285452685EFE0FFD0133A150021BFEA
:10BA10009E20B1F3054A4A85EFF05FB171B7A547A3
:10BA2000E39CF9F29E208DFBF5BDA547E396F9F264
:10BA30009E20E39307F2054A89B79E21639F071C66
:10BA4000397126DA4ED652D406DE22DC4AD8A0213D
:10BA5000ED47AA89AE84328A6315F4021787FB1F6B
:10BA6000034747399307F00F0144631FF7049947D1
:10BA7000F2506254D2544259B259225A3E85216141
:10BA80008280F5476311F4089786FB1F83C68636CC
:10BA90001307F00F9947E38DE6FC9770FB1FE780D3
:10BAA000A0FD2A8415C1302505C29317466063D4D2
:10BAB0000700814775BFF5454E85EFE0FFD23C2476
:10BAC00093E707F83CA4F5B7D62090448C30882043
:10BAD0003800EF907FDEAA8741FDB4203800014690
:10BAE000CE851785FB1F0345E530EFE09FC7AA878A
:10BAF00041F1B24799C323000A00BC207547E39A7D
:10BB0000E7FA69F07DB79770FB1FE780E0F62A89B6
:10BB10004DD185476317F404CE2088443000EF9060
:10BB20001F83AA8731F58347290015476382E702FF
:10BB3000E51793F7F70FC14663E1F6043317F028D2
:10BB40001377574411E7639AD7028327090195C7F2
:10BB5000B0203400CA854E85EFF0BFD82300AA007C
:10BB600089BF38219147E31587F05841E30207F078
:10BB7000CE208844300002976DB70345990097871F
:10BB8000FB1F83C7376D6381A702B42038000146CD
:10BB9000CE85EFE01FBD2A8409E9AC202800EFE044
:10BBA0007FB719C123000A000144034729008D47CC
:10BBB0006318F7043C840357C90063F4E7002316B5
:10BBC000F9008355C9004E85EFE0BFF91787FB1FC9
:10BBD0000357C737ED4763F5E7028357C900DD46D2
:10BBE00063F0F6029386370063D1E602116693850F
:10BBF000470013060629B3C505084E85EF80C0151A
:10BC00004A85EFF0BF92A287A5B511669305B00FE4
:10BC100013060629B355B70ACDB799473E858280EA
:10BC2000011106CE26CA4AC822CC4EC652C49784F9
:10BC3000FB1F938424628824930780029165330557
:10BC4000F502938565701789FB1F1309691A33453F
:10BC500005089740FB1FE78060409024930780020F
:10BC600081453306F6022320A9009740FB1FE78099
:10BC7000E074832709004D459DCB0144130A8002DF
:10BC8000FD599C24636DF40217050000130525DBA4
:10BC9000EFE0FFEB1705000013054583EF90CFDBC6
:10BCA000170500001305C590EF30B0560145F2406E
:10BCB0006244D2444249B249224A05618280B307B4
:10BCC0004403032509006146814505041374F40FFC
:10BCD0003E9523103501230105002314350123056A
:10BCE00005002302050231059740FB1FE780006D28
:10BCF00049BF014582801787FB1F0347375681479D
:10BD000063E4E70001458280922193864500631435
:10BD1000A6002E8582808507B685DDB71DC5411139
:10BD200022C406C638219307D00F2A8463EBE700AC
:10BD30000E2128310147F9465D46EFE09FA2F957F1
:10BD40003EA0B24022444101828082801787FB1FBF
:10BD50000347D7508147FD5663E3E700828016A171
:10BD60002301050085071105C5BF01458280978520
:10BD7000FB1F938535F79307000285469CA1FD576D
:10BD80001787FB1F2300F7F61787FB1FA30BF7F49A
:10BD90001787FB1F2307F7F49787FB1F2392D7F41E
:10BDA0009787FB1F239607069787FB1F23A007068D
:10BDB0009787FB1F23AA07049787FB1F23A4070469
:10BDC0001786FB1F130646F19787FB1F938787F69D
:10BDD0005CC29787FB1FA38F07009787FB1F938782
:10BDE000E7E9094718A298A398AB2380E7022388C4
:10BDF000E7021787FB1F1307A7F294A7D0C794AFDA
:10BE0000D8DB1785FB1F1305A5F20D471786FB1F0F
:10BE1000130646F19786FB1F938646EE238CE702B6
:10BE2000C8C323950700D0CB239D0700CCCFD4D324
:10BE3000238407022395070223A60702239D0702F6
:10BE40001787FB1F032747FBD8DF9787FB1F9387C5
:10BE500027E2170700001307870B23A00700D8C3AA
:10BE600023A407008280411106C6EFF0DFE809C570
:10BE70002821B240410182800145E5BF411122C421
:10BE800026C24AC006C6AA842E893284EFF0BFE6D5
:10BE9000AA8711E94165CA857D15EFF0DFE5AA871C
:10BEA000454581C786A3A0A30145B24022449244E0
:10BEB00002494101828021E309483547639E060318
:10BEC000011106CE22CC182210322206598E32C61B
:10BED000B377F64085E7CC452A842EC4EFF0BFF84F
:10BEE00032460147630EC50022856244A245F240F6
:10BEF00005616FF0BFF82D473A858280130700086F
:10BF0000F24062443A850561828083C80500094891
:10BF100063910803DC4103C807009C33A207B3E721
:10BF200007010D68130828906395070189476FF092
:10BF30009FF80545828001114EC606CE22CC26CA46
:10BF40004AC89789FB1F9389D9D903C7090093076A
:10BF5000F00F630FF7022A892945AE843284974097
:10BF6000FB1FE780602FAA8505C59307100B1EA154
:10BF70002302050002A562442311250166A1F240B7
:10BF800003C50900D2444249B24905616F80EF8B75
:10BF9000F2406244D2444249B24905618280411173
:10BFA00026C2AE849785FB1F83A505E522C406C67D
:10BFB0002A84EFF05FEB098909C922852244B24047
:10BFC000A685924441016FF08F8FB2402244924483
:10BFD000054541018280411122C426C24AC006C6DD
:10BFE000AA84130445001309850B1E209DC3084431
:10BFF00009C59740FB1FE7808013228531468145A4
:10C000009740FB1FE780803B3104231A04FEE31EA8
:10C0100024FDB2402244FD579EA0024992444101B2
:10C0200082809786FB1F83C676239787FB1F83A793
:10C0300027DD01476394E600014582808E23138645
:10C04000870B6394A5003E85828005071377F70F61
:10C05000B287CDB7AA871785FB1F0325E5DA01C98B
:10C060005A216314F700084582800841CDBF8280C1
:10C07000411106C6EFF01FFE09C50845B240410157
:10C0800082800145E5BF797122D41384450026D210
:10C090004AD052CC5AC82E8A06D64ECE56CA5EC652
:10C0A00022892287014B814481468147BD45122365
:10C0B00045CAB5EE46233E23B286A697B3C7070806
:10C0C000050B3107E315BBFEADC491659385457043
:10C0D00026859740FB1FE78060F8AA8B39C90C447E
:10C0E000D1C9814A8149522033853B019740FB1FCA
:10C0F000E78040265E200844BE99B3C909089740EE
:10C10000FB1FE780C00263980A003109854A832536
:10C1100089004A84E9F9314681452285850A97409C
:10C12000FB1FE780A02963826A053109CDB7630E42
:10C13000D6000145B250225492540259F249624A43
:10C14000D24A424BB24B456182803223E313F6FE62
:10C150005223B294B297B3C40408B3C707088DB78B
:10C160008547E3E367F70545F1B723267A012314F2
:10C170009A00D5BF1309C400854A814949BFAA87DF
:10C180001785FB1F032505C811E1828018453A2752
:10C190006314F700110582800841FDB7411106C6FE
:10C1A000EFF0FFFD09C50A21B2404101828001453F
:10C1B000E5BF411106C6EFF09FFC09C52821B2403A
:10C1C000410182804145E5BF41111786FB1F1306DF
:10C1D00066C322C40042AA8606C62E8501471DCC2E
:10C1E0001C44AE271C406396D5021DC71CC301C961
:10C1F0002146930544009740FB1FE780A015228548
:10C200009740FB1FE780A0F20145B2402244410164
:10C21000828022873E84E1B71CC2D1BF0545F5B7B5
:10C2200001119786FB1F938626BE26CAAA848842E0
:10C2300022CC06CE2E8401470DCD52211C41631520
:10C24000960215C71CC39740FB1FE78040EE2C00E9
:10C250002685EFF07FF701E519C0B2471CC0F24018
:10C260006244D244056182802A873E85F1B79CC230
:10C27000D9BF0545EDB7411122C42A84090506C678
:10C28000EFE0EFDBFD573CB0B24022444101828039
:10C29000411122C4416406C626C29307E4FF63012C
:10C2A000F502AA849DE19770FB1FE780008009E9F1
:10C2B0001305F4FF9760FB1FE780207F11C106A1E3
:10C2C000B240224492444101828085476392F50442
:10C2D0009760FB1FE780607D2A847DD1FD571EA1FA
:10C2E0003C201307F00F6382E7021307E00F638916
:10C2F000E70028300147F9465146A685EFE06FC6B2
:10C300002285EFF05FF7FD573CA0230204004DBFEC
:10C310008947E397F5FA8545EF30807855F1268512
:10C320009760FB1FE78060782A845DF951BF5D71DB
:10C33000A2C4CAC086C6A6C24EDE52DC56DA5AD89D
:10C340002E84AC21F9472A896392F5049760FB1F7C
:10C35000E780A0752A8405C138219307D00F63ECCC
:10C36000E70028310147F9460146CA85EFE06FBF73
:10C370002285EFF05FF00145B64026449644064919
:10C38000F259625AD25A425B61618280832A040068
:10C39000B7070001938707F037071200B3F7FA00D9
:10C3A00013070710B28981446388E7022EC697609D
:10C3B000FB1FE780806FB245AA8419CD502109CEBA
:10C3C00093174660E3C907FA4A85EFE0EFC1DC2026
:10C3D00093E707F8DCA045B7178AFB1F130A8A907A
:10C3E00003470A009307F00F1945E307F7F8E14701
:10C3F000E3E4B7F893D71500FD17171702001307EA
:10C40000276BB3E7E72003A80700E30708F603ABB1
:10C410004700E3030BF6B3CA0A0863850A00C9475D
:10C42000E39CF5F4562010440C300820380802989C
:10C4300021F52C084A85029B1DCD183015FF3820A8
:10C44000230AA100B9472308E1006314F702E24779
:10C4500098239C33A207D98F0C084A85FC81EF9062
:10C460008F8311D914080546D9454A85EFE0AFDA24
:10C4700021B7BC84D5B734209147E38EF6EE03454F
:10C480000A0038080146CA85EFE0AFADE31605EEB5
:10C490002C202808EFE00FA819C1238009001840BC
:10C4A000B7070001938707F07D8FB70712009387C6
:10C4B0000710E302F7ECE38004EC3C2021BF4111BC
:10C4C00022C406C62E849760FB1FE780005E09C960
:10C4D0005C21138717006315E40093F707F85CA14C
:10C4E000B240224441018280397152D42E8A4ED604
:10C4F0009305E100AA89528522DC4AD856D25AD047
:10C500005ECE06DE26DA3289368BBA8BBE8A97601B
:10C51000FB1FE780005C054425C1AA8428873944B5
:10C52000EFF05FB331C90328450063070804D687DD
:10C530005E87DA864A86A6854E8502982A840DEDA6
:10C540009307E00F638AFA02982089476316F7027F
:10C55000DC4098239C33A207D98F0D6713072790DF
:10C56000639CE7008347190003460900D285A207B0
:10C570005D8E4E85EFF03F9CF25022856254D2547E
:10C580004259B259225A925A025BF24B216182807F
:10C59000797122D422214ECEAA89228556CA06D686
:10C5A00026D24AD052CC5AC85EC662C4AE8AEFF0D8
:10C5B0005FA705E52285EF908FF6594411E101440C
:10C5C000B2502285225492540259F249624AD24A08
:10C5D000424BB24B224C4561828003C7890085479C
:10C5E0006307F700EFF03F9F03D52900E9B7AA855D
:10C5F000AA8413858900EFF01FA92A8415CDFA209B
:10C600009624D044CE2003D52900E147EFF0DFED9A
:10C61000D9472A846318F50023A604002685EFF085
:10C620009F9B71BF19E1268575BFDE20268523906B
:10C63000FA00EFF05F9A69B713894400014AB94BD9
:10C64000594C3D4B8355090085CDE14763077A017D
:10C650000357C900D94711E3E1470357290083561F
:10C6600049000326890003D52900EFF0FFE72A845B
:10C670006310850323240900050A3109E3146AFDC8
:10C680002685EFF05F952DD0D947E31BF4F205BF67
:10C6900065D5835709002390FA00F9BF011170870F
:10C6A0009307E00F1306E1000147894606CEEFF03D
:10C6B000BFE3F2400561828079714AD00359850059
:10C6C00022D426D22A84AE844A859305210106D637
:10C6D0009760FB1FE780E03F79C51C252AC693F7CA
:10C6E00007029DC7A881EFF0BF98B245AA8711E95C
:10C6F000239024013945B250225492540259456185
:10C7000082802A204946829701C51E249EA0E5B753
:10C71000035924004A85EFF0DF9001ED41657D1556
:10C72000EFF03F9009E51E2425459EA0E9B72310B0
:10C730002501130745008147BD46122339EE3147D5
:10C74000B387E7029305840031462EC691073E95D4
:10C750009740FB1FE78000C0B2453146480897402C
:10C76000FB1FE78020BF52242A2041478146DD4538
:10C77000EFE0CFC42ACE09E51E2445459EA0A5BF03
:10C780000C4852249740FB1FE780C0BC2A204C086D
:10C79000EF90AFD42DD15945B9BF85073107E39E3E
:10C7A000D7F825459DB705458DB7797122D42A84E0
:10C7B0000A254AD02E899305E1004ECE06D626D210
:10C7C000B2899760FB1FE780C0302DC91C25AA8461
:10C7D00093F707028DEF18389307200511E35C20CB
:10C7E000362450440E242A200147EFF0FFCF21E1E8
:10C7F0001C38B9E32A20EF908FCAAA8759458DCFFC
:10C80000B250225492540259F249456182802887DD
:10C81000EFF01F86AA870DC52A204946A685829774
:10C820005DD91E242310F9001C3899E7D1BFD947E0
:10C83000E319F5FE238009000145D9B70545D5B7B1
:10C840003945C5B7797122D44AD04ECE52CC56CA9A
:10C8500006D626D2AA892E8AB28A36899760FB1F0D
:10C86000E780A02409440DC53C211307E00FAA84EA
:10C870005D44638FE7001307F00F5944639AE700A4
:10C8800063920A02D2854E85EF906FCD2A8421C132
:10C89000B2502285225492540259F249624AD24A35
:10C8A0004561828003550A009305E10023170100CA
:10C8B0009760FB1FE780E0212887EFF09F8FAA8514
:10C8C00005464E85EF20107D2A844DDDD1B79307B4
:10C8D000F00FE30FF9FA938624007946A68517F541
:10C8E000FFFF1305E543EFD0DFF4A38124014DB72B
:10C8F000797126D24ECE52CC56CA5AC85EC606D6DA
:10C9000022D44AD062C466C2AA8A2E8BB28B368ADF
:10C91000BA899774FB1F83A4E44EB9C0804483DCBA
:10C9200044000149035CA400631499018440F5B7F5
:10C930003E2463F757010509410433490908EDB75F
:10C94000E36BFBFE63090A000C204840D2865E863A
:10C95000EF805F896DD16384090023908901A284EF
:10C96000B25022540259F249624AD24A424BB24B67
:10C97000224C924C26859254456182809A21B621A0
:10C98000854763E3E60429C3D421011113865500CA
:10C9900022CC1775FB1F1305A5392E84894506CEB9
:10C9A00032C6EF803F84C14719C9542032462E2039
:10C9B0000A200147EFF0DFF3A94711C18147F24098
:10C9C00062443E85056182803E8582802E860A22F1
:10C9D000AE21854763E1A50219CD542241110147DB
:10C9E000150606C6EFF0DFF0A94711C18147B24036
:10C9F0003E85410182803E8582802E860A22AE21BC
:10CA0000854763E1A50219CD54224111014715065E
:10CA100006C6EFF0FFEDA94711C18147B2403E8540
:10CA2000410182803E85828039714ED6BE2183D9F4
:10CA3000050006DE22DC26DA4AD852D456D25AD075
:10CA40005ECE62CC66CA63E437152A8A05456383E5
:10CA50000912416BAE8A2314010002C60144014948
:10CA60007D1B894B054CC94C83D52A000147814663
:10CA700001464E8523130100EFF09FE7AA8471C59C
:10CA800009EC13072002930661005A8695455285EA
:10CA9000EFE0CF922A84630E050E38849C2025C7D0
:10CAA00018856301870541476394E70ABE24414620
:10CAB000130524001CA0BE24A1831CB0CC409740C9
:10CAC000FB1FE780208949043C848507B3C707081A
:10CAD0007C8463FC2707BE24638967078509B3C983
:10CAE000090859B763967707BE2409461305240041
:10CAF0001CA0BE24A1831CB0CC409740FB1FE78044
:10CB000060851104D1B722C603596100B82413050A
:10CB10002400638F7701335999032305710118A00D
:10CB2000BE244146A1831CB0CC401379F90F41BF0C
:10CB30002305810118A0BE24135929001379F90F88
:10CB4000A1831CB0CC4009464DBF3C8429459DC300
:10CB50002C005285EF803FE809CD34001546D945B9
:10CB60005285EFD05FEB11C532459730FB1FE78050
:10CB7000005C0145F2506254D2544259B259225AD3
:10CB8000925A025BF24B624CD24C21618280054585
:10CB9000D5B74545C5B71777FB1F034727298547F5
:10CBA00063F7E706011122CC26CA4AC806CE2A84BA
:10CBB000AE8432899760FB1FE78020EF11C53821D2
:10CBC0009307E00F6307F704631B090022856244A3
:10CBD000F2404249A685D24405616F900F958A20A4
:10CBE0009305E100231701009760FB1FE78060EECB
:10CBF0002887EFF00FDCAA8505462285EF209049B3
:10CC000071D5F2406244D24442490561828059455F
:10CC100082805D45FDB7411122C406C626C293F746
:10CC200005022A84328585C3EFF0AFD8AA85054670
:10CC30002285EF20304695476305F500BD47631513
:10CC4000F502214515A093F78500B6849DC3EFF04A
:10CC50004FD6AA8505462285EF20D04309C59C34CE
:10CC600081C79C2491C30145B240224492444101B2
:10CC700082809397456063D70700EFF08FD3AA8532
:10CC80000146D1BF89890D45F9FDF9BF7971AE869D
:10CC900022D42A848A229305E10106D636C69760FB
:10CCA000FB1FE78000E311C90C2522852254B24600
:10CCB000B087B25045616FF01FF6B250225405455F
:10CCC00045618280411122C406C693F705022A8479
:10CCD00032858DC3EFF0EFCDAA8505462285EF2082
:10CCE000703B1547AA876305E5003D47631DE502D4
:10CCF000A14715A893F7850099CBEFF08FCBAA85B4
:10CD0000054622852244B24041016F20B038139776
:10CD1000456063570700EFF0CFC9AA850146D5B734
:10CD2000898991E18D47B24022443E85410182804C
:10CD30007971AE8622D42A848A229305E10136C60F
:10CD400006D69760FB1FE780C0D8B24609C90C25FC
:10CD500022852254B087B25045616FF0BFF6B250C1
:10CD600022540545456182803E257971416722D470
:10CD700026D24AD04ECE06D6231701007D17AA84AC
:10CD8000328436898149638DE7009420D040138531
:10CD900017001307E10033450508EFF07FB5AA89B6
:10CDA0009420D04089451775FB1F130565F8EF8067
:10CDB0006FC315C5A2242285EFF04FBE09C57D14AF
:10CDC0002A94334404086304090023108900B250F4
:10CDD0002254925402594E85F24945618280942032
:10CDE000D04089451775FB1F130545F4EF808FBFB1
:10CDF00071F19420D04089451775FB1F130585F20A
:10CE0000EF804FBE11C9E38809FA3C87E39587FAA2
:10CE100003D4A9007D1475B7A22475B7397122DC3B
:10CE200026DA4AD84ED652D456D25AD05ECE06DE34
:10CE3000BE8B9C252A8AAE84C18BB28A36843A89FD
:10CE4000C289468B9DEF942089476383F6065685F9
:10CE5000EFF04FA005CD83280500638908022286E4
:10CE60006254F250925A5A88CE87025BB2595E875A
:10CE7000CA86F24B4259A6855285D254225A216164
:10CE800082883285EFF0CF9EAA8709ED3945F250AE
:10CE90006254D2544259B259225A925A025BF24B0E
:10CEA000216182802946A6855285829749DDC5B7D2
:10CEB000DC4003C3170098238D6722033363E3002C
:10CEC0001386479013175360E343E6F81386F78FF2
:10CED000634BE60293862780630FD70863C8E60496
:10CEE000F977938707803E93854733430308E3E050
:10CEF00067F62D45E39D0BF8DC449023CC432310CB
:10CF0000C90022851DA2F5779387F76F3E938D4761
:10CF10003343030863E0671217170200130787B350
:10CF20003343E32083270300BA97828793873780B0
:10CF3000E31FF7F02D45E39C0BF485472310F90020
:10CF4000DC4481459C231CA0AA2405053345050823
:10CF50009760FB1FE780E0B7835709004DE9910711
:10CF60002310F90011468145130514009730FB1F6B
:10CF7000E780C04441A82D45E39B0BF0DC446C00E6
:10CF800083C917009823A209B3E9E90011472310C8
:10CF9000E9009C234E851CA0DC449C331CB09760A8
:10CFA000FB1FE78000B3AA8425C13086C1659306C4
:10CFB000E100FD158329C500EFF01FDB09ED94208A
:10CFC000D04089451775FB1F130545D6EF808FA10B
:10CFD00019E1FD577C8703C7090089476310F702F1
:10CFE00083A549000946130544009730FB1FE780DD
:10CFF00060368357090089072310F9003C873CA05D
:10D00000A1833CB0014561B523173101C5BF18218B
:10D010008907BA972310F9003E251CB03E25A1834D
:10D020003CA010214C41130534009730FB1FE780D2
:10D030006032C9BF2D45E39C0BE42310D900DC44CA
:10D040009C231CA0DC449C331CB06DBFC8449730AB
:10D05000FB1FE780C039334705081D45E36977E3C7
:10D060006380EB02B386790163C6E600330777413C
:10D07000B3490708CC44231039014E86DE9551B5DB
:10D080008149CDBF2D45E3940BE0CC445285EFE0C0
:10D090009FDD89472310F90008A0218108B09DB7C2
:10D0A0002D45E3960BDE89472310F90049BF2D4536
:10D0B000E39F0BDCDC441D472310E900982318A0F4
:10D0C000983318B0BA2338A0BA23218338B0D823B4
:10D0D00058A0FA2358B0FE23A1837CA025B75D7128
:10D0E000A6C2AA842A214EDE52DC56DA5AD85ED66F
:10D0F00062D466D26AD06ECE86C6A2C4CAC0AE8AD8
:10D10000C16BEF80EFA2130CF5FF2A8A8149977D4E
:10D11000FB1F938D2D0B977CFB1F938C2CCF177BC4
:10D12000FB1F130BEBCEFD1B334D0C08DE2463F607
:10D13000F90083D70D0063CD8701AA209775FB1FE7
:10D1400093854508EF80DFAA2A841DCD59442DA878
:10D150009C449305E100B3A7F92003C917009C2361
:10D1600022093369F9004A859760FB1FE7806096C2
:10D17000AA851DE923902A0103A54D0009C5973012
:10D18000FB1FE780C0FA0544B6402285264496443A
:10D190000649F259625AD25A425BB25B225C925CF7
:10D1A000025DF24D6161828083C8440083A60C0059
:10D1B0003087AA206A8881475A87EFF03FC62A84C1
:10D1C00019C923902A0103A54D005DDD9730FB1F8F
:10D1D000E780E0F555BF83A74D0099EFAA2051479E
:10D1E00081465E86BD45EFD07F9D23A2AD0009E557
:10D1F00023902A01454449BF83D70D0003570B00F4
:10D200003E97634747013307FA407D172310EB0031
:10D2100003A54D0003560B0083A50C003E95850920
:10D220009730FB1FE780001383D70D0003570B00D7
:10D23000B3C90908BA972390FD00CDBD397126DA2C
:10D24000AA842A214ED65AD006DE22DC4AD852D4ED
:10D2500056D25ECE62CC66CA6AC82E8BEF804F8DE6
:10D26000AA89D424AE248A2478001386D400EFF04F
:10D270002FE805C5938BB9FF2A84E5190149177C6E
:10D28000FB1F130CACB8977CFB1F938C6CB833CA94
:10D29000090863497901631B09109E24294523105D
:10D2A000FB009DA8035DC10083C8440083260C00D9
:10D2B000AA205288814766876A86A285EFF01FB64A
:10D2C00019C9AE2422859306E1006A86EFF0DFA932
:10D2D0002A8461F0C9B783D70C009228E313F6FEC5
:10D2E00083250C00C8489730FB1FE780201871D9B0
:10D2F0009779FB1F938909ED83A7490095EFAA2031
:10D300004166454781467D169D45EFD03F8B1DE127
:10D310009E2445452310FB00F2506254D2544259DA
:10D32000B259225A925A025BF24B624CD24C424D95
:10D330002161828023A2A900AE24835AA400228501
:10D340009306E1006A86EFF03FA22A84E3830AF89D
:10D3500083A749001307190033470708CA9723809A
:10D36000570183A7490093DA8A0093062900BA97E8
:10D370002380570113073900110983A74900B3C659
:10D380000608334707083349090811C93087B6979B
:10D3900090A383A749002182BA9790A3DDBDB697D9
:10D3A000FD5694A383A74900BA9794A3AA20977522
:10D3B000FB1F938525E11359290023902501EF8058
:10D3C000EFEC39D9594589BF411122C406C693F7FC
:10D3D00005012A84328585C3EFE0BFDDAA850546B5
:10D3E0002285EF20204B95476305F500BD47631D5F
:10D3F000F502214515A893F7450099CBEFE07FDBB7
:10D40000AA85054622852244B24041016F2080480A
:10D4100093F7050491C7EFE0DFD9AA850146DDB790
:10D4200013C5F5FF05890605B240224441018280FB
:10D43000797122D426D252CC06D64AD04ECE56CAC4
:10D440005AC82A8AAE840144DE206364F400014590
:10D4500081A083AA04009319140013891900B3272B
:10D46000542103CB0700B3872A0188239305E100E9
:10D470002205336565019750FB1FE78080651DE13C
:10D4800023806A019C4005453E990347090098B3F3
:10D49000B250225492540259F249624AD24A424B43
:10D4A000456182800C2530875285EFF0FFF101CD78
:10D4B0009C40BE9903C7090098A39C403E9903472E
:10D4C000090098B3F1B7050433440408B5BF01114E
:10D4D000AE8722CC2A848A239305E10006CE97509A
:10D4E000FB1FE780005F09C90C2522856244308755
:10D4F000F24005616FF05FEDF24062440545056161
:10D50000828039715AD02A8B2A2126DA4AD806DE3F
:10D5100022DC4ED652D456D25ECE62CC66CAAE84DF
:10D52000EF701FE12A898346CB008355AB0003557A
:10D530008B0078001306DB00EFF08FBB6305051648
:10D54000C16A130AA9FFAA8B01449779FB1F93892B
:10D55000E98B977CFB1F938CECC6FD1A6D19334A3F
:10D560000A08035CC10083C58B0003552B0062864B
:10D57000EFF09FE56318051483484B0083A609006C
:10D5800003552B00528881471777FB1F13074788E5
:10D590006286DE85EFF09F886316051205CC83D77F
:10D5A0002C001777FB1F0357A78611076395E70029
:10D5B000A29763C427079775FB1F9385A5C0BE215B
:10D5C00003552B003354F40282A1EF802FE615C1DE
:10D5D000594505A003552B00494781465686C54548
:10D5E000EFD0CFDD23A2AC0015E183D7AB004545DA
:10D5F0009EA0F2506254D2544259B259225A925AC1
:10D60000025BF24B624CD24C216182809777FB1F08
:10D6100083D7078091072391FC0083A74C0003D791
:10D62000AB006286A29798A383A74C00130714004F
:10D6300033470708BA9703D7AB009306E1005E852E
:10D64000218398A38355AB00176CFB1F130C4C7CF4
:10D65000EFF08FF103A74C003C87130624003346FC
:10D66000060832971CA303A74C0093063400A1833D
:10D67000B3C6060836971CA3AA8B03A54C00110459
:10D680003344040803560C0083A5090022956391D6
:10D690000B029730FB1FE780E0CB83570C00A2976B
:10D6A00033C4070809F883578B0029459EA091B71A
:10D6B0009730FB1FE78000CA83570C003E94334429
:10D6C000040845B583D7AB009EA0E31604EE83574C
:10D6D0008B009EA039BF1D71A6CACAC8AA8403596F
:10D6E00085002A21A2CCCEC6D2C4D6C2DAC05EDE64
:10D6F00062DC6AD886CE66DA6ED6AE8AEF705FC319
:10D70000130BD5FF01447115138CD400976BFB1FCD
:10D71000938BCB6F176AFB1F130A8A6F177DFB1F52
:10D72000130D4DAAB3490508635D6411D424AE24DA
:10D730001307E10162864A85EFF08F9BAA8C630292
:10D7400005100359A500B0870C25AA2032C6EFF0BA
:10D75000BFC7631D050E83C8440083A60B00324675
:10D76000AA204E8881475287E685EFF02FEB79EDAE
:10D7700015C483570A0003572D0089076302F70673
:10D780009775FB1F938505A4BE21AA20B357F40209
:10D790009EA1EF802FB80DC1594539A8AA20416636
:10D7A0004D4781467D16A545EFD04FC12322AD00E0
:10D7B0001DE123902A014545F6406644D64446497A
:10D7C000B649264A964A064BF25B625CD25C425DE1
:10D7D000B25D2561828083570A0089072311FD000D
:10D7E00083570A00A29763DE670583274D0003D79E
:10D7F000AC00930D2400A29798A383274D0003D774
:10D80000AC000504334404082183A29798A30325A0
:10D810004D0003560A0083A50B00B3CD0D086E958D
:10D820009730FB1FE78000B383570A00BE9DC16796
:10D83000FD1733C40D08E309F9EE0509334909085A
:10D84000E5B5294515FC23902A01BDB76DDC0DBF58
:10D850001E21411126C206C622C44AC0444189EB9A
:10D860008947B2402244924402493E854101828068
:10D870009420D0402A8489451765FB1F1305454B2A
:10D88000EF705F9611C93C202547E51793F7F70F16
:10D89000637FF700E147F1B79420D04089451765D1
:10D8A000FB1F1305A548EF70FF9371FD55BF176966
:10D8B000FB1F1309E942835609008547DDD21A2070
:10D8C0003697C166E3CFE6F89165938525703145BB
:10D8D0009720FB1FE7808078AA84CD4759D1314635
:10D8E00081459730FB1FE78060AD1A208355090002
:10D8F00001468147B386F500B3C6060863E9E7022F
:10D9000001C62E972310E90023A004002146A2851A
:10D91000138544009730FB1FE780C0A31767FB1FE8
:10D920001307474E1C4381CF3E879C43EDBF5040B9
:10D930001395470085072A9636A6054665BF04C39A
:10D94000814705B7011106CE22CC26CA4AC809E98B
:10D950000944F24022856244D244424905618280F2
:10D960002AC6AA84280036896C845085EFF05FEEC1
:10D970002A8465F1E30F09FCBE24F9DB91659385E8
:10D98000557031459720FB1FE780406DAA8715C170
:10D99000BA249766FB1F93862647232005005AA1C9
:10D9A00098422324250101C7BA861843EDBF9CC2C3
:10D9B0004DB74D4479BF9767FB1F9387B7439823B3
:10D9C0000DE3054798A3058909CD9766FB1F93864C
:10D9D000262A414691451765FB1F1305252A6FF03E
:10D9E0007FF6014582809767FB1FA38CA72E82805C
:10D9F00041677D176315E5002E856FE02FB5411156
:10DA000006C6EFE04FAF09C5FD571EA12301050073
:10DA1000B24041018280011126CA06CE22CC4AC8FA
:10DA20008547AA846392F5042685EFE08FDF31E90C
:10DA300041699305F9FF1307E10089461766FB1F4B
:10DA40001306062E0545EFE0BFEA2A847D1905C4BA
:10DA50004C442685EFF0DFF9308722858146CA8560
:10DA6000EFF08FB02A84E5B789476396F5008545C6
:10DA7000EF20000355D9F2406244D2444249056187
:10DA80008280EFE04FD56DB7411122C406C626C291
:10DA90001764FB1F1304047C08349767FB1F23A142
:10DAA00007369767FB1F23AB07349767FB1F23A538
:10DAB000073459C59307200C3305F502916593850A
:10DAC00015709764FB1F9384A4331905334505082B
:10DAD0009720FB1FE780805810349307200C814566
:10DAE0003306F60288C019069730FB1FE780008DC9
:10DAF0009C4018348145938647007D5563EAE506CE
:10DB00009306800BB306D70201460507FD55B6976D
:10DB10009766FB1F23A4F62EBE868EA2ACB2ACA2E3
:10DB20002382060005069906E369E6FEF95696A3E8
:10DB300099463307D702BA971767FB1F232EF72A98
:10DB400017E5FFFF1305E57EEFD00F8117F5FFFF07
:10DB500013052597EF70EFF017E5FFFF13058573A9
:10DB6000EF10306BB2402244924401454101828063
:10DB7000239EA6FE36861388460B23100600232418
:10DB800006003106E31B06FF85059386860BBDB7AD
:10DB9000411106C622C42A84EFC0CFA2EFE02F9D18
:10DBA0001765FB1F032545259767FB1F238B8712EE
:10DBB000EFE0CF999767FB1F238687122244B2407C
:10DBC00017050000130565E541016F1090649397F8
:10DBD000556063DB072E79711765FB1F03456510E0
:10DBE00022D44AD006D626D24ECE2E899720FB1FAD
:10DBF000E780806C2A8441CD18219307000B6315C0
:10DC0000F70885479764FB1F93844420DC849C407D
:10DC10002315010081EFEF00C07591659385357084
:10DC20009720FB1FE780804388C031C9614681454A
:10DC30001765FB1F130505599720FB1FE780007828
:10DC40008349440089476393F90825279764FB1F9C
:10DC5000938444578AA02A20A685EF703FD4AA86D1
:10DC60009E202A201A248DEE6363F7001EA40E2442
:10DC7000EFC03FEF2285EFC01FC49C8491C74C20AA
:10DC800013058400EFD04FCC2285EF60EFB6B25081
:10DC900022549254F2491315F96802594561828061
:10DCA0006363F7001EA41E24D9459766FB1F938665
:10DCB00066510D469EA0EFC01FD68D4545DD176508
:10DCC000FB1F13052550EFD02FC86DB79387A9FF11
:10DCD00093F7F70F4947E36FF7F8170702001307A9
:10DCE00067D8B3C7E7209C43BA9782879305A10002
:10DCF0002285EFF0AFD4AA8435DDD9476394F40AC6
:10DD000085092A2093F9F90F9766FB1F9386864BA6
:10DD10004E86D945EFC03FD031DDCE854DB7930556
:10DD2000A1002285EFF03F9BF9B7835984006C0076
:10DD30004E859750FB1FE780C0D9AA842DC12A20A9
:10DD400041669306E10055477D16AD45EFC01FE7DC
:10DD50009769FB1F9389094723A2A900AA8655CD7D
:10DD6000834844000358E10030862A20A685814775
:10DD70004E87EFF0AF8AAA846312050E2A20CE8563
:10DD8000EF70FFDEE30805EE2A20D945CE862D464A
:10DD9000EFC07FC8AD45E30F05EC4E852DB72315C9
:10DDA000310185441830D147E306F7EC5C209769D0
:10DDB000FB1F938929412A202380F9003C85CE85C9
:10DDC000238299002391F900EF70EFECE30405EA58
:10DDD0002A20CE860546D945EFC0FFC3E30C05E8EF
:10DDE000854565BF835984006C004E859750FB1FA5
:10DDF000E78020CEAA8445D52A2041669306E1001B
:10DE000059477D16B545EFC07FDB9769FB1F9389A6
:10DE1000693B23A2A900AA8609E51E24C5447C8586
:10DE200051B7834844000358E1003E2430862A203D
:10DE3000A6854E87EFE09FFEAA840DE12A20CE85BD
:10DE4000EF705FD6E30805E22A20D945CE86354635
:10DE5000EFC07FBCB545E30F05E081B7D94703A507
:10DE600049006397F4009720FB1FE780402C19B509
:10DE70009720FB1FE780A02B1E247C8525B79305E8
:10DE8000A1002285EFF0AFA5BDB59305A1002285C5
:10DE9000EFF02FE78DB5130691009305A1002285C1
:10DEA000EFE0BF9089BD9305A1002285EFE0DF8000
:10DEB000AA84E31405E4A30401006DBB9305A1004B
:10DEC0002285EFE0EFEC05BD01458280F1CE011126
:10DED00056C2AE8A854526CA4EC652C406CE22CC4C
:10DEE0004AC82A8AB284B689EF10903BD1471DC533
:10DEF0001767FB1F034797F39767FB1F83C7D7F28B
:10DF0000014999E03E89BA87131749001764FB1F3E
:10DF10000324C4F03A94636DF900D547F24062449B
:10DF2000D2444249B249224A924A3E8505618280E2
:10DF300036201307040191C605091379F90F3A84B5
:10DF4000D9BFB1C89565938525C0130500029720F8
:10DF5000FB1FE780A01048C469D113060002814569
:10DF6000130909049720FB1FE780404523000400A4
:10DF700023112401231344019C341767FB1F03273B
:10DF800027EA998C1CA45C4491849180C4AF23A09F
:10DF90008900814761B7232604002300040023136E
:10DFA000440123045401E5B785473E858280AA8653
:10DFB0009765FB1F83C595E71767FB1F032707E6D8
:10DFC00081476394F5000145828032233A8519C266
:10DFD000E30CD6FE850793F7F70F4107DDB7AA8656
:10DFE0001766FB1F034696E41767FB1F032707E32B
:10DFF00081476314F600014582802E233A8581C54E
:10E000004C23E38BD5FE850793F7F70F4107D5B770
:10E01000AA869765FB1F83C545E11767FB1F03278A
:10E0200027E081476394F5000145828012233A85F9
:10E0300019C2E30CD6FE850793F7F70F4107DDB74A
:10E04000AA861768FB1F034838DE9767FB1F83A764
:10E05000E7DC01476314E80001458280B2233E8576
:10E0600009CAF2236317D600D04701C63222E3065D
:10E07000B6FE05071377F70FC107E9BF411126C2A6
:10E08000444522C406C62A8495C0C84409C59720C1
:10E09000FB1FE780C009C84809C59720FB1FE78020
:10E0A000000926859720FB1FE780600822854146EE
:10E0B00081459720FB1FE7806030FD571CB4B240BC
:10E0C0002244924441018280011122CC2A842A21D7
:10E0D00006CE2EC6EF102069324622858145EF001C
:10E0E000505822856244F24005616FF03FF905C542
:10E0F0003E21411122C406C62A8491CBDD45EF00A2
:10E10000505922852244B24041016FF03FF7B2409E
:10E110002244410182808280411122C4B14713040C
:10E12000C5FFB307F40226C29764FB1F9384040B58
:10E1300006C6A697BA276315B702C84315C1930749
:10E14000F00F6305F6001C21639CC7009720FB1F9E
:10E15000E780E0FDB1473304F402A29423A2040057
:10E16000B2402244924441018280411122C42E8453
:10E1700026C24946AA848145228506C69720FB1FF0
:10E18000E780C0238DCCD82C9767FB1F83A747C996
:10E190001207BA979A231AA0BA23FE233AA0176748
:10E1A000FB1F035727C85AA09A207AA0BA201AA4A6
:10E1B000DA203AA4FA205AA49A241EA87AA4B240DB
:10E1C00022449244410182802A869765FB1F83C5C1
:10E1D000F5C51768FB1F0328A8C49766FB1F83A615
:10E1E000E6C3014701456393E50082809C2281CF0D
:10E1F000DC4691CBDC2F9207C2976316F60093079B
:10E20000150013F5F70F05071377F70FC106E1BFE8
:10E21000130600643386C50293069500AA85170588
:10E220000000130505ED6F60AF9D411122C406C6C5
:10E230002A840835EF608FBAFD571CB4B2402244DF
:10E2400041018280011122CC4AC84EC652C456C236
:10E250005AC006CE26CA2A89AE890144176AFB1F16
:10E26000130A9ABC976AFB1F938A4ABB1D4B8347CC
:10E270000A006369F404639D09029769FB1F93898F
:10E28000F9BA176AFB1F130A6AB9930AF00F83C71A
:10E2900009006364F4061144A14422851306F00FBB
:10E2A000CA850504EFF05FE733440408E31794FEE2
:10E2B000F2406244D2444249B249224A924A024B55
:10E2C0000561828083A40A0093174400BE949C20B9
:10E2D0008DC3FE20639F270163956901AA20EF107B
:10E2E000804826854E868145EF00B0372685EFF0C1
:10E2F000FFD805041374F40F9DBF83240A009317FD
:10E300004400BE949C208DC39C34638F5701FE2033
:10E31000639C27012685EFF05FF12685D145EF004C
:10E3200050372685EFF09FD505041374F40F85B799
:10E33000C167F917630BF502411122C406C6854770
:10E340002A846399F50022852244B2408145410127
:10E350006FF05FEF89476396F5008545EF104074D5
:10E360007DD1B24022444101828082809D456FF080
:10E370007FED1765FB1F0355E5AA8280011106CECC
:10E3800068876C861767FB1F034707AA85476318D2
:10E39000F70070009305E1000545EF50B01CF24016
:10E3A00005618280A947631DF6029C319821A2076E
:10E3B000D98F1EA1BC31B821A207D98F3EA1DC3173
:10E3C000D821A207D98F5EA1FC31F821A207D98FED
:10E3D0007EA19C359825A207D98F1EA50145828074
:10E3E000054582809147631EF6009C319821A20763
:10E3F000D98F1EA1BC31B821A207D98F3EA10145FA
:10E400008280054582809387C5FF0D47B3C6070804
:10E41000636ED70031473387E7029767FB1F938707
:10E42000E7DBBA97A8A38EA30145828009458280C5
:10E43000930740203355F50A71159767FB1F239307
:10E44000A79E9767FB1F2383B79E9767FB1FA38E2B
:10E45000B79C8280956541111905938535C006C624
:10E46000334505089720FB1FE78040BF01C9B24034
:10E47000E95541011723FB1F6700E3D8B240410172
:10E4800082809767FB1FA383079A9767FB1F238FE1
:10E4900007989767FB1F238A07989767FB1FA38539
:10E4A00007989767FB1F23810798854741111767D6
:10E4B000FB1FA30AF79606C622C426C22A849767C2
:10E4C000FB1F238207969767FB1F239D079497677F
:10E4D000FB1F23A50794EF10E0311765FB1F130501
:10E4E000E5CF1306000381459767FB1F23818794BF
:10E4F0009720FB1FE78080EC1764FB1F13048491B7
:10E5000008209764FB1F938434921DC995659385F9
:10E5100045C012059720FB1FE78040B41767FB1F1B
:10E520002320A79011CD1C30102081459CA0976717
:10E53000FB1F238CC78E12069720FB1FE78000E885
:10E540009C201765FB1F034565D11764FB1F13044F
:10E55000F48D3E951375F50F956508A0938555C00C
:10E5600012059720FB1FE78060AF9764FB1F938421
:10E57000E48A88C035CD1020814512069720FB1F04
:10E58000E780C0E398401420814725077D56639BB0
:10E59000F604EF106047B1473305F50295659385A2
:10E5A00065C0334505089720FB1FE78020AB9767C0
:10E5B000FB1F23A3A7862A8401CDEF10E044314638
:10E5C0003306C502814522859720FB1FE78000DFC7
:10E5D0002244B2409244170500001305A5D541011D
:10E5E0006F102043850710A393F7F70F410745B736
:10E5F0009767FB1FA38C07829767FB1FA386078281
:10E6000049BF411126C206C622C44AC0AE849397B0
:10E61000556063DB07081769FB1F13094981034530
:10E6200009009720FB1FE78020C92A8421C91821EF
:10E63000930700096311F7041831CD476314F706F7
:10E640009756FB1F9386867E28219C221768FB1F06
:10E650000348B88F13066400814501476318E5023B
:10E6600091C19CA29C2281CB03450900854597401E
:10E67000FB1FE78060342285EF501F981395F468E4
:10E68000B240224492440249410182800E22050791
:10E690001377F70FAE9793F7F70F09068545B3D7B2
:10E6A000070B6DBF0123C1BF13F5150071D9EF0032
:10E6B000105319CD9757FB1F83C7477791CB8545DB
:10E6C0001755FB1F0345A5769740FB1FE780C02E1B
:10E6D00013C5140075B70547637EC7029C319421AA
:10E6E000A207D58F1EA16399E700BC31B821A2070C
:10E6F000D98F3EA1014582800947E39DE7FEBC31E9
:10E70000B821A207D98F3EA1DC31D821A207D98F29
:10E710005EA1CDB7054582809147631EF6009C310E
:10E720009821A207D98F1EA1BC31B821A207D98F89
:10E730003EA101458280054582809147631EF60017
:10E740009C319821A207D98F1EA1BC31B821A20704
:10E75000D98F3EA10145828005458280A14763187B
:10E76000F6029C319821A207D98F1EA1BC31B82195
:10E77000A207D98F3EA1DC31D821A207D98F5EA193
:10E78000FC31F821A207D98F7EA101458280054581
:10E79000828089476319F6009C319821A207D98F9E
:10E7A0001EA101458280054582803E2279714ECEB0
:10E7B00006D622D426D24AD01307F007AE89637159
:10E7C000F70209473AC47C86300093F5F50FEF0055
:10E7D0007078B250225492540259F24945618280B5
:10E7E0005A22D9462A89328463F7E6007E2263F4EE
:10E7F000F6006379F70023140100300093F5F90F58
:10E800004A85F1B70A2202C4EFF09F80AA8435C579
:10E81000EFF09F9B9C246369F5001146A246CE85CC
:10E820004A85EF00F06975B7340026869305F00F2E
:10E830004A85EFF0AFE975F1A2471A24DC479AA3A5
:10E840003A20BAA35A20DAA37A20FAA3DA209AA7A8
:10E85000DC4495C793F4F90F2286A6854A858297F2
:10E86000C167FD172A86E31BF5FA22459947F9454A
:10E870001CA144A1EFF0DF99A9BF094645B70146A5
:10E8800071BFA947631DF6029C319821A207D98F59
:10E890001EA1BC31B821A207D98F3EA1DC31D821FD
:10E8A000A207D98F5EA1FC31F821A207D98F7EA1E2
:10E8B0009C359825A207D98F1EA501458280054564
:10E8C00082809C211CA19C311CB1BC31B821A207C3
:10E8D000D98F3EA1828023220500D8218947630475
:10E8E000F70005458280F62101114EC606CE22CCE6
:10E8F00026CA4AC80D47AE896379D7049C4584333C
:10E900009023A033A204D18CB02322049387440027
:10E91000518C639CD7029307C4FF2A89B3C70708A9
:10E920006361F70203A58900231199002310890070
:10E93000F1559720FB1FE780008D2322A900014598
:10E9400031A02285EFF0AFE671FD0545F24062444B
:10E95000D2444249B24905618280797122D426D2DB
:10E960002E8406D64AD01C201947AA84B28563900B
:10E97000E70630202800EFF03FDA0DE92884EFF0B9
:10E980000FE30C302A890DC92E86171700001307D4
:10E99000E7D134009D452685EF00D0304A850946F1
:10E9A0008145C1214A85EFF06FED0145B2502254F7
:10E9B000925402594561828089477C803C840A8652
:10E9C0007C813C857C822685EF00D058F9BF494781
:10E9D0006395E70232202800EFF05FD861F9175500
:10E9E000FB1F1305A57F5E25E9D3183068253C0081
:10E9F000C9460146A685DD2C4DBF5147639DE70002
:10EA000032202800EFF01F9A55F10C303000268597
:10EA1000EFF0BFD959BF5947639CE7043220280063
:10EA2000EFF05F9C41F52C842685EFF06FE115C96E
:10EA3000584534851E23B697B3C707081EA3B5D71C
:10EA40005C47A5D79757FB1F83C7473EB9DF85456E
:10EA50001755FB1F0345A53D9740FB1FE780C0F5F9
:10EA6000A9B789473EC03C840C300A867C82A1BF8E
:10EA70000C30231001000A8681BF5D71A2C456DAF2
:10EA800086C6A6C2CAC04EDE52DCAA8A88312E844F
:10EA900032C6EFF0CFD4B24501ED0144B640228535
:10EAA000264496440649F259625AD25A61618280DC
:10EAB0002302050023110500834904008547AA8429
:10EAC0006399F90030202808EFF0FFC02A84054937
:10EAD0001DA09D476391F90418218D47E31FF7FAA4
:10EAE000302028080549EFF05FC52A8409E505466E
:10EAF00081452685BD262685EFF02FF388243C0826
:10EB00000147CE862286D685D522E30909F82685D7
:10EB1000EFF0CFD661B7CD47639BF900182191473D
:10EB2000E31DF7F630202808EFF0BFC645B7D547FC
:10EB3000E395F9F6034A05008947E310FAF6302019
:10EB400028080549EFF0FFD32A8455F583570102C1
:10EB5000A1EBB8841306F003DC44930607FCB3C6AC
:10EB60000608636AD600B085D94663F6C600B48647
:10EB7000D94563EDD500BAA30145EF00D03E054964
:10EB800003560102D2852685AD2CB5B7AC87BAA352
:10EB9000D2A38EA3F6A385479CA0014A0149CDB715
:10EBA000014AF9BF7971AA8522D426D22221AA84EA
:10EBB000280806D64AD0EFF01FD2F24599E53DE18C
:10EBC00085452285EFF08FFB75A0BC8415476395C2
:10EBD000E706B8858D4763F7E7046800EFF07FCE5E
:10EBE0000359E100DD4763FB27018C86B707170057
:10EBF0008507100822853EC8EF00D035BC85110975
:10EC0000638527012285EFF06FF61C8672466C0043
:10EC1000858B1106228591CFEFF03FE601C5228555
:10EC2000EFF0CFF4884449DD9710FB1FE7802050B8
:10EC300041BFEFF09FD2DDB711476389E70013872B
:10EC4000A7FF85463347070863ECE6023147F11713
:10EC5000B387E7021757FB1F13074758BA979A2342
:10EC600071D3A8233008A2850D204DFDB8849147AB
:10EC7000E318F7F4B250225492540259456182804D
:10EC80002C082285212E59FDF5B701114AC82A8981
:10EC9000314526CA4EC606CE22CCAE89B284971024
:10ECA000FB1FE780605B29C19307000A2311350130
:10ECB0001EA12A842146110595C0A6859710FB1F29
:10ECC000E7804069A2854A85EF502FB80145F240A0
:10ECD0006244D2444249B24905618280814597101D
:10ECE000FB1FE780A06DF9BF0545D5B701114AC8E4
:10ECF0002A891305000226CA4EC652C456C25AC0FB
:10ED000006CE22CCAE8A328BB6893A8ABE84971060
:10ED1000FB1FE780605421C9930720FA1CA1A300C0
:10ED200065012311550123024501A30235012A84FF
:10ED3000614621059DC0A6859710FB1FE780806175
:10ED4000A2856244F240D244B249224A924A024B1E
:10ED50004A85424905616F504FAF81459710FB1FAF
:10ED6000E780C065F1BFF2406244D2444249B249F3
:10ED7000224A924A024B056182805C45797122D415
:10ED800006D62A84AE86A5C7BA23F88513072006BF
:10ED90006396E504FA231756FB1F0356A60833575C
:10EDA000C70AB22B9E2B1377F70F918F93F7F70FAC
:10EDB00001E6890793F7F70FBA97FD17B3C7E70284
:10EDC000FC863E206E200824FC8401473C08014656
:10EDD000EFF0DFF1B250225445618280D82F97576F
:10EDE000FB1F83A7E7031207BA97FE23D1BF2EC6E6
:10EDF0001946814528089710FB1FE780205CB24622
:10EE0000C9B7797122D406D626D22A8491CD082496
:10EE10002E866E202254B2509254814701479306A9
:10EE2000000645616FF09FECB284280059469710A8
:10EE3000FB1FE780A058648499E43E2048446C009E
:10EE40007C85EFF08FB26E2008243C0001479306CA
:10EE500000060146EFF09FE9B250225492544561FA
:10EE60008280797106D6814799E53E2170867C843F
:10EE70005C4589EF3C002E866E21082501479306EC
:10EE80000006EFF0BFE6B25045618280BE237C856C
:10EE9000D5B7411122C406C61C2111472A846392AA
:10EEA000E7022E866E21082581470147CD46EFF007
:10EEB000FFE349466E202244B240154541016FF000
:10EEC000AFA513F7B70F89466317D7000146EFF0D8
:10EED0005FF35146C5B70D476398E7002244B2403F
:10EEE000014641016FF0FFF7B240224441018280A8
:10EEF0009A21B14771173307F7029757FB1F938782
:10EF0000E72DBA97D84301EBD841AAA70145D8C34A
:10EF1000BA219AA7828059458280797126D24445C8
:10EF200022D44AD006D62A842E89B1C4C84419C531
:10EF30009710FB1FE780A01F23A604009E206E20D1
:10EF400008247C85BE200147930640067C869E24CB
:10EF50004A867C879C483EC83E207C843C00EFF07B
:10EF6000FFD8A38E240123A80400B2502254925447
:10EF70000259456182802800314681459710FB1F68
:10EF8000E780C0433E206E2008247C8401473C007B
:10EF9000930640064A86EFF07FD5C1BF797152CC07
:10EFA0002A8A8A2126D206D622D44AD04ECE56CAE2
:10EFB000AE84EFE0DFFF6302051240452A89630E4D
:10EFC00004107E21639B47111E24638A0710542C72
:10EFD000975AFB1F938ACAE403A70A009206FD17FB
:10EFE00036977A23B3C707081EA46316F700930564
:10EFF0003006EFF09FD85C48B5EBC8408349150058
:10F000001C21A209B3E9F900BE2013872900631A65
:10F01000F702F9559710FB1FE780E01EC8C0239147
:10F020003401034589002686D285EFF01FC61DED09
:10F03000B250225492540259F249624AD24A45616E
:10F0400082809565938515C04E859710FB1FE780DC
:10F05000E00048C8C840231C3401F9559710FB1F35
:10F06000E780601ABE20C8C0F917BEA048482DCD61
:10F07000B220362C1E2C3308D60063C90707582C43
:10F0800083A70A0095451207BA97BE2363CA0705EE
:10F09000CC4036959710FB1FE780C02B3A2CBE2042
:10F0A000BA971A2CB3C707083EAC6398E702035718
:10F0B000290003458900300078845848D2857C8532
:10F0C0003AC6EFF09FBC11C548489710FB1FE78078
:10F0D0000006232A0400232C0400054591BF99450E
:10F0E0004A85EFE07FFED5BFA545DDBF9145CDBF89
:10F0F000BE21F9C3011126CA06CE22CC1757FB1F29
:10F10000035747D2AA846D456363F70A2E844840AB
:10F1100091459710FB1FE780000F3E20AA861CA197
:10F120003E20A1831CB11E203CA11E20A1833CB126
:10F130003220C167F917110633460608639FF402AF
:10F140002AC4314532C69710FB1FE780E010AA851C
:10F150004D45B1CD930700F93246A2469CA1F9571F
:10F16000BEA18947DCA1F2A194C51755FB1F034539
:10F1700005CCEF409FED01451DA881452685EF4058
:10F18000105311E91757FB1F130747CA1C23E5D774
:10F19000FD171CA3CDB789476302F5029D476301A4
:10F1A000F502C9476300F502FD47E30DF5FCF240A7
:10F1B0006244D244056182806D4582805145C5BF5D
:10F1C0001145F5B70945E5B7011122CC4AC83144CC
:10F1D0001309C5FF3304890226CA9754FB1F938481
:10F1E000E4FF06CE26945C40A9C31757FB1F0347D4
:10F1F000E7C30DC768843EC62A241E242C007C85E4
:10F20000EFF01FEF11C548409710FB1FE78020F279
:10F21000B1473309F902CA9423A204000545F2401C
:10F220006244D2444249056182800145CDBF797173
:10F2300026D244454ECE52CCFE20BA289759FB1F09
:10F2400083D949BE06D622D44AD056CAB3D9F90AC0
:10F250002A8A9E282DCF998F4E8463D4370133C4D8
:10F26000070889452285EFF0EF9E2A89CD4A31C5EE
:10F27000BE202AC660857C84BE2899EB9E2813098F
:10F2800025001CA19E28A1831CB16374340582282B
:10F29000BE28CC4422864A85BE959710FB1FE78086
:10F2A000600B03556A002C00EFF09FE4AA8A15C595
:10F2B0004A859710FB1FE78080E7B2502254925492
:10F2C0000259F249624A5685D24A456182808907CD
:10F2D00061B779143344040865BFBA289E203A9474
:10F2E0009A28FD17B3C70708334404089EA0A2A8B4
:10F2F0006376E400F9F3FD57DCBCC1B78145528564
:10F30000EFF0BFC15DBF797122D44ECE56CA5AC844
:10F310005EC662C406D626D24AD052CC9759FB1F8D
:10F32000938969B003CA0900975AFB1F938A0AAFF1
:10F33000054B5284930BF00F175CFB1F130CDCAED4
:10F3400083A40A0093174400BE9403C90400631DFC
:10F350006907DC44B5CBD84725CB9A2339CB9757DF
:10F36000FB1F83C7A7AC99CF2685EFF05FECAA857A
:10F3700005ED05049757FB1F83C717AB6351F402D4
:10F3800023808900B25022549254F249624AD24AF0
:10F39000424BB24B224C4A850259456182809757B5
:10F3A000FB1F238207A8F9BF2685EFF01FB701498D
:10F3B000D1BFDC3F639A7701930520062685EFF0E5
:10F3C000DF9BDC44A38E070083470C000504137405
:10F3D000F40F6363F4000144E31444F7C9BF41111F
:10F3E000154506C6EFF05FDE09C50545B24041018F
:10F3F00082801945EFF05FDD6DF91145EFF0DFDC3C
:10F400006DF51D45EFF05FDC6DF11755FB1F0345F2
:10F41000B5A169DDB24041016FF0FFEE9E210D47BD
:10F42000F117B3C707086363F706DC41411122C433
:10F4300006C626C22E84A9CF8545AA84952539CD36
:10F440002685AD2BC167F917638FF40009ED3E20C7
:10F4500099CB162019476395E6041757FB1F0357EE
:10F46000679C63FFE7029757FB1F83C7279CA28512
:10F47000268599C72244B240924441016FF05FC78C
:10F480002244B240924441016FF09FA60945828018
:10F490000945B24022449244410182805145D5BF82
:10F4A0006D45C5BF797126D252CCAA842E8A5D459E
:10F4B00089454AD04ECE56CA06D622D4B289B68ADB
:10F4C0003A89EFE03FF925C52A8401456306090022
:10F4D000D685130544000299935785003CB09307E5
:10F4E0004500230044017C85954728A07C84A30027
:10F4F000340122C69757FB1F83C747932C002685EC
:10F5000085C7EFF0FFBEAA8411C522859710FB1FA7
:10F51000E780E0C1B25022540259F249624AD24A0D
:10F520002685925445618280EFF09F9CE9BFCD44CF
:10F53000D5B7797126D24AD052CC56CA2E8906D672
:10F54000BE8522D44ECE9947B284368ABA8A6314D5
:10F55000F9062A220944EFE09FA52AC625C55C4585
:10F5600083596500BE239EA0B247154723805701EB
:10F57000BAA31757FB1F1307178B10239305160009
:10F5800093F5F50F0CA3D0A399E1854614A3514739
:10F590006317E9001547BAA0DC479A249AA7528757
:10F5A000A686CA854E85EFF0FFEF2A8432450DC44A
:10F5B000EFE0DFAC01A842867400AA89EFE01F915A
:10F5C0002A845DD1B2502285225492540259F249C4
:10F5D000624AD24A45618280F945EFE07FC3DDB7D8
:10F5E0009E211CA19E21A1831CB1BE213CA1BE2154
:10F5F000A1833CB1114582809E211CA19E21A18343
:10F600001CB1BE213CA1BE21A1833CB1DE215CA185
:10F61000DE21A1835CB1FE217CA1FE21A1837CB10E
:10F62000214582809E211CA19E21A1831CB10945F8
:10F6300082809E211CA19E21A1831CB1BE213CA1E0
:10F64000BE21A1833CB1DE215CA1DE21A1835CB19E
:10F65000FE217CA1FE21A1837CB19E251CA59E25B7
:10F66000A1831CB5294582809A218546AA8718A1C5
:10F670009A21218318B19A216319D700BA2138A1A0
:10F68000BA21218338B1114582800945631DA70045
:10F69000BA211945B8A3BA212183B8B3DA21D8A376
:10F6A000DA212183D8B382809E211CA19E21A183CF
:10F6B0001CB1BE213CA1BE21A1833CB11145828079
:10F6C000797126D24AD04ECEB2842A89AE89294693
:10F6D0008145480022D406D636849710FB1FE78068
:10F6E000E0CD64868DE43E207C829747FB1F83D764
:10F6F00067737C845C4481CFD42F1747FB1F03279B
:10F7000027729E27920636973A237C8578834A850E
:10F7100017070000130727F2540013F6F90FD54519
:10F72000EFF05FD82A8911C195E085471CA023021C
:10F730000400014681452285EFF0AFECB25022541F
:10F740009254F2494A850259456182802285EFE050
:10F75000FF92EDB7B28617070000130727F12E8638
:10F7600085456FF03FD401116887416570000148FD
:10F770009307F00F0D47970600009386A6E699457C
:10F780007D1506CEEFF0FFDAF24005618280B28788
:10F7900001482E86114797060000938626E6C94544
:10F7A0006FF03FD9B286170700001307E7E72E86F0
:10F7B000CD456FF03FCF011122CC26CA4AC84EC6B4
:10F7C00006CEAA842E891754FB1F130424A497592C
:10F7D000FB1F9389A9A61C4081C7CA8526858297ED
:10F7E0001104E31A34FFF2406244D2444249B24960
:10F7F00005618280411122C406C626C21747FB1F3D
:10F800001307C7737C2B783B1754FB1F130484A486
:10F810001CB4BA9793F7F70F1CA4A5CB1305C0032C
:10F820003385A702A56585059744FB1F9384446033
:10F830009710FB1FE780808210249307C003814547
:10F840003306F60288C09710FB1FE78020B7142408
:10F850009C4001477D566341D7022244B240924406
:10F860001306000381451755FB1F1305259A410117
:10F870001713FB1F670083B4B2A32382070023A6DC
:10F88000070205079387C703F9B7B24022449244A1
:10F8900041018280411122C426C24AC006C62A897B
:10F8A0002E84B2849730FB1FE780402709EDC167A3
:10F8B000F91751456313F9000145B24022449244BF
:10F8C00002494101828054555C2195C213F72701FA
:10F8D0004146630BC700C18B3D45E5D3BC2E0145B6
:10F8E000E3FD87FC3145D1BF1545F5D4F9B7C18B90
:10F8F0000145E1F71545D1B779714AD0416922D464
:10F9000026D24ECE52CC56CA5AC806D6AA84014434
:10F910009759FB1F93890994174AFB1F130A4A51F1
:10F92000930AC0037D19054B83C789006364F40003
:10F93000014525A83307540383270A00BA97BA2341
:10F940006316270105041374F40FF9BFC8333000A0
:10F9500093856700EFB091201946A685280097107F
:10F96000FB1FE780A0B0E31F65FDB2502254925404
:10F970000259F249624AD24A424B4561828041664D
:10F98000AA869755FB1F83C5658D1747FB1F032765
:10F99000274A81477D166394F5000145828003580C
:10F9A00027003A856306C80003480700E308D8FE2D
:10F9B000850793F7F70F1307C703F1BF411106C679
:10F9C0009730FB1FE780801509C54A29B2404101E5
:10F9D00082800145E5BF1747FB1F03276745975600
:10F9E000FB1F83C6A6871107814701456393F60075
:10F9F0008280102301C605051375F50F850793F75F
:10FA0000F70F1307C703DDB71755FB1F0345058520
:10FA100082801747FB1F1307677F81473A86B146ED
:10FA20000C4391E5B3C7C72088C301458280850791
:10FA30001107E397D7FE4D458280411106C622C4C7
:10FA40009730FB1FE780800D0DCD2A842A21854544
:10FA5000EFF07FD6485409C59700FB1FE780206D63
:10FA600022851306C00381459710FB1FE780009590
:10FA7000FD573EA0230204000145B240224441014B
:10FA800082800945DDBF411106C69730FB1FE78024
:10FA9000E00809C54825B240410182800145E5BF23
:10FAA000C167F9176305F502411122C406C62E8409
:10FAB0009730FB1FE7808006AA87014589C7DC23B2
:10FAC0007D8C33358000B24022444101828005455F
:10FAD0008280411122C406C62E849730FB1FE78026
:10FAE000E00301CD5A29AA87054563048700C2AB0C
:10FAF0000145B2402244410182800545DDBF39CD38
:10FB000001114AC8416922CC26CA4EC652C456C207
:10FB100006CEAA8401449749FB1F9389A973174A0B
:10FB2000FB1F130AEA30930AC0037D1983C78900BB
:10FB3000634BF400F2406244D2444249B249224A43
:10FB4000924A05618280B307540303250A003E955B
:10FB50003E216383270182940504C9BF82809747B1
:10FB6000FB1F83A7E72CC1661746FB1F0346066FE2
:10FB7000890701450147FD1691456313E600828020
:10FB800003D807006309D80003C8A7006315B800AD
:10FB900005051375F50F05071377F70F9387C7034F
:10FBA000E9BF9746FB1F83A6A6281746FB1F0346FF
:10FBB000E66A910601478147631FE600858393C784
:10FBC000F7FF0545B3C707086361E5023315A028B1
:10FBD0003345050882808C2299C1CE36CD8F05072A
:10FBE0001377F70F9386C603C1BF93F61700F9FE8C
:10FBF000050585831375F50FC1BF797156CAAA8AA9
:10FC00002E8526D24AD04ECE52CC5AC85EC662C489
:10FC100006D622D4AE84328B368CBA8B3E8AC28909
:10FC200046899730FB1FE78060EF3DED41657D150C
:10FC30009730FB1FE78080EE2A84554531C819466E
:10FC4000DE8513056400A30284019700FB1FE78093
:10FC500060708357010326A0230264013EA88357E6
:10FC6000410323005401232604025EA82306440115
:10FC70002317340123182401EFF0BFF20AB8232A16
:10FC800004022685232C04028145EFF0DFB20145F2
:10FC9000B250225492540259F249624AD24A424B1B
:10FCA000B24B224C456182804545DDB79746FB1F2C
:10FCB00083C6C65A1747FB1F0327871781476395DB
:10FCC000F60041657D1582800E3B1306C7036394E1
:10FCD000A5002A238280850793F7F70F3287C5B7DF
:10FCE00041661748FB1F034868579746FB1F83A6CA
:10FCF000261401477D16954811436314E800014519
:10FD00008280BE223685638EC702CC5A9DC9BC3123
:10FD1000AC2189CD938597FD93F5F50FE372B3FE82
:10FD20009387D7FA93F7D70F89EF82809385F7FDF2
:10FD300093F5F50FE3F6B8FC9387D7FA93F7D70F4F
:10FD4000E1D305071377F70F9386C6037DB74166A6
:10FD50009745FB1F83C585501747FB1F0327470D9A
:10FD600081477D1625486394F5000145828036233E
:10FD70003A85638BC600545B81CAB4329386E6FD34
:10FD800093F6F60FE374D8FE850793F7F70F130782
:10FD9000C703D1BF011122CC2A84494506CEEF60AA
:10FDA000DFD71DC12AC622859730FB1FE78000D709
:10FDB00001CD624432460E39F2401745FB1F034520
:10FDC000954905616F408FCEF240624405618280A3
:10FDD00079714ECE52CCAE892A8A930530054145C1
:10FDE00026D24AD056CA5AC806D622D4328B368971
:10FDF000BA8A9700FB1FE7806026CD4429C92A8470
:10FE000089446381090441468145231261019700B9
:10FE1000FB1FE780A05A5686CE8522859700FB1FE0
:10FE2000E78040532146630F0902CA8528009700E6
:10FE3000FB1FE7802052A28650002C005285EF3035
:10FE40003076AA8422859700FB1FE780402EB250AF
:10FE500022540259F249624AD24A424B26859254B0
:10FE600045618280814528009700FB1FE78000558F
:10FE7000D9B7411122C4405926C206C6AA8429CC4A
:10FE8000085409C59700FB1FE780602A285809C558
:10FE90009700FB1FE780A029685809C59700FB1F42
:10FEA000E780E028285C09C59700FB1FE780202831
:10FEB000685C09C59700FB1FE780602703250408DD
:10FEC00009C59700FB1FE780802622859700FB1F4E
:10FED000E780E02523AA040222448E38B2409244EF
:10FEE0001745FB1F0345353741016F408FE5411131
:10FEF00026C206C622C4AE849730FB1FE78000C22C
:10FF000031C9032345032A84630603048328C307F6
:10FF100003288307832743070327030783466300D8
:10FF200003560300834523002685EF601FC7228503
:10FF3000EFF03FF4EFF0BFE111CD2244B240924424
:10FF40001745FB1F03453531854541011733FB1F1D
:10FF5000670083A6B240224492444101828041114D
:10FF600022C426C206C6AA842E849730FB1FE780CF
:10FF7000E0BA5C5989CF9E23639B9700854763183D
:10FF8000F4002244B240924441016FF09FEEB2402F
:10FF90002244924441018280411106C622C426C2F5
:10FFA000EFF01FD429C144592A8495CCBC209DC7A9
:10FFB0009747FB1F83A747E889C7DC4399C326857A
:10FFC0008297B8309307F002631FF7002A2022447B
:10FFD000B2409244814541016FF07FF19747FB1F8A
:10FFE00083A747E5D1BFB2402244924441018280B9
:10FFF000411126C24AC006C622C4AA842E8997305F
:020000025000AC
:10000000FB1FE780A0B105CD405955C41E20639465
:10001000970A3C30130710026395E7083C20ADCFE8
:100020007C5403270408DE2B15E313F7170019CFC0
:1000300018545A23058B19CB930720023CB0B240C9
:1000400022449244024905454101828013F727006A
:1000500001CB18545A23098B01C793074002F9BFFB
:10006000918B81CB1C54DE23918B81C79307600257
:10007000F1B79747FB1F83A727DCF1D3DC43E1D31C
:100080002285829738309307F0028145E319F7FA09
:100090002685EFF0DFE565B79747FB1F83A787D974
:1000A000E9BF1307A0026398E7006304090013097E
:1000B0002003CA85F1BF631C090026859730FB1F0A
:1000C000E780C0A509C55C2193E707015CA1A6856F
:1000D0004A85EF604FBCA5B7011126CA99476C85C8
:1000E000AA842E858D4522CC4AC806CE3289368414
:1000F0007C84EFE02FB62AC61DC9AA854A850294E2
:100100002A8419E52C002685EFF04FB12A8411C509
:1001100032459700FB1FE78080012685EFF09FC7DF
:10012000F24022856244D2444249056182804D44B6
:10013000EDB7411122C42E862E84971600009386B7
:100140008675894506C626C24AC02A89EFF0DFF8BF
:100150000C20AA844A85EFF09FD9B240224402497C
:1001600026859244410182809747FB1F83A787CC55
:1001700085CB9C4395C71D71A2CC86CE98411008B3
:100180002A843AC8D84185453ACA829711C548861B
:100190002A206C00EFF0FFF9F6406644256182806A
:1001A0008280AA872E8591CFFC5781CF982398A172
:1001B000983398B1B82BB8A1982FDC4BB8B1DCC1FB
:1001C0008280414681451703FB1F6700231F974725
:1001D000FB1F83A767C681C79C4791C382870945D8
:1001E00082801747FB1F032767CB1DC75843AA8789
:1001F00005450DC703A50708411106C6930605026C
:100200001306050C93050506130505040297B24075
:100210001375F50F410182800545828082804DC9AA
:10022000357122CD2A840A2126CB52C556C35AC124
:1002300006CF4AC94EC7DEDE2E8AB28A368B973089
:10024000FB1FE780A08DAA8431C50C182285EFF032
:100250005FF53C20938B6400A9CBEF507FFD2A898A
:10026000014583C95400EF503FFAAA840C100818C6
:10027000EF10A04408542C10EF10C044DE88A68B69
:100280005AC04E88DE874A8714103010D6855285B2
:10029000EF20206CFA406A44DA444A49BA492A4AB3
:1002A0009A4A0A4BF65B0D618280EF507FF8AA896B
:1002B000014503C95400EF503FF52ACE08540C10F5
:1002C000EF10A03F2C100818EF10C03FF2484DBFB0
:1002D0008280AA8701CD1855414511CBFC5781CBAF
:1002E00028333D476375A700882F8280414582806F
:1002F0006DC5411122C406C626C2AA872E840945AF
:10030000E1C998337D761306F67F98A1B8234D4551
:1003100098B1B833B8A1D823B8B1D433DA21858ADB
:10032000A2061377F7EF558FDAA1D43333470708C6
:100330001377F7DF93D61648A606558FDAA1D43384
:10034000334707081377F7BF93D62648AA06558F79
:10035000DAA1D43333470708718F93D63648AE06F7
:10036000558FDAA1F42333470708799B858A558F87
:10037000DAA1F42333470708759B898A558FDAA1E0
:10038000F423334707086D9B918A558FDAA1F82330
:10039000DE21218BDD9BD98FDEA1EF600FF8AA84CF
:1003A0005145EF608FF7383093F4F40FAA87494531
:1003B0006360970293F7F70F63ECE700182091470B
:1003C000614563E7E7001830854763E3E7000145CF
:1003D000B24022449244410182800945828015C581
:1003E0002A87AE87094585C5411106C61433138592
:1003F0001700194694A1930527009700FB1FE7807B
:1004000060F5B240014541018280094582808280C9
:100410000DC9AA872E8709459DC5411106C6B4237B
:10042000903313052700A206D18E96A1214693850D
:1004300037009700FB1FE780E0F1B2400145410122
:1004400082800945828082801DC12A87AE87094546
:100450008DC141113E8541469305170006C69700A0
:10046000FB1FE78020EFB240014541018280094532
:1004700082808280AA87094591CB89C99C333D47F8
:1004800061456365F7009CA101458280828005C5B6
:100490002A87AE87094595C141113E8513060004A0
:1004A0009305170006C69700FB1FE780A0EAB2403D
:1004B0000145410182800945828082801D71A2CC64
:1004C0002A84084586CEA6CA2306010004213547A2
:1004D0009387F4FF93F7F70F6362F70A17D70100CA
:1004E00013070763B3C7E7209C43BA9782870C08BA
:1004F000EFF01FE0C947631CF50499475C862A208A
:100500006C00EFF01FC3F6406644D644256182803C
:100510000C08EFF03FF61DED2A209720FB1FE78027
:10052000E05FA14705C15825631CF7041747FB1F6F
:10053000032787909D4719C7184309C71008A68548
:100540000297AA875C8629A00C08EFF07FEC69D59A
:100550001C86D5F72A20EFF0FF8375B70C08EFF063
:100560001FE8F5B71C312308F1007DB70C08EFF048
:100570001FF2F1BF0C08EFF03FEDD1BF9D47BDBFAB
:100580001747FB1F0327078B75B7411122C406C607
:1005900026C24AC01821930720092A84631AF7103B
:1005A0001C3139476395E70A56210967610781477E
:1005B0006398E6089744FB1F93844488884049C1A8
:1005C0000C4403C90500631D09001C218505214653
:1005D000B9CB29059700FB1FE780C0D79C40A5C376
:1005E00049459700FB1FE78020C72A841DC1930758
:1005F00010FC1CA1A30025018C400905414689057A
:100600009700FB1FE78000D59C40A2858833EF3020
:10061000DFA388409700FB1FE78060B19747FB1F6F
:1006200023AE078029A809059700FB1FE78080D229
:10063000EF30C07605495DF19C4023802701854756
:10064000B2402244924402493E8541018280130710
:10065000E003639DE706382195476319F7024A21B5
:10066000EFF06FC29147E31CF5FC9737FB1F83A7A0
:10067000677CF1D79C47E1D772244A209305640038
:100680002244B2409244024941018287A147631B40
:10069000F7006C204A202244B240924402494101B2
:1006A0006FF01F95930600038147E31BD7F8D5B77A
:1006B0009306000A8147E315D7F8EFF03FE00844BE
:1006C0003DDD9700FB1FE78080A695BF81478DBF6A
:1006D000011122CC06CE26CA4AC8094415CDAE84E3
:1006E00009449DC92A898D456800EF50FF851C8704
:1006F00026866C0093F7F70393E707044A855C8727
:10070000EF20201C2A8409E90D466C001385340073
:100710009700FB1FE78000C4F24022856244D24468
:100720004249056182805D714EDE86C6A2C4A6C2C2
:10073000CAC052DC56DA5AD85ED6894955C93289C0
:1007400089495DC6138B45002A8AAE8A334B0B0854
:10075000930530055A859700FB1FE78020902A8477
:10076000CD4959C5EF50BFAEAA845686D28593DADB
:10077000840013DA040193FBF40F1305440093FA89
:10078000FA0F137AFA0FE1809700FB1FE780C0D2BF
:10079000A301740123015401A300440104A0EF50FC
:1007A0007FAAAA85414608089700FB1FE780C0D0B2
:1007B000214734005A86A2850808EF200037AA890D
:1007C0001DE121462C0023007901A30059012301DA
:1007D0004901A3019900130549009700FB1FE78019
:1007E000A0CDEF509FA722859700FB1FE7802094A4
:1007F000B640264496440649625AD25A425BB25BDE
:100800004E85F25961618280011126CAAA842E8523
:100810004AC806CE22CC2E899720FB1FE7800030E5
:100820004DCD40594DCC5C30094793F6B70F6387E7
:10083000E60011471305E00F639DE7061E200945FA
:1008400063992707130984004146A6854A859700C6
:10085000FB1FE78020B04146A68513058401970061
:10086000FB1FE78020AF383085469307F7FE93F7EC
:10087000F70F63E6F6041306C4033285C14532C69A
:10088000EF508FEC32469306C402CA852285EFF002
:100890001F993C2089CB22856244F240D2444249D0
:1008A00005616F1080073830C947E306F7FE3CB09A
:1008B0000145F2406244D244424905618280930777
:1008C0001005E317F7FE3C20E5D722856244F2408D
:1008D000D244424905616F10800A0945D9BF494594
:1008E000C9BF797152CC2A8A328522D44AD04ECEE1
:1008F00006D626D2AE8932899720FB1FE7800022D8
:10090000494405C9445949448DC49E206393270333
:10091000DC30A18B85EB0944B8309307B005631A2E
:10092000F7002685EF108002BC20ADCB9307C005F1
:10093000BCB0B2502285225492540259F249624A04
:10094000456182801739FB1F130949558327090028
:100950001304E00FF9DF9C47E9DF1384840122854B
:100960004146D2859700FB1FE780C09E8327090080
:1009700083A5040822869C47938505042E850A8753
:10098000814682972A844146CE850A859700FB1FBF
:10099000E780C0AD49D11374F40FBDBF9307E005E4
:1009A00041BF39C9011122CC26CA06CEAA842E84A1
:1009B000094595CD0D468D0528009700FB1FE78062
:1009C00060991C8570002C0093F7F70393E70704E8
:1009D00026855C85EF10F06E19E90D46A28568004A
:1009E0009700FB1FE78080A87D153335A000F240FB
:1009F0006244D2440561828009458280011152C45B
:100A00002A8A32854EC656C25AC006CE22CC26CA83
:100A10004AC82E8BB28AB6899720FB1FE780001048
:100A200009ED8944F24062444249B249224A924A5D
:100A3000024B2685D244056182805C592A89C544CF
:100A4000F5F34D45EF606F8D1374F50F5145EF6071
:100A5000CF8CE38809FC03C78901E36487FC9377A3
:100A6000F50FE3E0E7FC930530051305400897F028
:100A7000FA1FE780A05E232AA9022A84CD445DD113
:100A80001306400881459700FB1FE7802093A301D0
:100A9000040023014401230264012310540123268E
:100AA000340723240402A302040063070A002285FA
:100AB000EF00F060AA8419E18144ADB74A85EFF0F8
:100AC0004FBB8DB7397122DC06DE26DA4AD84ED606
:100AD00052D456D25AD05ECE62CC66CA0944630A5A
:100AE0000610BA84094463060710AA8B2E89328B3C
:100AF000368C9720FB1FE7806002AA8A514475C993
:100B000093053005414597F0FA1FE7802055AA89E3
:100B10004D4465C198309C2003CA340022075D8F84
:100B2000BC20620AC207D98F336AFA0083A78A02FF
:100B300063E647017D5709446398E70A63070900A4
:100B400083C74A000544898BC5C3214681450A8570
:100B50009700FB1FE7808086930C4C0093053005BF
:100B6000B3CC0C08668597F0FA1FE780204F2A89DE
:100B70004D443DC96286DA8511059700FB1FE78069
:100B8000A0931146A6854A859700FB1FE780C09277
:100B9000414693858A014E859700FB1FE780C091EF
:100BA00021478A866686CA854E85EF1010782A848A
:100BB0001DE521468A8528009700FB1FE780C08F2E
:100BC00021469385440028009700FB1FE780008A98
:100BD0008547631EF502D2855E85EF60EFAF4A85DB
:100BE00097F0FA1FE780A0544E8597F0FA1FE78030
:100BF0000054F25022856254D2544259B259225ABA
:100C0000925A025BF24B624CD24C216182800544C5
:100C1000F9B7797122D406D626D24AD04ECE2E8488
:100C20009397556063D607049734FB1F93848462BF
:100C3000A83097F0FA1FE78020682AC609CDEFF0A8
:100C4000DF94B24511E5A8209307F00F631FF5006C
:100C50002E85EF306FBA1319F468B25022549254B3
:100C6000F2494A85025945618280EF300FBEE5B7EF
:100C700013F9150063070900EFF00FB213491400D0
:100C8000E9BFE1DD854421A0850493F4F40FEFE092
:100C9000BFD7E3F4A4FCB3179028B3C90708E18FCA
:100CA000E5D74E85EFF08F80C167FD176305F5002E
:100CB000DD45EFF0CFA33349340145B79737FB1F2C
:100CC00023AE07169737FB1F23A807169737FB1F7E
:100CD00023A207169737FB1F9387075717070000B4
:100CE0001307675998C3170700001307072DD8C3C8
:100CF00017F7FFFF1307070E98C79737FB1F938758
:100D0000E753171700001307274098C31717000071
:100D1000130767FAD8C3171700001307E72398C70C
:100D200082809737FB1F83C72753A18B014789C751
:100D30001737FB1F130747519737FB1F23AEE70EEB
:100D4000014582809737FB1F83C70751918B01476D
:100D500089C71737FB1F1307674E9737FB1F23AB56
:100D6000E70C01458280011106CE2AC6EFF01FF57F
:100D7000324599459737FB1FA38FA74CEFD0AFE8BB
:100D8000F24017F5FFFF1305C51D05616FE07FC831
:100D90001C5599C321458280011122CC26CA2A8480
:100DA000AE84130500049305300506CE97F0FA1FB4
:100DB000E780C02A08D469C513060004A68597F009
:100DC000FA1FE78020597454B82A93778700F5C733
:100DD0001C54BC23A18BF5C383270408D5E39305DA
:100DE00030051305001097F0FA1FE7802027AA8727
:100DF0002320A4080D45D1C774549C309832D9C71C
:100E00003337E0000E07936707016C545CB0B829D4
:100E1000058B19CB1854854638230D8B6316D700E4
:100E200078201367170078A00327040809C77820E3
:100E30001367870078A005476396E70C9304840046
:100E400041468145268597F0FA1FE78020574146A5
:100E500081451305840197F0FA1FE7802056130699
:100E6000C4033285C14532C6EF500F8E8327040874
:100E70003246BDC72285EF0090309307000525CD8F
:100E80002145F2406244D24405618280A14735FF8A
:100E9000BC20918B91E7BC2A918B99E38547B5B72C
:100EA0009820942295473307F70297D7010093873C
:100EB000A7C9BA97B6979C2389BF9C3081C7903247
:100EC000E14721F6BC205D8F118B69DB98209547A7
:100ED00094223307F70297D701009387A7C8D1BFA1
:100EE00022859306C402A685EFF06FB32285EF003A
:100EF000D02259F5C1470A203CB08145EF50DFE7C9
:100F0000014541B713F7870135CFC18B93048400A6
:100F10004146B1C78905268597F0FA1FE7808043CF
:100F2000414681451305840197F0FA1FE780004987
:100F30007C201306C403328593E747007CA0C1459B
:100F400032C6EF506F8083270408324685C322855E
:100F5000EF00F02215F5930720053CB055B7814509
:100F6000268597F0FA1FE78060455DBF9306C402AF
:100F7000A6852285EFF0AFAA2285EF00101ACD4793
:100F800069DDFDBD094785456388E70093F7D70F05
:100F900011476396E70089450A20EF50FFDD7C206A
:100FA00093E747007CA08327040881C793071005B7
:100FB0006DB7C5475DB73C2163800724797122D4A2
:100FC00006D626D24AD03C31130750052A84639DA9
:100FD000E706034975001306C503C1459357390059
:100FE000AA973285842732C6EF401FF69737FB1F3A
:100FF00083A7C7EAA1C79C47B1C303250408137997
:1010000079003246B3D62441858A93050504180831
:1010100093E606081305050882971375F50F19ED79
:1010200041460C081305C40297F0FA1FE78080328E
:101030002285EF00900E930760053CB0B250225419
:101040009254025945618280130710026392E702AD
:101050001C5503270508DE2361E713F7071069C352
:1010600078555A2B1377071045CF930770023CB081
:101070003C3013077002639BE70C3C5885E39305F3
:101080003005714597F0FA1FE78040FD28D819C553
:101090007146814597F0FA1FE78040322458B1C469
:1010A000BC2C89E72285EFF0CFA2A8AC2858814557
:1010B000414697F0FA1FE780603028583D472C2DB5
:1010C0009387F5FF93F7F70F6364F700EF40DFE7CF
:1010D000EF302F823C58A1458AAB13852701EF40A2
:1010E000BFE62C580A20EF001033930780020A2035
:1010F0003CB09720FB1FE78060A2414609C57E25D2
:1011000013D617003E962254B25092540259173506
:10111000FB1F034555140606854545616F300F9941
:1011200013F7072009CB78545A2B1377072001C7F0
:10113000930790022DBF93F707409DDB7C54DE2B75
:1011400093F7074095D79307B00215B713078002AE
:10115000639FE7023C5899C78E2B0A20138627010C
:10116000EF00D0301C54DE2313F7072011C778544A
:101170005A2B1377072035EF93F70740A5CB7C5404
:10118000DE2B93F70740BDC39307B0028DB713075B
:101190009002639BE700EF504F8AAA850A20EF0078
:1011A000F02B9307A002A1B71307A0026396E702F2
:1011B000EF500F88AA85854701456384F500814576
:1011C00005452EC6EF504F842A86B2450A20EF000F
:1011D00090251C54DE234DB71307B0026398E70037
:1011E000EF504F86AA850A20EF00B02B9307F0023C
:1011F000A9B593079002E5BD8280411122C44059F0
:1012000026C206C67C54AA84DE2B13F7071011C72A
:1012100018545A23137707100DE313F7072011C74B
:1012200018545A231377072009EB93F707408DCB07
:101230001C54DE2393F7074085C7930710023CB088
:101240002285EFF05FD738309307F002631EF70076
:101250002244AA20B2409244814541016FE03FC937
:101260009307F0023CB0EDB7B240224492444101F2
:101270008280397122DC405926DA4AD84ED606DE01
:101280002A89AE84B289630604382A211E2063911C
:10129000A7123C20638A07389387E5FF93F7F70F7F
:1012A0002D476363F73817D701001307678DB3C75E
:1012B000E7209C43BA97828722856254F250D25429
:1012C0004259B259B28521616FF09FAC4146CE853B
:1012D0001305C40497F0FA1FE780C0072285BD25D7
:1012E000383093074005631AF700930790053335AC
:1012F000A000931435003CB06DA893066005D1475B
:10130000E317D7FE9307A005DDB71309C4054A8587
:101310004146CE8597F0FA1FE780C00303250408F5
:101320005DC53C30130790056397E7002285452D86
:101330009307E005A5A81307A0056394E7087C3090
:1013400013D73700229714279D8BB3D6F640858A92
:101350009737FB1F83A787B493E60608B1CB9C475A
:10136000A1CB9305050818084A8613050504829742
:101370001375F50F15ED41460C081305C40497F0DD
:10138000FA1FE780A00E7C304D47850793F7F70FD3
:101390007CB0E36DF7F885451735FB1F0345B5EBCA
:1013A0009710FB1FE7804061930750053CB031A8C0
:1013B000A144F25062544259B2592685D254216157
:1013C00082801307C005E383E7F68144DDB7930904
:1013D00084004A86CE8522851408EFE05FE441460A
:1013E0009305C404080897F0FA1FE780200871D11C
:1013F0008A861306C403CA854E85EF10A069A144EE
:101400000DE12285EFE0FFEC2A870A209737FB1FCA
:1014100083A707E4814601468A858297B334A000FA
:101420008E0493072002C1BD0C22EFE05FAC71BFB8
:101430003830930720026319F71E7C5889EB930517
:101440003005714597F0FA1FE78040C168D86858A9
:10145000630C051C4146CE8597F0FA1FE78080EFAC
:1014600064582285EFE0FFE6A8AC930730023DBF49
:101470003830930730026319F71A1E226858214644
:10148000938529001EA9490597F0FA1FE78080EC93
:101490007C54DE2B13F727002DC718545A23098BD1
:1014A0002DC39307400219B7383093074002631DDC
:1014B000F7163C5C81EB85455D4597F0FA1FE780A8
:1014C000E0B928DC285CE30205F083C70900414647
:1014D000CE857CA997F0FA1FE780C0E793075002FA
:1014E000F1B53830930750026310F714285C1946A1
:1014F00093851900410597F0FA1FE780A0E57C5419
:10150000DE2B918B95CF1C54DE23918B95CB9307CB
:10151000600269BD7C5C89EB93053005514597F00D
:10152000FA1FE780A0B368DC685CE30305E8414686
:10153000CE8597F0FA1FE780E0E17C5C7D5798CB81
:101540004A85EFF09FCB51B503250408130600042C
:10155000CE851305050497F0FA1FE780A0DF2285EA
:10156000EFE03FC83C30130700056395E7009307A1
:1015700040052DBD13071005E38FE7E01307200595
:10158000E395E7E49737FB1F83A74791E38207E2E0
:101590009C47E38F07E08325040893048400180820
:1015A00093850508814626862E8582970A20100895
:1015B000A685EF505F859307B005CDBB3830930704
:1015C000E0056313F7068325040841464E8597F02E
:1015D000FA1FE780A0E9AD44E30D05DC032504080C
:1015E0004146CE8597F0FA1FE780C0D62285EFE00E
:1015F0005FCE2A872C580A209737FB1F83A747C541
:10160000814601468297B334A0008E0493071002EE
:10161000DDB1AD47E39BF5DA14222E2113066500F8
:101620000821EF40FFF955B39D4461B3AA870945EE
:1016300041C6D9C11CA29C211CB29C313CA2BC2138
:101640003CB2BC31A30206005CA2DE2193D78748DE
:101650005CB2DA211377072001C793E727005CB259
:10166000DE2193F7074089C75C3293E747005CB2FD
:10167000DE211317B028F98F89C75C3293E7870002
:101680005CB223030600DE21858B7CA2DA21098B64
:1016900001C793E727007CA2DE21918B89C77C22BA
:1016A00093E747007CA2DE21A18B89C77C2293E7C8
:1016B00087007CA20145828082802E86AA8505450E
:1016C0006FF0DFF62E86AA8509456FF03FF68DC5CF
:1016D0002A87094505C7411106C6AE878D4694A1E4
:1016E000138517004146BA8597F0FA1FE78080C638
:1016F000B2400145410182800945828082808DC5CA
:101700002A87094505C7411106C6AE87914694A1AF
:10171000138517004146BA8597F0FA1FE78080C30A
:10172000B2400145410182800945828082808DC599
:101730002A87094505C7411106C6AE87994694A177
:10174000138517004146BA8597F0FA1FE78080C0DD
:10175000B2400145410182800945828082809DC955
:101760002A87094515CB411106C69D4694A116232B
:10177000AE871385370094B116232146A182B4A108
:101780009305270097F0FA1FE780C0BCB2400145DF
:10179000410182800945828082808DC52A87094562
:1017A00005C7411106C6AE87A14694A1138517004F
:1017B0004146BA8597F0FA1FE780C0B9B2400145AB
:1017C0004101828009458280828085C92A87094536
:1017D0001DC7411106C6A54694A11423AE871385E3
:1017E000270094B119469305170097F0FA1FE78078
:1017F00060B6B24001454101828009458280828005
:101800008DC52A87094505C7411106C6AE87A94679
:1018100094A1138517004146BA8597F0FA1FE78017
:1018200060B3B240014541018280094582808280D7
:1018300095C52A8709450DC7411106C6AE87B14631
:1018400094A11385170013060004BA8597F0FA1FB8
:10185000E78040B0B2400145410182800945828065
:1018600082808DC52A87094505C7411106C6AE8706
:10187000B54694A1138517004146BA8597F0FA1F23
:10188000E78040ADB2400145410182800945828038
:101890008280AA87094581C999C7154798A19C23C9
:1018A00001459CB182808280AA87094581C999C778
:1018B0002D4798A19C2301459CB1828082800DC553
:1018C0005D718A8586C6A2C42A84EFE09F8D0A20B6
:1018D0000A8697060000938686DE9D45EFE0CFFFDF
:1018E000B640264461618280054582800DC55D71E8
:1018F0008A8586C6A2C42A84EFE0BF8A0A200A86A7
:1019000097060000938646DC9D45EFE0EFFCB6406D
:10191000264461618280054582805D71A2C4930581
:10192000C5022A8441460A8586C697F0FA1FE780D9
:1019300060A20A200A8697060000938686D9C545CC
:10194000EFE08FF9B6402644616182805D71A2C4E8
:101950009305C5032A8441460A8586C697F0FA1F77
:10196000E780409F0A200A8697060000938666D982
:10197000C545EFE06FF6B640264461618280972747
:10198000FB1F83A7A751A9CB9C435D71A2C486C648
:101990002A841305E00F8DCF032504089305050C59
:1019A00013050508829783250408130600040A8599
:1019B0009385050897F0FA1FE780C0990A209706DB
:1019C0000000938626E70A8693051004EFE0CFF027
:1019D000B6402644616182801305E00F8280317138
:1019E00022DD2A840A2126DB06DF4AD94ED752D5CA
:1019F00056D35AD15ECF62CD66CB9710FB1FE780DE
:101A0000E0113C58AA8489EB93053005714597E0B5
:101A1000FA1FE780A06428D82858CD4715C9714619
:101A2000814597F0FA1FE780609903290407228512
:101A3000EFE03F8A230DA9003C201729FB1F130963
:101A4000E94563820712832709008DE39307E00FBE
:101A5000FA506A54DA544A59BA592A5A9A5A0A5BBD
:101A6000FA4B6A4CDA4C3E852961828003AC07014F
:101A7000E30E0CFC032B0408EF408FFBAA8B0145FF
:101A8000EF408FF8DC303458130B0B029309C4037A
:101A9000130AC405938A64002A8736C0B337F0005E
:101AA000930801045688B33670015286CE855A8554
:101AB000029C1C54B8232307E1029833A306E102D9
:101AC0009C232306F10283270900C9D383AB470176
:101AD000E38E0BF6DC30B337F0003ECEEF404FF52F
:101AE0002A8B0145EF404FF203270408F2472AC032
:101AF0003AC2B338600156887810930684004E8647
:101B0000D2858800829B7C54B82B2305E102983350
:101B1000A304E1029C232304F1028327090003AB01
:101B20004701EF40EFF02A890145EF40EFED83C810
:101B300054009C082A883EC2B3381001B3372001F4
:101B40003810930684015286CE8556C08800029BC9
:101B50000A2097060000938606D19008C545EFE05D
:101B6000AFD7AA87F5B5D43083270900032B040823
:101B7000B336D00083AC070136CEEF406FEBAA8BB3
:101B80000145EF406FE83C58F246130B0B02130A75
:101B9000C4059309C403938A64002A889308010446
:101BA0004E86D2853EC05687B33770015A85829CD7
:101BB0001C54930B0103B8232307E1029833A306B7
:101BC000E1029C232306F1028327090083AC47012D
:101BD000DC30B337F0003ECEEF408FE52A8B014575
:101BE000EF408FE2F2472AC0B33860015688781080
:101BF000930684004E86D2855EC28800829C83252F
